:020000040800F2
:1000000000200010859302085DD80108FDE2000879
:1000100059D8010855D8010851D80108000000003E
:100020000000000000000000000000004DD80108A2
:1000300049D801080000000045D801084DE100083A
:10004000ED930208ED930208ED930208ED93020888
:10005000ED930208ED93020809390008353A0008CB
:10006000F9390008BD39000881390008B54B00088E
:10007000A54B0008954B0008854B0008754B000800
:10008000614B00084D4B0008ED930208ED93020808
:1000900045DB0108ED930208ED930208453900089D
:1000A0003DDA00088DDA0008ED9302089DDA0008B9
:1000B0007DDA00086DDA0008ED930208ED9302087E
:1000C000ED930208ED930208ED930208ED93020808
:1000D000ED930208ED930208ED93020881E1000818
:1000E000CF380008ED93020835D80108ED930208D7
:1000F0004DDA0008ED9302085DDA0008ED9302087E
:10010000000000000000000000000000ED93020865
:10011000ED930208ED930208C9460108AD460108B7
:10012000394B0008254B0008114B0008FD4A000818
:10013000E94A0008ED9302080000000000000000FA
:10014000ED930208ED930208ED9302080000000011
:10015000000000000000000000000000000000009F
:100160000000000000000000ED930208ED9302087B
:10017000ED930208000000000000000000000000F5
:0801800000000000ED930208ED
:100188002DE9F04FB0F908502DED028B0D81EDB23D
:10019800382D8FB00C4600F0358480462ED9802D3E
:1001A80000F0928079D8522D00F0F18040F20A8454
:1001B800542D00F059846E2D40F00281754B0A6869
:1001C8001B88754DFF2BA8BFFF23511C216013709E
:1001D800A96881F3100189B2204604F030F86F4B0A
:1001E8002046198804F02BF8296801F30F0189B219
:1001F8002046012504F023F82B4647E0042D00F0A3
:10020800278440F2C783202D00F0A58040F2E583C3
:10021800242D00F03584282D40F0D2800B68DFF8BB
:100228009C815F4E591C022221601A7023680627A0
:100238005A1C22601F7023680A22591C21601A70F8
:10024800236801255A1922601D70B8F8001020464D
:1002580003F0F5FFB8F80210204603F0F0FF23681A
:100268005A1922601F7023685022591921601A7088
:1002780023680022591921601A703188204603F03A
:10028800DEFF7188204603F0DAFF2B46284663819B
:100298000FB0BDEC028BBDE8F08F822D2ED0C0F0E0
:1002A8000484A02D00F0F583FE2D40F089803D4D9B
:1002B80005F1080635F8021B204603F0C0FFAE42E0
:1002C800F8D101252B46E1E7374B1D780B3D15F09A
:1002D800FF05F6D0354F00220A2621683B88481CC6
:1002E80020600E702168FF2B02F10102A8BFFF23D6
:1002F800481CAA4220600B70EFDBE2E70B682C4A2F
:10030800254D11782B4A581C2060197011892046F8
:1003180003F095FF1F4B22681B88FF2B02F1010198
:10032800A8BFFF2321601370A96881F3100189B267
:10033800204603F084FF296801F30F0189B22046A3
:1003480003F07DFF1C4B22681978531C012523609C
:100358002B4611709AE70B68164D591C6A78216074
:100368001A7023682A78591C21601A702368AA78A1
:10037800591C21601A702989204603F060FF236800
:100388006A79591C21601A702268A979DDE70A6820
:100398000021DAE7B43C0020103C00207050002017
:1003A800D0290020A83C0020BC4400203840002070
:1003B800CA3C002078510020B73E0020F0370020CA
:1003C800A5F10A03E72B00F2EA80DFE813F07007D3
:1003D800E800E800E800E800E800E800E800E800D5
:1003E800E800E800E800E800E800E800E800E800C5
:1003F800E800E800E800E800E800E800E800AB07EB
:10040800E800E800E8008307E800E800E8003008B2
:10041800E800EF07E800D607E800CA07E800A008E8
:10042800E8007A08E8000C04E800E800E8000404A2
:100438007108E8006D08E800E8006408E8003A0878
:10044800E800E800E800F703E800E800E800E80052
:100458005407E8003207E8002007FC06E800E80037
:10046800E800E800E800E800E800C706E8009C06A5
:10047800E8006B06E8001506E800D205E800E80089
:10048800E800E800AC057105680537052505E800B2
:10049800E8000C052109E800CE08B108E800E800EA
:1004A800E800E800A508E800E8004009E800E800DE
:1004B800E8002F096209FB04BC04E800E800E80032
:1004C800AB04E800E8005E04E800E800E800E800A3
:1004D800E800E800E800E800E800E800E800E800D4
:1004E800E800E800E800AC05E800E800E800E800FB
:1004F800E800E800E800E800E800E800E800E800B4
:10050800E800E800E800E800E800E800E800E800A3
:10051800E800E800E800E800E800E800E800E80093
:10052800E800E800E800E800E800E800E800E80083
:10053800E800E800E800E800E800E800E800E80073
:10054800E800E800E800E800E800E800E800E80063
:10055800E800E800E800E800E800E800E800E80053
:10056800E800E800E800E800E800E800E800E80043
:10057800E800E800E800E800E800E800E800E80033
:10058800E800E800E800E800E800E800E800E80023
:10059800E800E800E800E800E80051042604742DAB
:1005A80000F0E382772D00F0CE82292DD8F8006084
:1005B80000F0ED82392D01F05D87212D01F034879F
:1005C800D8F804200B3D931BEF2D01F2DF8001A129
:1005D80051F825F0CD1C000895170008951700085C
:1005E8009517000895170008951700089517000833
:1005F8009517000895170008951700089517000823
:100608009517000895170008951700089517000812
:100618009517000895170008951700089517000802
:1006280095170008951700089517000895170008F2
:1006380095170008271C0008951700080D1C0008CE
:1006480095170008EB1B0008951700089517000878
:1006580095170008BF1B000895170008591B0008CC
:1006680095170008211B000895170008F91A0008BB
:1006780095170008E51A000895170008831A00085E
:1006880095170008E1190008951700089517000844
:100698009517000895170008CB0200089517000861
:1006A800C11900089517000895170008A519000832
:1006B800951700084D1900089517000895170008A8
:1006C8009517000895170008951700089517000852
:1006D8009517000895170008C11800089517000815
:1006E80075180008951700089517000837180008AE
:1006F8009517000895170008951700089517000822
:10070800951700089517000895170008932000080A
:10071800951700080D20000895170008671F0008A6
:1007280095170008AD1E0008951700087F1E0008E1
:100738005F1E000895170008951700089517000810
:1007480095170008951700089517000895170008D1
:1007580095170008951700089517000895170008C1
:1007680095170008951700089517000895170008B1
:1007780095170008951700089517000895170008A1
:100788009517000895170008951700089517000891
:100798009517000895170008951700089517000881
:1007A8009517000895170008951700089517000871
:1007B8009517000895170008951700089517000861
:1007C8009517000895170008951700089517000851
:1007D8009517000895170008951700089517000841
:1007E8009517000895170008951700089517000831
:1007F8009517000895170008951700089517000821
:100808009517000895170008951700089517000810
:100818009517000895170008951700089517000800
:1008280095170008951700089517000895170008F0
:1008380095170008951700089517000895170008E0
:1008480095170008951700089517000895170008D0
:1008580095170008951700089517000895170008C0
:1008680095170008951700089517000895170008B0
:1008780095170008951700089517000895170008A0
:10088800951700082F1E00089517000895170008EF
:100898009517000895170008951700089517000880
:1008A8009517000895170008951700089517000870
:1008B8009517000895170008951700089517000860
:1008C8009517000895170008D31D0008951700080C
:1008D8004322000895170008952100087B2100088D
:1008E8005F21000895170008B91D00089517000832
:1008F8008F1D0008951700082F1D00089517000880
:10090800071D000895170008951700081518000816
:10091800E1170008CD1700089F1700087117000895
:100928004F17000895170008951700089517000835
:1009380095170008951700089517000895170008DF
:1009480095170008951700089517000895170008CF
:1009580095170008951700089517000895170008BF
:10096800951700083517000895170008951700080F
:10097800CD16000895170008951700089517000868
:10098800951700089517000895170008951700088F
:10099800811C0008022D00F0CD8000F2C080012DDE
:1009A8007FF40EAD0B680022591C21601A70236871
:1009B8005A1C22601D7022682421531C23602B4678
:1009C800117063E4442D7FF4FBAC002A3FF479AC4A
:1009D800BE4B136001252B4658E4052D7FF4F0AC7F
:1009E8000B22BB49204603F0FCFB0822B9492046EC
:1009F80003F0F7FB01250722B749204603F0F1FB76
:100A08002B4643E40A68B54B0125511C216015703B
:100A18002268052150192060117022680A21501996
:100A2800206011702268002150192060117022681E
:100A3800197850192060117022685978501920606F
:100A4800117022689978531923602B4611701DE4A0
:100A58002A46A349204603F0C4FB0021204603F0A0
:100A6800EEFB2268002170E40B6800215A1C22600A
:100A7800197022680125531923602B46117005E46B
:100A8800984B19682046012503F0C2FB2B46FFF757
:100A9800FDBB954B0846196803F0BAFB934B2046FB
:100AA800196803F0B5FB924BEBE7924B1E780A3EB0
:100AB80016F0FF063FF405AC8F4B904F1E4403F130
:100AC80001080A2314E0502B01F0D383002529469E
:100AD8002268501C20602046137003F0B0FB2946A2
:100AE800204603F0ACFBB0453FF4EBAB18F8013BF4
:100AF8000A2BE8D1824A9568116805EB85054FF6FF
:100B0800FF726D009542A8BF15469142A8BF1146D5
:100B180025EAE57521EAE171ADB289B2D8E70B683B
:100B280003215A1C2260197023680222581C206075
:100B38001A709EE7042273492046012503F051FBF1
:100B48002B46FFF7A3BBD8F80030D8F804209A4208
:100B58001EBF5A1CC8F8002019786B4A08BF00212C
:100B6800204620F079F8FFF7ACBBD8F80030D8F869
:100B780004209A421EBF5A1CC8F800201978634AFC
:100B880008BF0021204620F067F8FFF79ABB731CC6
:100B9800C8F8003033780A2B01F0A884502B40F0B5
:100BA800F586404603F00DFB594E3080404603F071
:100BB80008FB012570802B46FFF768BB23680025DA
:100BC8005A1C2260294620461D7003F021FB294645
:100BD800204603F01DFB00212046012503F018FBE9
:100BE8002B46FFF753BB4B4D4B4E05F1180795F9B4
:100BF800023096F906209A4201F0F88396F90E2001
:100C08009A4201F0F38396F916209A4201F0EE8396
:100C18000835AF42EBD1FFF754BB404B03F17005E9
:100C280022681978501C2060117022685978501C6D
:100C38002060117022689978501C20601170226819
:100C4800D978501C2060117022681979501C2060D6
:100C5800117022685979501C2060117022689979A6
:100C68000733501C9D4220601170D9D1FFF729BB72
:100C78002B4D2046E98903F0E2FAA989204601258F
:100C880003F0DDFA2B46FFF701BB2368194F591C07
:100C98003A7821601A703B78002B3FF412AB00259C
:100CA800EEB230461BF030F823684278591C2160B8
:100CB80030461A701BF028F80189204603F0BFFA65
:100CC8003B7801359D42EBDBFFF7FBBA4DC80008C6
:100CD8001CE1020828E10208980903083F330020B4
:100CE800113F002090340020ACF7FF1FB0F7FF1F22
:100CF800B4F7FF1FBC440020BCBB0208D429002065
:100D08009C29002014E10208C5FF01080D0B020808
:100D1800D02900204C5700209C4E00202C25002074
:100D2800003800209B4D2046298A03F088FA698AFA
:100D3800204603F084FAA98A2046012503F07FFAA9
:100D48002B46FFF7A3BADFF89CE20027FEB27146F4
:100D580000232268501C206016702268501C2060F6
:100D68001370226811F8010F0133551C062B2560FA
:100D78001070EED10137062F0EF1060EE6D1864926
:100D880000232268501C206017702268501C2060C5
:100D98001370226811F8010F0133551C0B2B2560C5
:100DA8001070EED123687D49581C072220601A7004
:100DB80023680022581C20601A70226891F8F010ED
:100DC800FFF7C3BA2368764A76491078764A5D1CDD
:100DD8002560187023689278581C20601A70226861
:100DE8008978FFF7B2BA714D2046298803F027FAAF
:100DF8006988204603F023FAB5F904306C49DA17FC
:100E080081FB0313C2EBA30399B22046012503F02B
:100E180016FA2B46FFF73ABA664E3378002B3FF4A2
:100E280050AA654F002537F8021F204603F007FA3D
:100E3800337801359D42F6DBFFF743BA5F4D604ECC
:100E4800DFF8A481DFF8A4919FED5E8A05F1200701
:100E58000EE0FCEEE77ACDED017ABDF804102046ED
:100E6800043503F0ECF9BD4206F118063FF429AA4F
:100E7800717C0029F3D098F80030D5ED007A012B69
:100E8800E7D1D9F80030DB0441F10A83F5EE407A66
:100E9800F1EE10FA41F0528340F2DC51DFE7102204
:100EA80049492046012503F09CF92B46FFF7EEB986
:100EB800464B9B8AB3F5006F01F20883B3F5806F48
:100EC80001F22583B3F5007F34BF01270227404D87
:100ED80005F10C0655F8041B91FBF7F1204689B281
:100EE80003F0ADF9B542F5D13A4D3B4F05F10C068B
:100EF800B5EC010AD7ED087A80EE270A28F0CCFC79
:100F080081B2204603F09BF9AE42F1D1334D05F191
:100F18000C0655F8041B204689B203F090F9AE423E
:100F2800F7D1FFF7CEB90023DFF8C490DFF8C4B0DB
:100F38000493039305930693984601214FF6FF7A8D
:100F480007E008F10108B8F10B0F01F0968119F9D3
:100F5800011F4F1C4AFA08F3F3D0DE07F1D5BBF89E
:100F6800003043FA08F3D807EBD505A803F04CFB8B
:100F7800E7E723680C4A0B49D078194A5D1C2560BD
:100F8800187023685279581C20601A702268C97832
:100F9800FFF7DBB96C4B002057500020744F00203E
:100FA800C44600201038002000380020883F002068
:100FB80067666666903F00203E4500204036002068
:100FC800AC4A00200000404230360020403F00205C
:100FD800783F002060490020D8460020B03B002020
:100FE800F852002033500020904B00206C4900201C
:100FF800C0BB0208725000200021204603F01FF9F0
:101008000021204603F01BF90021204603F017F9C0
:101018002368B94D00265A1C22601E7023682A686E
:10102800591C92F82C2021601A7023682A68591CD0
:1010380092F8362021601A7023682A68591C92F8A1
:10104800372021601A7023685A1C22601E7023689A
:101058005A1C22601E7023685A1C22601E702B685E
:101068002046598F03F0EBF82B682046198F03F0C0
:10107800E6F82A68236892F82E20591C21601A7015
:1010880023685A1C22601E702B682046598E03F074
:10109800D6F82B682046998E012503F0D0F82B4608
:1010A800FFF7F4B8954E23687279934D591C216067
:1010B8001A702B682046198C03F0C1F82B6820465B
:1010C800D98B03F0BCF87189204603F0B8F8B189D0
:1010D800204603F0B4F82B682046598C03F0AFF88B
:1010E8002B682046998C03F0AAF8F189204603F072
:1010F800A6F8318A204603F0A2F82B68226893F8F4
:101108002610FFF722B97D4FFB78002B01F0D18123
:1011180023680822591C21601A7023680122991833
:1011280021601A702368764D591C2A7921601A703B
:101138002368AA78591C21601A702988204603F070
:101148007EF8E989204603F07AF82368FA79591C71
:1011580021601A702268E978FFF7F7B825F0C6FC15
:10116800FF28064601F0B5810EA9002501F82D5D7E
:101178000DF10A008DF80A5025F098FC0EA800F829
:101188002C5D25F087FC0EA800F8245D25F076FC80
:1011980023685A1C22601E7023689DF80A20591C77
:1011A80021601A7023689DF80B20591C21601A7061
:1011B80023689DF80C20591C21601A7022689DF83C
:1011C8001410FFF7C2B823684E4E01255A1C22603E
:1011D8001D702368B278591921601A7026F016FE1E
:1011E8002368494A49495F1927601870B1F9001006
:1011F800B2F9000003F0ACF923685A19226018709C
:101208003188204603F01BF82B46FFF73FB82368C8
:1012180000255A1C22601D7023685A1C22601D700C
:1012280023685A1C226029461D70204602F0F0FFF0
:10123800D1E4374E3378002B3FF443A8354F0025CF
:10124800B846236817F81520591C21601A7098F8B9
:10125800011001EB810101EB810101F2EE2189B25C
:10126800204602F0ECFF337801359D4208F1020870
:10127800E7DBFFF726B82368274D591C2A79216038
:101288001A7023686A79591C21601A7029882046C7
:1012980002F0D5FF2368AA79591C21601A70698861
:1012A800204602F0CCFF2268E979FFF74EB81B4DC3
:1012B800284627F0E5F900287FF703A82B460544C0
:1012C800226813F8011B501C9D4220601170F7D151
:1012D800FEF7F7BF124D2046298802F0B0FFA98813
:1012E800204602F0ACFF29892046012502F0A7FF1D
:1012F8002B46FEF7CBBF00BF183F0020C446002096
:101308006C4B002070340020A05D0020A25D0020FE
:10131800903F002054560020A03B0020DC370020DE
:10132800BC2C0020AE4D05F1500628781FF0E8FCD3
:101338002368027A591C21601A7023686A78591C3C
:1013480021601A702368AA78591C21601A702368D2
:10135800EA780435591CAE4221601A70E5D1FEF7CF
:10136800B0BFA04D05F1800655F8041F204602F0D5
:101378004FFFB542F8D1FEF7A4BF9B4D05F14006DB
:10138800B5F88010204602F05AFF236895F88220AD
:10139800591C21601A70236895F883200435591C5C
:1013A800AE4221601A70EBD1FEF78BBF8F4D2368D8
:1013B8002A7A591C21601A70A98B204602F03FFF37
:1013C800298B204602F03BFF698B204602F037FF4D
:1013D8002368EA7C591C21601A70A98C204602F007
:1013E8002EFFE98C204602F02AFF2368AA7F591CA9
:1013F80021601A70236895F82020591C21601A7002
:10140800698C204602F01BFF2368EA7A591C216088
:101418001A70E968204602F0FBFE23682A7C591CF2
:1014280021601A70226895F82110FEF78EBF704B64
:1014380022681978501C2060117022685978FEF7CC
:1014480084BF23686A4A6B4D11786B4A581C206028
:1014580019701168204602F0DBFE2368634A591CA4
:10146800127A21601A702988204602F0E8FEA988BD
:10147800204602F0E4FE2989204602F0E0FE002121
:10148800204602F0DCFE01250021204602F0D7FEAE
:101498002B46FEF7FBBE082254492046012502F0E0
:1014A800A0FE2B46FEF7F2BE544B22689978C1E79E
:1014B80022680121531823600D460B461170FEF770
:1014C800E5BE4F4B03F15A0522685979501C20603C
:1014D800117022681978501C2060117022685978A0
:1014E800501C2060117022689978501C206011707F
:1014F8002268D978501C2060117022681979063347
:10150800501C9D4220601170DED1FEF7DABE374BC9
:101518002268597DFEF719BF3A4952232268501CA8
:101528002060137011F8013F002BF7D1FEF7C9BEF8
:10153800354D00232268286803EB4301561C405CA4
:10154800266010702A6820680A44461C5278266073
:1015580002702A6820680A4401339278411C0A2BD9
:1015680021600270E6D1FEF7ACBE284D23682A68D8
:10157800591C127821601A702B6822689978531CBC
:101588002360002311702A6821681A4401335279B4
:10159800481C032B20600A70F5D123682A68591C5F
:1015A800127A21601A7023682A68591CD27821603F
:1015B8001A7023682A68591C127921601A702B68DE
:1015C8002046598902F03BFE23682A68591C527A42
:1015D80021601A702B6822685978FEF7B6BE00BFE2
:1015E80040380020704F0020744F0020B84E002073
:1015F8003C380020BC2C0020903400201C380020EF
:10160800753A00208CBB0208183F0020045D0020BA
:10161800BC4B2046196802F0FBFDBB4B20461988DD
:10162800012502F00CFE2B46FEF730BEB74D2046D2
:10163800298802F004FE6988204602F000FEA98885
:101648002046012502F0FBFD2B46FEF71FBEB04DDC
:1016580005F16006A988204602F0F1FDE9882046D8
:1016680002F0EDFD2989204602F0E9FD2368AA7AF7
:10167800591C21601A702368EA7A591C21601A7073
:1016880055F80C1B204602F0C3FDB542E2D1FEF727
:1016980018BE22689F4B9D491878551C256010700C
:1016A80022685878551C2560107022689B78501C59
:1016B80020601370C9882046012502F0C0FD2B4622
:1016C800FEF7E4BD731CC8F8003033780F2B5DD8E3
:1016D800B21CC8F80020C3EBC3038F4A7178D154F9
:1016E800F11CC8F800101344B2785A70321DC8F8BB
:1016F8000020F2789A70721DC8F800203279DA70EA
:10170800B21DC8F8002072791A71F21DC8F80020BD
:10171800B2795A7106F10802C8F80020F2799A7174
:10172800012510F065F92B46FEF7B0BD404602F0E2
:1017380048FD7A4EF081404602F043FD0125B08114
:101748002B46FEF7A3BD404602F03BFD744E3082A7
:10175800404602F036FD7082404602F032FD012517
:10176800B0822B46FEF792BD3346721CC8F80020A3
:1017780013F8020BC8F80030F31C7178C8F8003071
:10178800B27821F0ADFA00287EF49BAD4FF0FF351A
:101798002B46FEF77BBD3346721CC8F80020614A11
:1017A80013F8021B1170C8F800305C4A7378937004
:1017B800F31CC8F800305C4BB2789A7001252B46B0
:1017C800FEF764BD594B5A4918684E22012527F087
:1017D800EFFE2B46FEF75ABD3246731CC8F80030A0
:1017E8004C4B12F8021B1970C8F8002072785A7016
:1017F800F21CC8F80020B2789A70404602F0E1FC6A
:10180800424B0125D8802B46FEF740BD404602F0EA
:10181800D8FC3E4E3080404602F0D3FC70804046F3
:1018280002F0CFFC0125B0802B46FEF72FBD414BBF
:101838001B78012B3EF645AD731C3146C8F80030C5
:101848003D4F11F8023BBB70F31CD21AC8F80010C8
:10185800012A7078C8F8003040F34B87404602F000
:10186800B0FC012538802B46FEF710BD731CC8F864
:1018780000303778112F89D8B31CC8F800302F4DA5
:10188800737805F81730404602F09BFC40F6CA030F
:101898009842A8BF184640F2EE23984205EB47014C
:1018A800B8BF18460125A0F2EE222B46192092FB5C
:1018B800F0F24A70FEF7EABC3346721C204DC8F8B5
:1018C800002013F8022B2A71C8F8003073786B7166
:1018D800404602F076FCD8F8003028805A1CC8F838
:1018E80000201B78AB71404602F06BFCD8F8003042
:1018F80068805A1CC8F800201B78EB7101252B461C
:10190800FEF7C4BC2C2200204C1F0020902700208A
:1019180038240020F83700202C250020003800202B
:101928006C4B0020C446002010380020183F0020CF
:1019380050BF02086D340020703400205456002037
:10194800A03B0020731CC8F80030D24B3278D24F2D
:101958001A7000233B60404602F01CFCD8F80020B7
:101968003B68CE49CE4D0343501C3B60C8F800008D
:1019780013780B72404602F024FC2860404602F0BF
:1019880020FC6860404602F01CFCA860404602F05B
:1019980018FC404602F015FCFEF793BCC14B06F15B
:1019A80008020136C8F8006016F8011C03F8011F88
:1019B800B242F6D1FEF785BC3346721CC8F8002047
:1019C800B94A13F8021B9170C8F800307378537045
:1019D80001252B46FEF75ABC0722B3FBF2F2C2EBF5
:1019E800C2055B1B7FF4D2AED2B2571EFFB2002AEB
:1019F8003EF467ACDFF8C89201371D4632E099F92A
:101A08000A209A4200F0DA8599F912209A427FF466
:101A1800BDAE022609EBC60A40468AF8023002F03B
:101A2800D0FBD8F8003029F836001A46591CC8F8F7
:101A3800001012F8021B8AF80310C8F800205A7820
:101A48008AF80420DA1CC8F800209A788AF8062058
:101A58001E1DC8F800600135DB788AF80530AF42F2
:101A68003EF42FAC731CC8F8003096F9003099F991
:101A780002209A42C3D10026CCE7731CC8F8003074
:101A880033780E2B3FF682AEB21CC8F8002070786F
:101A980003283FF67BAE8549062202FB03F28B182A
:101AA800F51C5871C8F80050B0788854321DC8F831
:101AB8000020F2785A70721DC8F8002032799A70A6
:101AC800B21DC8F800207279DA70F21DC8F800203B
:101AD800B2791A7101252B46FEF7D8BB731CC8F8DA
:101AE80000306E4B32785A7501252B46FEF7CEBB77
:101AF800721CC8F8002035781F2D3FF647AE052B1D
:101B08007FF444AE404602F045FB694B43F825009C
:101B18001BF062FBFEF7D5BB654D05F1400640465C
:101B280002F04FFBD8F80030A5F88000591C1A467F
:101B3800C8F8001012F8021B85F88210C8F80020B7
:101B48005B7885F883300435B542E8D1FEF7B9BB38
:101B5800731C524DC8F8003033782B72404602F09F
:101B680030FBA883404602F02CFB2883404602F055
:101B780028FBD8F800206883531CC8F80030127876
:101B8800EA74D8F80420D31A032B00F31A85D8F87E
:101B98000030D11A052900F39685D21A002A7EF75B
:101BA80090AB5A1CC8F800201B7885F82130012515
:101BB8002B46FEF76BBB731CC8F8003035493078EC
:101BC8000870D21A002A7EF77CABB31CC8F8003024
:101BD8007378003318BF012301254B702B46FEF79D
:101BE80055BB404602F0EDFA2D4E3060404602F0FB
:101BF800E8FA7060404602F0E4FA0125B0602B462E
:101C0800FEF744BB244E00233360404602F0C2FA7C
:101C180033680125034333602B46FEF737BB731C3B
:101C2800C8F800303578132D3FF6B0ADB31CC8F8AE
:101C3800003070781FF04AF800283FF4A7AD1D4B1C
:101C4800027803F82520F21CC8F8002003EB85036E
:101C5800B2785A70321DC8F80020F2789A70721D56
:101C6800C8F8002014493279DA700868012525F08F
:101C7800ADFA2B46FEF70ABB104B1B78DB073FF586
:101C880085AD01250AF016FF0BF0F0F82B46FEF79C
:101C9800FDBA00BF3C38002090340020B84E002028
:101CA800BC2C0020B74E00201C380020753A0020BC
:101CB800744F002040380020183F0020FE560020B6
:101CC8004C570020C149102B4FF0000228BF1023A9
:101CD8000A604A608A60CA600A74002B3EF4F1AA5E
:101CE800D8F80020013913440132C8F8002012F84E
:101CF800010C01F8010F9A42F6D1FEF7E2BAB44F8F
:101D08003B78002B3EF4DDAAB24E0025404602F097
:101D180058FA10F04BFB3B78A6EC010A01359D42BE
:101D2800F4DBFEF7CEBA0D2B7FF430AD731CC8F888
:101D380000303578072D3FF629ADA74F40460C26D1
:101D480002F03FFA06FB05F6BD19A880404602F0EE
:101D580038FAE880404602F034FAD8F80030288192
:101D68001A46591CC8F8001012F8021BA972C8F8C4
:101D780000205B78EB72404602F00CFA0125B8515E
:101D88002B46FEF783BA731CC8F800303078060675
:101D980000F1BB84914B1B78DD073EF592AA03281E
:101DA80028BF002001250AF06DFE2B46FEF76EBA0B
:101DB8008A4B1B78D8073EF584AA01250BF03EFA1A
:101DC8000BF054F82B46FEF761BAC3F34705122D02
:101DD8003FF6DCACBDB10EAB0DF1120703EB4509C4
:101DE8003E46A9F12609404602F0EBF926F8020F13
:101DF800B145F8D17A4B37F8022F23F8022FBE42AB
:101E0800F9D1112D09D8774A6B00023B1344002100
:101E1800223223F8021F9342FBD1734A01231D4645
:101E28001370FEF733BA3346721CC8F8002013F853
:101E3800025BC8F80030F31C7078C8F80030B1783D
:101E4800002D00F02D84012D7EF43BAA12F046FCF3
:101E58002B46FEF71BBA614B1B7813F001017FF488
:101E680095AC731CC8F800303078012512F07CFB63
:101E78002B46FEF70BBA3346721CC8F800205B4AA3
:101E880013F8021BD170C8F80030594A737853719F
:101E9800F31CC8F80030574BB278DA7001252B468E
:101EA800FEF7F4B9404602F08CF9404602F089F991
:101EB800404602F086F9404602F08EF9D8F8003024
:101EC8004D4D1946581C2A68C8F8000011F8020B35
:101ED80082F82C00C8F80010597882F83610D91CFE
:101EE800C8F800109B7882F83730404602F074F941
:101EF800404602F071F9404602F06EF940462E68FD
:101F080002F05FF9708740462E6802F05AF9D8F857
:101F18000030D8F804203087D11A01290DDD591C6A
:101F28002A68C8F800101B7882F82E30404602F064
:101F380053F9D8F80030D8F80420D31A032B09DD58
:101F480040462E6802F03DF9708640462E6802F041
:101F580038F9B086286810F0F9F8FEF7B2B9731CA2
:101F6800C8F80030244D254F33787B7140462E68E1
:101F780002F027F9308440462E6802F022F9D8F89A
:101F88000420D8F80030F083D11A072900F35383CE
:101F9800D11A032900F38A83D21A002A06DD591CB4
:101FA8002A68C8F800101B7882F826300AF0C0FEAC
:101FB8001EF08CFF124B1B68002B00F0288328684A
:101FC80001250FF0A3FD2B46FEF760B9DC37002092
:101FD800BC440020E826002038240020FE560020BB
:101FE8008E53002090530020B45300200038002066
:101FF800F852002010380020183F0020C446002066
:10200800243800203346721CC8F80020BD4F13F84E
:10201800022BBA70C8F80030BB4A73781370F31CEF
:10202800C8F80030B94DB3782B71331DC8F80030AB
:10203800F378092BA8BF09234046AB7002F0C1F81A
:10204800D8F80030D8F804202880D11A012907DDF3
:10205800404602F0B6F8D8F80030D8F80420E881F5
:102068009A4240F0DF820AF063FED8F80030D8F8D0
:1020780004209A423EF425A95A1CC8F800201B786F
:10208800EB7001252B46FEF701B9404602F099F89E
:10209800054624F02BFDFF283EF413A90EA90023C2
:1020A80001F82D3DEE080DF10A008DF80A300136D1
:1020B80024F0FCFC9DF80A30F6B205F00705B3429F
:1020C80005F1010503D19DF80B30AB4203D0294639
:1020D800304624F0F7FCD8F80030D8F80420D21A9B
:1020E800012A7EF7EEA85A1C0EA8C8F80020002284
:1020F8001D7800F82C2D24F0CDFC9DF80C30AB4257
:102108000AD0834B1B683BB19A79AA4204D31B6857
:102118001B690BB128469847D8F800300EA85A1CFE
:10212800C8F8002000221D7800F8242D24F0A6FC11
:102138009DF81430AB423EF4C4A8754B1B68002BC5
:102148003EF4BFA81B685B69002B3EF4BAA828467A
:102158009847FEF7B6B86F4B1B78DA073EF5B1A87B
:102168006D4A1378012543F0040313702B46FEF7DC
:102178008DB8684B1B78D9073EF5A3A8674B4FF479
:10218800C87201251A802B46FEF780B8092B7FF705
:10219800FDAA634F3346721C3D68C8F8002013F847
:1021A800022B2A70C8F800307378AB70F31CC8F89B
:1021B8000030B378642BA8BF6423321D6B71C8F854
:1021C8000020F378642BA8BF6423721DAB71C8F894
:1021D80000203379EB71B31DC8F800307379642B94
:1021E800A8BF6423F21D2B72C8F80020B379EB70E6
:1021F80006F10803C8F80030F3792B71404601F066
:10220800E0FFD8F80420D8F800306881D11A0029F6
:102218000DDD591C3868C8F80010521A002A1978C0
:10222800417204DD9A1CC8F800205B7843700125D0
:1022380025F03EF82B46FEF729B83A4B1868F31CF0
:1022480002462136991EC8F8001013F8031C1170B5
:10225800591EC8F8001013F8021C5170C8F8003055
:1022680013F8011C91700333B34202F10302E9D160
:1022780071E6BD683968FEF740BCDFF8B0A04FF0E2
:1022880000084FF0080908F10108C8F1200209FA0E
:1022980002F2A8F120032AFA08F6164329FA03F3F2
:1022A8001E43B8F1250F06F001024FF000030CD0D1
:1022B8001343E8D05FFA88F024F082FF0028E2D0C8
:1022C800414605A802F0A0F9DDE7124B1B78DA07B2
:1022D80000F107810026144FB04602E00136252E92
:1022E80026D03146384602F09EF90028F6D031460D
:1022F80005A802F098F9002840F0CD8008F10108FF
:10230800ECE700BFC4460020F43700206C4B0020E7
:10231800B8590020FE560020C4320020245D002059
:10232800045D0020183F0020BC46002090E33FF4E5
:10233800CC4BCD4EB3F85010204601F080FFCB4B6C
:102348001988204689B201F07AFFC94B1A685301EF
:1023580003F02001C2F340030B43C2F3800143EAB8
:102368004103C2F3C00143EA8103C2F3401143EAC7
:10237800C10102F010021143204601F060FF03A9D9
:102388000422204601F02DFF23683178B94A581CF1
:102398002060197011886429A8BF6421204601F0C3
:1023A8004EFF962D00F0A8800021204601F047FF3F
:1023B8002168B8F1190348BFA8F11203A3F3C403B5
:1023C8004A1C226020461A460B7004A901F009FF36
:1023D8002368A94A581C10212060197011882046CA
:1023E800012501F015FF2B46FDF750BF2268511C4F
:1023F800216013702988204601F021FF2368EA78BC
:10240800591C21601A7023682A79591C21601A7096
:102418002368AA79591C21601A7023686A79591CA3
:1024280021601A70FEF7F4BB3346721CC8F800200E
:10243800924D13F8022B6A70C8F8003073782B702D
:10244800F31CC8F80030B378AB70404601F0B9FE11
:10245800D8F800302881591C1A46C8F8001012F81C
:10246800021B6971C8F800205B78AB7101252B4607
:10247800FDF70CBF731CC8F8003033780A2B49D01D
:10248800404601F0A9FE404601F0A6FE404601F094
:10249800A3FEFDF716BF414603A802F0B5F82DE7E5
:1024A800F4EEC87AF1EE10FA67DA4FF47A71FEF7B3
:1024B800D6BC2368B978724A581C20601970236802
:1024C8001278591C21601A70FEF72CBE0827FEF7F7
:1024D800FEBC22680125531923602B461070FDF7B6
:1024E800D5BE059B43F001030593F3E6404601F092
:1024F80068FE644EFEF759BB23680322591C21600D
:102508001A7023687278591C21601A7050E70427E2
:10251800FEF7DDBCB31CC8F800305B4B72781A704C
:10252800F21CC8F80020B2785A70321DC8F8002092
:10253800F2789A7001252B46FDF7A8BEF4EEC87A0A
:10254800F1EE10FA3EF5A8AC9FED507AF4EEC77A9A
:10255800FDEEE77AF1EE10FA17EE901A1FD86FF435
:10256800F973303903FB01F140F2E73391FBF3F1E2
:1025780001F2DB5189B2FEF772BCFDEEE77A40F258
:10258800E73317EE901A303903FB01F140F2CF73AD
:1025980091FBF3F101F2E93189B2FEF760BC40F238
:1025A800F313A1F5836103FB01F140F2E73391FBDB
:1025B800F3F101F2DD5189B2FEF751BC0126FFF7B4
:1025C80029BA404601F0FDFDA884404601F0F9FD16
:1025D800D8F80030D8F80420E884D11A03297FF706
:1025E800D8AA1A46591CC8F8001012F8021BA97775
:1025F800C8F800205B7885F82030404601F0E1FDFE
:10260800D8F80030D8F804206884FFF7C2BA204808
:102618002049214A214B036001250B6013602B469A
:10262800FDF734BE5A1CC8F800201B78003318BFC9
:102638000123FB7117E5404601F0C3FD7881404650
:1026480001F0BFFDB88140462E6801F0BAFD7084E4
:1026580040462E6801F0B5FDD8F80030D8F80420BF
:10266800B08495E4681000200C3F002084280020E6
:102678007051002088280020E03E0020785100207A
:10268800F4370020F03700203F33002000E0824478
:10269800A4250020F825002060260020A72900088E
:1026A80001250FF0C9FB2B46FDF7F0BD404601F0B0
:1026B80088FDF881404601F084FDD8F80030D8F84C
:1026C8000420388268E45A1CC8F800201B78EB7292
:1026D800404601F05FFDD8F80030E8605A1CC8F8A1
:1026E80000201B782B74D8F80030D8F80420FFF7A6
:1026F80054BA0B4BB1781A88012512FB00F22B460D
:1027080092FBF1F23A80FDF7C1BD00F07F0003288B
:1027180028BF0020012511F0FDFF2B46FDF7B6BDAF
:10272800A05D0020152303701623C370172383713F
:102738002D2343702E2303712F23C3717047002864
:1027480070B51EDB0928044620DD012303EB830353
:102758005B00B0FBF3F2092AF8D87BB10D4EB4FB4D
:10276800F3F00928CCBF57223022A6FB03E5024428
:1027780003FB1044EB0801F8012BF0D100230B7088
:1027880070BD2D230B7040420131DBE7303001F87A
:10279800010BF3E7CDCCCCCC884230B44FF0010428
:1027A8002ED301FB04F4B0FBF4F58D42F9D284B1C9
:1027B800AAB901E0B0FBF4F5092DCCBF57223022AD
:1027C8002A4404FB150003F8012BB4FBF1F4002C98
:1027D800F0D100221A7030BC7047B0FBF4F5092D17
:1027E800CCBF372230222A4404FB150003F8012B02
:1027F800B4FBF1F4002CF0D100221A7030BC704701
:102808000546002AEBD1D7E703685A1C0260197005
:1028180070472DE9F047089C2578002B80468946AB
:102828000CBF4FF0200A4FF0300A661C35B3002A5F
:1028380029DD334601E0024698B113F8011B501E0A
:102848000029F8D1971E60B13D46013D51464046EA
:10285800C8476B1C002BF8DC257827EAE7700130A5
:1028680055B1041B29464046C847301916F8015B84
:10287800002DF7D1BDE8F087BDE8F087002A04DC19
:102888002846BDE8F0870020EBE7571EDCE78368A1
:102898004268D0ED037A00EB83010133934281ED66
:1028A800040A836004BF0023836000EB830393ED75
:1028B800047A036870EE277A9A42C0ED037A77EEBD
:1028C800C77AC0ED037A0CDA013307EE103AF8EE56
:1028D800C76AB7EE007A87EEA60A036030EE070AE9
:1028E800704707EE102AB8EEC77A87EE870A704756
:1028F80090ED057A90ED004AD0ED066AD0ED014AD8
:10290800D0ED047A90ED035AD0ED025AA4EE007A85
:10291800B0EE406AB0EE470AB0EE667AA6EE247AC8
:1029280067EEC07AA0EE457AE6EE257A80ED057A64
:10293800C0ED067A7047D0ED057A90ED013AD0EDFA
:10294800003AD0ED064A90ED024A90ED077A90EDF4
:10295800035A90ED086AD0ED045AC0ED067AF0EEFD
:10296800406A27EE830AC0ED056AA3EEA60A80ED49
:10297800087AA4EE240AA5EE470AA5EEC60A80ED59
:10298800070A7047D0ED007A90ED017A30EE670AB9
:10299800E7EE007AB0EE670AC0ED007A704770473C
:1029A8000A44914214D030B40139551E41F2210233
:1029B80011F8014F082380EA042004044CBF82EA7E
:1029C80040004000013B80B2F7D18D42F0D130BCCD
:1029D80070472DE9F04FDFF820B2DFF820E2BBF8AE
:1029E8000020DEF80060BBF90430BBF90250BBF9E7
:1029F8000A80C2EB261404FB04F424135200C2EB31
:102A0800E60203FB04F305FB02F29B1303EBE2234C
:102A1800B3F5FA364FEAE37589B045F1FF37324628
:102A2800A6FB0645CDE9024502FB07F205EB42028B
:102A3800CDE90467029EBBF90840039208FB02FC3B
:102A48004FEAE87906FB09CC3A46A8FB0689049EBA
:102A5800CBF81830E51704FB02F206FB0522A4FBAD
:102A68000667E14417444FEA182242EA09620092D5
:102A78004FEA292201923D03DDE90078340345EA53
:102A880016553F19BBF80660069048EB05083C1C34
:102A980048F5004503EB8302A4FB068906FB05996C
:102AA800803213124FEA69064FEAE977079356EA2C
:102AB80007038A4600F09280DDE90489BBF90E20FD
:102AC800DEF80440BBF910004946C4F5801ED31750
:102AD800DDE9024502FB01F108FB0311A2FB082313
:102AE8000B444FEA43492B46C11700FB03F304FB91
:102AF8000133A0FB0401BBF90C401944E300019326
:102B08007346DC170023009349EAD2394FEA42485A
:102B1800DDE9002310EB080041EB0901E507121875
:102B28004FEACE744B4145EA5E05A41A65EB0305EE
:102B3800221945EB050312196B4199019001801880
:102B480041EA926159418B00820043EA907310195F
:102B580043EB05018B00820043EA9073104600198D
:102B6800194632463B46694126F034FABBF916202D
:102B78004C13450B45EAC14502FB04F6D31705FB88
:102B88000366A2FB05233344BBF9146002FB04F47B
:102B980005FB034406FB01FEA2FB0523F7172344AC
:102BA80000FB07EE540EA6FB0067774444EAC31403
:102BB8004FEAD64800194FEA636548EA4738694141
:102BC8004FEAE74918EB0008BBF9124049EB010945
:102BD8004FEA182646EA096620013618069B0BB10B
:102BE800360A1E60BAF1000F02D0079BCAF80030FF
:102BF80009B0BDE8F08F00BFF8320020E01D0020CA
:102C08007047704750F8043C012280F8452010387E
:102C180003B11847704790F8203033B1012B03D126
:102C28004FF400638382704770474FF48063838258
:102C3800704770B5044682B01430E56D06236A46C5
:102C48004321A847B0B19DF804009DF800609DF8A5
:102C580001109DF802509DF803209DF8053041EAC7
:102C6800062143EA002342EA0522A187E287A4F865
:102C78004030012002B070BD70B5044682B0083003
:102C8800656A06236A463B21A847A8B19DF8040057
:102C98009DF800609DF801109DF802509DF80320F2
:102CA8009DF8053041EA062143EA002342EA05225D
:102CB800E18222836383012002B070BD70B404688E
:102CC800037B2268022101FA03F31A4213D04269F6
:102CD8000A49582000FB02124FF6FE7650685289C6
:102CE800C5680068296831402960C168D24392B23A
:102CF8000A40C260636070BC704700BF944B0020FC
:102D080030B4094B1C7864B1084B002503EBC404AC
:102D18001A6899885562D06808330143A342D16084
:102D2800F6D130BC704700BF544E0020584E0020EA
:102D380010B40268047B11680223A340194209D029
:102D48000649406800240C7001684FF6FE74214063
:102D5800016053605DF8044B704700BF4D4F002081
:102D6800F0B4334C00EB800004EB80046468002C62
:102D78005BD0304E49004FF42040CDB2B060A1691D
:102D8800090444D460682C4F45F08071384041F400
:102D9800903101434FF420406160B06003E0411E70
:102DA800002838D00846A1698F07F8D54FF420408D
:102DB800A262B06002E0421E68B31046A269110622
:102DC800F9D562681C4945F0007545F480350A401C
:102DD80015434FF420406560B06002E0421ED0B158
:102DE8001046A2699207F9D5A362A3694FF420405F
:102DF8009B06B06005D4431E68B11846A3699B06BC
:102E0800F9D52023B060E3610120F0BC7047411E72
:102E180008B10846B3E7094A138801339BB24FF05B
:102E2800FF31B1601380F0BC70472046F0BC70479A
:102E38008C2C0020E01D0020009800FC8428002035
:102E4800134600200A4668218AE7262219210270C3
:102E5800272200238270417001221A210271837196
:102E6800C1704271C37170472DE9F3410569064687
:102E78000F467DBBD0F80080C8F30A0323B30023B4
:102E8800D6F8008001931FF053F8042819D1224C7A
:102E9800236943F001032361BBB2A8F800301FF097
:102EA80047F804282ED108F102030193019B3F0C37
:102EB8001F801FF03DF82369042823F001032361D4
:102EC80025D06FF0010505E01FF032F8042805D081
:102ED8004FF0FF35284602B0BDE8F0810E4C23695B
:102EE80043F002032361C4F81480236943F04003CC
:102EF80023611FF01DF82369042823F002032361CE
:102F0800BDD0E5E7236923F001032361D9E73368DE
:102F180004333360DEE700BF00200240F8B5044602
:102F28000D468E180027B54201D12069F8BDE36827
:102F3800591CE160234415F8012B1A720429F2D1B7
:102F4800A1682046FFF790FFE7602061EBE7024B9E
:102F580018680BF0AFB900BF4446002010B490E8E1
:102F68000600047B40690223A3404B6013685DF8A8
:102F7800044B4FF6FE710B4013600BF03BB92DE983
:102F8800F04F4B484B4B4C4C4FF090414FF0010ADF
:102F98004FF002094FF004084FF0080C4FF0100EE4
:102FA80020274026802530F8022B12F0010F03D08D
:102FB8001960A3F804A0083312F0020F03D01960B7
:102FC800A3F80490083312F0040F03D01960A3F893
:102FD8000480083312F0080F03D01960A3F804C066
:102FE800083312F0100F03D01960A3F804E0083377
:102FF80012F0200F02D019609F80083312F0400FA2
:1030080002D019609E80083312F0800F02D0196038
:103018009D80083312F4807F05D04FF4807B1960BF
:10302800A3F804B0083312F4007F05D04FF4007BF6
:103038001960A3F804B0083312F4806F05D04FF478
:10304800806B1960A3F804B0083312F4006F05D040
:103058004FF4006B1960A3F804B0083312F4805FD2
:1030680005D04FF4805B1960A3F804B0083312F45C
:10307800005F05D04FF4005B1960A3F804B0083373
:1030880012F4804F05D04FF4804B1960A3F804B0B8
:103098000833D20B04D04FF4004219609A800833E9
:1030A80001F58061A1427FF47EAFBDE8F08F00BFDB
:1030B800A8DD02083858002000180048002867D00A
:1030C80003682DE9F04F03F138445C4EA40A01254A
:1030D800345D04F01F066409022C05FA06F558D081
:1030E800032C00F0A580012C58D08088B0FA80F419
:1030F800C4F11F04A4B2E50803EB850504F0070436
:103108002E6AA4000F27A74026EA07062E622E6A19
:1031180001F00307A2407C1E3243012CC1F3810C4D
:10312800C1F300182A62C1F341113CD9C60700F166
:103138008980850700F19580440700F1A380020784
:1031480000F1B180C60600F1BF80850600F1CD8090
:10315800440600F1DB80020600F1E980C60500F1B3
:10316800F780850500F10581440500F1138102050A
:1031780000F12181C60400F12F81850400F13D8111
:10318800440400F14B81020400F15981BDE8F08F3D
:1031980070472B4CA6693543A561A6E7284C66699C
:1031A80035436561A1E7002422464FF0010E4FF038
:1031B800030904E00132102A04F10204E6D00EFAF1
:1031C80002F636EA0005F5D1D3F808A009FA04F5A5
:1031D800ED430AEA050AC3F808A0D3F808B00CFAC8
:1031E80004FA4AEA0B0AC3F808A0B3F804A01FFAC5
:1031F8008AFA2AEA06069E80B3F804A008FA02F6BC
:1032080046EA0A06B6B29E801E682E401E60D3F8B3
:1032180000A007FA04F646EA0A061E60D3F80CA0D6
:1032280001FA04F605EA0A0A46EA0A05DD60C1E77A
:10323800034CE6693543E56157E700BFBCDD02088A
:10324800001002401A6822F003021A601A683A4312
:103258001A60DA6822F003020A438507DA607FF50C
:103268006BAF1A6822F00C021A601A6842EA8702E9
:103278001A60DA6822F00C0242EA81024407DA6036
:103288007FF55DAF1A6822F030021A601A6842EAC8
:1032980007121A60DA6822F0300242EA0112DA6094
:1032A80002077FF54FAF1A6822F0C0021A601A6849
:1032B80042EA87121A60DA6822F0C00242EA8112F2
:1032C800C606DA607FF541AF1A6822F440721A60C8
:1032D8001A6842EA07221A60DA6822F4407242EA5F
:1032E80001228506DA607FF533AF1A6822F440625E
:1032F8001A601A6842EA87221A60DA6822F4406281
:1033080042EA81224406DA607FF525AF1A6822F482
:1033180040521A601A6842EA07321A60DA6822F4E0
:10332800405242EA0132DA6002067FF517AF1A68A6
:1033380022F440421A601A6842EA87321A60DA6850
:1033480022F4404242EA8132C605DA607FF509AFCD
:103358001A6822F440321A601A6842EA07421A6070
:10336800DA6822F4403242EA01428505DA607FF5E4
:10337800FBAE1A6822F440221A601A6842EA8742B1
:103388001A60DA6822F4402242EA81424405DA608F
:103398007FF5EDAE1A6822F440121A601A6842EA04
:1033A80007521A60DA6822F4401242EA0152DA60DF
:1033B80002057FF5DFAE1A6822F440021A601A6827
:1033C80042EA87521A60DA6822F4400242EA8152DD
:1033D800C604DA607FF5D1AE1A6822F040721A602E
:1033E8001A6842EA07621A60DA6822F0407242EA12
:1033F80001628504DA607FF5C3AE1A6822F0406284
:103408001A601A6842EA87621A60DA6822F0406233
:1034180042EA81624404DA607FF5B5AE1A6822F0A8
:1034280040521A601A6842EA07721A60DA6822F093
:10343800405242EA0172DA6002047FF5A7AE1A68C8
:1034480022F040421A601A6842EA87771F60DA68F9
:1034580022F0404242EA8171D960BDE8F08F00282D
:1034680052D0036803F138422DE9F04F920A514DCA
:10347800AA5C02F01F0552090124022A04FA05F485
:1034880043D0032A00F09080012A43D001F00307BB
:103498007A1E012AC1F3810CC1F300188088C1F398
:1034A80041113CD9C60700F18980850700F1958054
:1034B800440700F1A380020700F1B180C60600F1BD
:1034C800BF80850600F1CD80440600F1DB8002064E
:1034D80000F1E980C60500F1F780850500F1058156
:1034E800440500F11381020500F12181C60400F1B1
:1034F8002F81850400F13D81440400F14B810204D1
:1035080000F15981BDE8F08F70472B4A95692C432B
:103518009461BBE7284A55692C435461B6E70024F7
:1035280022464FF0010E4FF0030904E00132102A41
:1035380004F10204E6D00EFA02F636EA0005F5D1E7
:10354800D3F808A009FA04F5ED430AEA050AC3F816
:1035580008A0D3F808B00CFA04FA4AEA0B0AC3F830
:1035680008A0B3F804A01FFA8AFA2AEA06069E8081
:10357800B3F804A008FA02F646EA0A06B6B29E8034
:103588001E682E401E60D3F800A007FA04F646EA2B
:103598000A061E60D3F80CA001FA04F605EA0A0A26
:1035A80046EA0A05DD60C1E7034AD5692C43D461C0
:1035B8006CE700BFBCDD0208001002401A6822F068
:1035C80003021A601A683A431A60DA6822F00302A2
:1035D8000A438507DA607FF56BAF1A6822F00C02A0
:1035E8001A601A6842EA87021A60DA6822F00C0246
:1035F80042EA81024407DA607FF55DAF1A6822F07B
:1036080030021A601A6842EA07121A60DA6822F071
:10361800300242EA0112DA6002077FF54FAF1A68FA
:1036280022F0C0021A601A6842EA87121A60DA6841
:1036380022F0C00242EA8112C606DA607FF541AF85
:103648001A6822F440721A601A6842EA07221A605D
:10365800DA6822F4407242EA01228506DA607FF5D0
:1036680033AF1A6822F440621A601A6842EA872265
:103678001A60DA6822F4406242EA81224406DA607B
:103688007FF525AF1A6822F440521A601A6842EA98
:1036980007321A60DA6822F4405242EA0132DA60EC
:1036A80002067FF517AF1A6822F440421A601A68BA
:1036B80042EA87321A60DA6822F4404242EA8132EA
:1036C800C605DA607FF509AF1A6822F440321A603D
:1036D8001A6842EA07421A60DA6822F4403242EA7B
:1036E80001428505DA607FF5FBAE1A6822F44022B4
:1036F8001A601A6842EA87421A60DA6822F440229D
:1037080042EA81424405DA607FF5EDAE1A6822F498
:1037180040121A601A6842EA07521A60DA6822F4FC
:10372800401242EA0152DA6002057FF5DFAE1A68FC
:1037380022F440021A601A6842EA87521A60DA686C
:1037480022F4400242EA8152C604DA607FF5D1AE23
:103758001A6822F040721A601A6842EA07621A6010
:10376800DA6822F0407242EA01628504DA607FF585
:10377800C3AE1A6822F040621A601A6842EA876289
:103788001A60DA6822F0406242EA81624404DA6030
:103798007FF5B5AE1A6822F040521A601A6842EAFC
:1037A80007721A60DA6822F0405242EA0172DA605F
:1037B80002047FF5A7AE1A6822F040421A601A6820
:1037C80042EA87771F60DA6822F0404242EA817154
:1037D800D960BDE8F08F70B5044690F8590000280C
:1037E80033D104F11405236E80226B2128469847B3
:1037F80064200AF009FC236E284603226B219847AF
:10380800236E94F854201921284698470F200AF06F
:10381800FBFB236E94F8522028461A219847236E02
:10382800284618221B219847236E284618221C2157
:103838009847236E28460222372198472846236E48
:1038480001223821BDE8704018470AF0CDF8054636
:10385800D0B1202300218371C171FFF700FE2146FA
:103868000F4B41F8103F284622F06EF9AB88B3FAA7
:1038780083F3C3F11F035A1CB3D001229A400949AC
:103888000B6813430B60ACE70146FFF7E8FD2146E0
:10389800034B41F8103F284622F056F90122EEE783
:1038A8000D2C00080004014010B1036882889A6159
:1038B800704738B100298388026814BF002110219D
:1038C8008B40936170472DE9F0410B4E3468736962
:1038D8001C400FD0DFF824800127B4FA84F3C3F129
:1038E8001F0307FA03F558F8230003689847AC4309
:1038F8007561F2D1BDE8F081000401400057002055
:103908002DE9F0410B4E346873691C400FD0DFF885
:1039180028800127B4FA84F3C3F11F0307FA03F5DB
:1039280058F8230003689847AC437561F2D1BDE8A5
:10393800F08100BF00040140005700202DE9F0414C
:103948000B4E346873691C400FD0DFF828800127BC
:10395800B4FA84F3C3F11F0307FA03F558F82300F8
:1039680003689847AC437561F2D1BDE8F08100BFA8
:1039780000040140005700202DE9F0410B4E346847
:1039880073691C400FD0DFF828800127B4FA84F34C
:10399800C3F11F0307FA03F558F823000368984793
:1039A800AC437561F2D1BDE8F08100BF000401406D
:1039B800005700202DE9F0410B4E346873691C4014
:1039C8000FD0DFF828800127B4FA84F3C3F11F036E
:1039D80007FA03F558F8230003689847AC43756164
:1039E800F2D1BDE8F08100BF00040140005700207B
:1039F8002DE9F0410B4E346873691C400FD0DFF895
:103A080028800127B4FA84F3C3F11F0307FA03F5EA
:103A180058F8230003689847AC437561F2D1BDE8B4
:103A2800F08100BF00040140005700202DE9F0415B
:103A38000B4E346873691C400FD0DFF828800127CB
:103A4800B4FA84F3C3F11F0307FA03F558F8230007
:103A580003689847AC437561F2D1BDE8F08100BFB7
:103A68000004014000570020084A094808B5936936
:103A780043F0010393610021402227F0CEFF054B5C
:103A88004FF0FF321A60C3F8032008BD001002404F
:103A980000570020405700202DE9F0410446184601
:103AA8000D461646984624F0EBFD2768E672284432
:103AB800A07229467D69434632462046AC46BDE899
:103AC800F0416047036810B504461B6898472368AF
:103AD80020469B689847A37B0133A37310BDF8B5B4
:103AE800574C0601A7190546387A20F06BFB3B7A3C
:103AF80003F01F015B090122022B02FA01F278D0C0
:103B0800032B71D0012B67D0A3190135187909F05F
:103B18006BFFEDB2074610B11223C5718371A3196B
:103B2800587909F061FF10B11323C5718371A31986
:103B3800987909F059FF10B11423C5718371A5193B
:103B48000E21EA793846FFF7B9FA687909F04CFF8F
:103B5800EA790E21FFF7B2FAA87909F045FFEA7968
:103B68000E21FFF7ABFAA359364A934251D0364A91
:103B7800934259D0354A934240D03444227B002A9C
:103B88002FD1012002249A8822F480521204120CA8
:103B98009A80998889B241F4805199801A8802F4F0
:103BA800415242F44572024322431A809A8822F411
:103BB80070621204120C42F4E0629A809A8B22F42A
:103BC80000621204120C07219A8319821A8892B291
:103BD80042F040021A80F8BD1D4B996A0A439A6266
:103BE80092E700200446CEE7194B19690A431A6187
:103BF8008AE7174BD9680A43DA6085E702F5EA32A3
:103C0800116941F400411161116921F40041116108
:103C1800B3E702F56042D16841F48051D160D168C0
:103C280021F48051D160A8E702F5EC32116941F422
:103C380080411161116921F4804111619DE700BF44
:103C4800C83200200030014000380040003C0040ED
:103C580000100240427A02B9704710B50446036862
:103C6800406804F10A0198470023637210BD437A43
:103C78005A1C0344D2B242729972037A934200D812
:103C880002B9704710B504460368406804F10A0198
:103C980098470023637210BD10B40B49002301E05C
:103CA800272B0CD011F8132082424FEA430403F16A
:103CB8000103F5D121445DF8044B48787047002092
:103CC8005DF8044B704700BFCCBB020870B5448850
:103CD80006460D46C4F30B0422460021284627F069
:103CE8009CFE3369094A934209D3094A934206D292
:103CF800224628461946BDE8704025F059BC23B134
:103D080021462846BDE87040184770BDE0160308F4
:103D1800C0170308064B07498B4202D300231846F5
:103D280070471A88C2F30B029042F8D01433F3E7B5
:103D3800D0120308E0160308024A136823EA0000B9
:103D48001060704790340020F8B5174D2B78A42BDD
:103D580028D16B78BE2B25D1022229464FF6FF7059
:103D6800FEF71EFE114FAC1C22884AB1A618BE42AF
:103D780018D2052A16D92146FEF712FE3446F3E773
:103D880021460222FEF70CFE0222A118FEF708FEC9
:103D98000634074B641B1C8041F60F53C31A584264
:103DA8005841F8BD0020F8BD00F0030800000408E1
:103DB800862800202DE9F04FDFF848914C4F8BB052
:103DC8000326A7EB09071822002104A827F025FEDF
:103DD800484BCDF8109005971A69120604D5464A43
:103DE8005A6002F188325A6001228DF82420342268
:103DF800DA60424B424C1B88ADF80030022269461B
:103E080004A8FFF78BF8022269464FF6FF70FEF709
:103E1800C7FDDFF8F4A080464FF0000B544536D3B9
:103E28000AAC002524F8245D0222214604A8FFF7E5
:103E380075F8022221464046FEF7B2FD40BAC0435B
:103E4800ADF80800022202A904A8FFF767F807984E
:103E580060B106ABC0F104022946184427F0DDFD25
:103E6800069904A8FFF700F8079508909DF82430F4
:103E7800089A23B11F490B6943F080030B61013E87
:103E88002DD0002A9FD1FFF75FFF50B32CE0658843
:103E98008DF80DB0C5F30B05AB1DADF808302388C0
:103EA800C3F30B02ADF80A201B0B062202A904A8D3
:103EB8008DF80C30FFF732F8062202A94046FEF7CB
:103EC8006FFD616880462A4604A8FFF727F86168F5
:103ED80040462A46FEF764FD143480469EE7002AD1
:103EE800D1D0052008F0F0FD0BB0BDE8F08F00BF81
:103EF8000000040800200240230167451ABC02089C
:103F0800D012030800F00308E01603080378202BFA
:103F1800024600F10100F9D0092BF7D02D2B2CD047
:103F28002B2B03BF5378B7EE000A0246B7EE000A00
:103F3800A3F13001C8B209289FED467A10D8F2EEF5
:103F4800046A07EE901AF8EEE77A12F8013FE7EEF6
:103F5800267AA3F13001C8B20928B0EE677AF0D901
:103F68002E2B4CD003F0DF03452B0BD0F7EE007A55
:103F780067EE276A20EE260A70475378BFEE000ADC
:103F88000246D5E710B451782D2959D02B290ABFFC
:103F98009178501C901C0024A1F13003092B53D8B0
:103FA800002303EB830301EB430310F8011FA1F186
:103FB8003002092AA3F13003F3D9B3F59A7F28BF59
:103FC8004FF49A73072B42D9DFED236A1A46F7EEAE
:103FD800007A083A072A67EEA67AFAD803F00703A8
:103FE8002BB1F2EE046A013B67EEA67AFBD124B34B
:103FF800C7EE276A5DF8044B20EE260A704753780F
:10400800A3F13001C8B2092802F10102AAD8F2EEE0
:10401800046AF0EE665A07EE901AF8EEE77A12F89C
:10402800013F87EEA66AA3F13001C8B2092866EEFF
:10403800A56A37EE067AEED994E767EE276AD9E7DC
:10404800901C91780124A7E7F7EE007ACFE7F7EE06
:10405800007AC5E70000000020BCBE4CB5EEC00ADF
:10406800DFED317AF1EE10FACCBF30EE270A30EEF0
:10407800670ADFED2E7A20EE270A30B5FDEEC07A0A
:1040880087B017EE904A054684EAE470002303A936
:10409800A0EBE4700193009302931BF087FB002CC4
:1040A800ACBF20232D2303A88DF8003024F0E8FAB4
:1040B800012803A924D002282DD0032805BF3023C6
:1040C800684668468DF8013027F0CDFC684624F034
:1040D800D7FA0338C4B222466946284627F021FD9C
:1040E80000232B55284624F0CBFA2E22431C2A54B1
:1040F8000DEB0401E81827F0D3FC284607B030BDC3
:10410800302368468DF801308DF802308DF8033081
:1041180027F0A9FCDAE7302368468DF801308DF8DE
:10412800023027F0A0FCD1E76F12033A00007A446E
:104138002DE9F041064615460846B6FBF2F43CB9AF
:1041480005FB1464124B1B5D00F8013BBDE8F081D0
:10415800B4FBF2F767B90E4B05FB174705FB146470
:10416800DA5D00F8012B1B5D00F8013BBDE8F0812A
:10417800B7FBF2F8B8F1000F02D04046FFF7D8FFBE
:1041880005FB1878024B13F8082000F8012BE3E729
:1041980034E1020830B402681146531C036011F878
:1041A800024B0160D31C517803609378151D05609C
:1041B8001B0443EA0123D078234343EA006030BC60
:1041C80070470368591C1A46016012F8021B026006
:1041D800587841EA0020704703685A1C0260187832
:1041E800704738B504460068154625F0E1F922689D
:1041F8002A44226038BD036810B40A0A5C1C0460B3
:104208001A7003685A1C026019705DF8044B7047F5
:1042180003685A1C026010B4197003680A0A5C1C0F
:1042280004601A7003680A0C5C1C04601A70036846
:10423800090E5A1C026019705DF8044B7047036838
:104248005A1C026019700368090A5A1C0260197026
:1042580070472DE9F047002488B080460F461E4677
:10426800A14605AD531C0393117839B3252933D1E1
:10427800931CCDF810900393507830284ED04FF00F
:10428800000AA0F13003DBB2092B42D96C2819D0FF
:10429800642800F0938024D825281CD063D9582896
:1042A80076D063281BD131784046B847039A531C0F
:1042B80003931178043601340029D7D1204608B079
:1042C800BDE8F087039B5A1C03921B78642B7CD0B3
:1042D8002AD8252B54D1252140460134B847039AC2
:1042E800C0E7732833D044D975284FD106F1040E9E
:1042F80030682B4600220A217646FEF74DFA049ACA
:104308000095534639464046FEF783FA039A04441B
:10431800A8E704AA03A91BF025FAB7E7D31C03935F
:1043280090784FF0010AACE7732B10D05BD9752B4E
:104338003AD0782B96D1A3F15802B2FA82F23068BB
:1043480052092B4610210436FEF726FAD7E73368C0
:10435800049A0093394600234046FEF75AFA043679
:104368000444039A7EE70028B9D1204608B0BDE886
:10437800F0876E28B3D1039A336804361C6071E75E
:104388002AD9582BD7D0632B8DD06BE77828A6D1A4
:10439800A0F15802B2FA82F2306852092B46102175
:1043A800FEF7FAF90436AAE706F1040E30682B4640
:1043B80000220A217646FEF7EFF9A0E7331D3068A0
:1043C80029461E46FEF7BBF999E7331D3068294692
:1043D8001E46FEF7B4F992E7002B7FF443AF204660
:1043E80008B0BDE8F0876E2BC6D03BE70EB400B529
:1043F80084B005AB019053F8042B0649039301A838
:10440800FFF727FF019B00221A7004B05DF804EB48
:1044180003B07047112800080FB430B583B006AB5D
:104428000A490B4853F8042B096800680193FFF701
:1044380010FF084C0546206809F030FF0028FAD024
:10444800284603B0BDE8304004B07047042A002075
:10445800082A002044460020DFED2B7AB4EEE70A54
:10446800F1EE10FA4ADDDFED296A9FED297A01E0C5
:10447800B0EE670AB4EEC70AF1EE10FA70EE667A8B
:10448800F6DC9FED247AF4EEC77AF1EE10FA38D50F
:10449800DFED1E6A9FED207A01E0F0EE407AF4EE3F
:1044A800C77AF1EE10FA37EEA60AF6D4DFED1B7ADA
:1044B800B4EEE70AF1EE10FA14DDDFED137A37EE09
:1044C800C00A60EE006A9FED166A9FED167ADFED6E
:1044D800167AA6EE867A20EE266AE6EE877AA6EEA9
:1044E800270A7047DFED117AB4EEE70AF1EE10FA09
:1044F80044BFDFED087A37EEC00AE2E7F0EE407A13
:10450800BFE7B0EE670AD1E7DB0F4940DB0FC940D0
:10451800E4CB1641DB0F49C0E4CB16C1DB0FC93F22
:1045280092E741B99730083C15A82ABEDB0FC9BFEE
:1045380080EAE073A3EBE0738B4205DB002801DD22
:10454800401A704702D170470020704708447047EE
:1045580009B909E0194690FBF1F301FB130308467A
:10456800002BF7D1084670470146FBE710B507EE68
:10457800901A2DED028BB8EE678ADFED217A28EECE
:10458800008A044628EE278AB0EE480A25F0D0F9BA
:10459800F0EE408AB0EE480A25F02CF9F7EE007AE2
:1045A8009FED187AF0EE675AE8EE875A0023A36168
:1045B800B0EE676AC7EEA56A63612362E361A8EE9D
:1045C800C76ABDEC028B77EEC07AB6EE007AF8EED9
:1045D800005A27EE877A20EE250A27EE267A26EE5D
:1045E800266A67EEA67A20EE260A84ED046AC4EDF0
:1045F800017A84ED007A84ED027A84ED030A10BD15
:1046080027D4D236F304353F10B44C09012250F8B0
:10461800243001F01F0102FA01F10B4340F8243065
:104628005DF8044B70474B0901F01F0150F8232037
:10463800012303FA01F1114214BF18460020704704
:10464800F8B5224B1B78012B32D0214B822703F17E
:10465800EA0628215A22782555242D201F705970E2
:104668009A70DD7019715A719C71D8714E33B342CA
:10467800F4D1184C184B194919481C2262700126AC
:10468800002230255A709A701E70DD702127A7709D
:104698001FF07CF9134B40F24C4140F26C721980C8
:1046A8009980198199815A80DA805A81DA81F8BD16
:1046B8000D4A0E480E494FF4486640F22E45022432
:1046C8001680158284700B70BFE700BF003A002087
:1046D800543300207851002040380020B84E002084
:1046E8005CE10208205600206C4B0020C4460020E4
:1046F800F4370020B0F1FF3F0AD0022810B403DCE1
:104708005DF8044BFEF72CBB00205DF8044B7047A6
:10471800002070470378012B00D07047417990F949
:1047280004003123F422E5E7F0B55B4B5B4A97B010
:104738001968914200AF00F0A3805949594A0023F3
:104748004FF47000C1F888003B607B60136843F445
:104758008033136003E03B68B3F5A04F09D01368BA
:1047680003F400337B603B6801333B607B68002BBC
:10477800F1D04C4B1B6813F4003318BF01237B6046
:104788007B68012B52D0464C464B474AE260474A69
:10479800596A11605A6A42F080725A625A6942F440
:1047A800FC025A610025032207F10801012341F6A2
:1047B800FF764FF09040FD60BE603A73BB7320F007
:1047C800A3FF4FF6FF7307F108013948BB6020F0DB
:1047D8009BFF07F108013748374E20F095FF07F196
:1047E8000801364820F090FF07F10801344820F00E
:1047F8008BFF07F10801334820F086FF07F1080016
:1048080020F038FDBB683049304AA1FB031330491A
:104818009B0CF0204FF0070E5C370B60566084F855
:1048280023009560C2F800E0BD46F0BD294A1D4B43
:10483800122111605A685A605A685A605A6842F4DC
:1048480080625A605A6822F47C125A605A6842F4AC
:10485800E8125A601A6842F080721A601A68920167
:10486800FCD559680F4A21F003015960596841F095
:1048780002015960536803F00C03082BFAD182E750
:1048880000221A6062B6144B1B6883F30888134B26
:104898001B689847FEE700BFFC9F0020EFBEADDE17
:1048A80000ED00E0001002400005FA057441002008
:1048B80000040048000800483F190100000C0048A7
:1048C800001000480014004883DE1B4310E000E09D
:1048D800B45600200020024000D8FF1F04D8FF1F54
:1048E80070B50F4C0F4DC0EBC00004EB8004686935
:1048F80026693043686182B09209667BA160002511
:10490800012101A863618DF804608DF805208DF8F8
:1049180006508DF8071020F0A1FB02B070BD00BF53
:104928004814002000100240074BC0EBC00030B410
:1049380003EB8000054C056963692B4363610176CD
:10494800427630BC704700BF481400200010024077
:104958002DE9F04F5E4C54F8204083B0002C71D004
:10496800666D984691465B4B7268E264A16023606D
:1049780004F15A014FF4807304F5AD726161A261CC
:10498800E36023610746307E1FF01CFCF068A8B185
:10499800514B00215A68904203F11C0300F09280A9
:1049A80001310C29F6D100207A1CD2B20C21FFF774
:1049B800BBFFE36CF26822632433A364B068D8B108
:1049C800454B00215A68904203F11C0378D001310D
:1049D8000C29F7D100257A1CD2B20B212846FFF703
:1049E800A3FF2346F27E3D492846FFF779FFE36C93
:1049F800B26862632833636494F8590008F0F4FFDE
:104A0800054694F8580008F0EFFF18F0080F8246A2
:104A180096F819B01AD0CDB118F0110F4FF00B035A
:104A280007F1010714BF4E213E21EF715A46AB71C1
:104A38002846FEF743FB18F0010F45D0236B5BB304
:104A4800636B4BB3204603B0BDE8F08F18F0010F3D
:104A58000CBF4FF02E084FF04E0819F0020F09D086
:104A680045B10B227B1CAA71EB7128465A46414678
:104A7800FEF724FB19F0010FE0D0BAF1000FDDD0EA
:104A880001370C238AF807705A4641468AF80630DF
:104A98005046FEF713FBD1E7337FB27E8DF8042032
:104AA8009B090021012201A88DF805308DF8061018
:104AB8008DF8072020F0D2FA204603B0BDE8F08F29
:104AC800CDB288E7C8B26FE72B68AA881A85B5E720
:104AD8006C2C00201CBC020848140020652F00081C
:104AE8000348D0F83C3113B100F59A701847704765
:104AF800481400200348D0F8203113B100F58C7019
:104B080018477047481400200348D0F804310BB107
:104B1800FC301847704700BF481400200348D0F8FD
:104B2800E8300BB1E0301847704700BF4814002048
:104B38000348D0F8CC300BB1C4301847704700BFD9
:104B4800481400200348D0F8B0300BB1A8301847FB
:104B5800704700BF481400200348D0F894300BB1C8
:104B68008C301847704700BF481400200248836FF4
:104B78000BB1703018477047481400200248C36DC5
:104B88000BB1543018477047481400200248036C92
:104B98000BB1383018477047481400200248436A60
:104BA8000BB11C301847704748140020024883682E
:104BB80003B11847704700BF48140020F0B53E4CB9
:104BC800059D00EB800004EB80046468002C71D024
:104BD8003A4E49004FF42040CFB2B060A1690904B1
:104BE80054D46068DFF8E0E047F4903100EA0E0042
:104BF80001434FF420406160B06003E0411E00288B
:104C080048D00846A1698907F8D54FF42040A26228
:104C1800B06003E0421E00283CD01046A26952064C
:104C2800F8D5274A6168DFF8A0E0B06042EA03429D
:104C3800174301EA0E0217436760C3B1013BDBB2B9
:104C480001332B44A0694FF4204210F0040002F114
:104C5800FF3207D1511C26D0A06910F0040002F1E0
:104C6800FF32F7D0626A05F8012B9D42EAD14FF472
:104C78002040B06002E0431E60B11846A3699B065D
:104C8800F9D52023B060E3610120F0BD411E08B1D1
:104C98000846A3E70B4A138801339BB24FF0FF3154
:104CA8001380B160F0BD0749B2600B8801339BB235
:104CB8000B80F0BD2046F0BD8C2C0020E01D0020AC
:104CC8000024000284280020009800FC70B590F9A8
:104CD80004506C1C82B00AD0022D08DC16460A4625
:104CE800417900962846FFF769FF02B070BD0020A1
:104CF80002B070BD70B50378012B82B004D10623D1
:104D08006A46F721FFF7E2FF9DF801209DF804307D
:104D18009DF800609DF803509DF802409DF805003D
:104D2800074912011B0142EA063243EA053342EA07
:104D3800141243EA10134A600B6002B070BD00BF42
:104D4800E01D002000B583B0002000920A466821CB
:104D5800FFF734FF03B05DF804FB421C76D002284D
:104D680074DC2DE9F843142303FB00F33C4FFA5895
:104D78003B44002A6BD01C1D94E810030546907B29
:104D88001FF020FA374B9C4263D0374A136B23F04D
:104D9800100313631023344A116B6E1C0B43136307
:104DA800F6B2B8F1000F04D0152388F8076088F828
:104DB8000630142303FB057340465B7C002B14BFAD
:104DC8003E211E210422FEF779F9B9F1000F04D023
:104DD800162389F8076089F80630142000FB05754A
:104DE80004226B7C002B14BF3E211E214846FEF78F
:104DF80065F921682D7C1D4B1D481E4A21F00101D3
:104E080021602168002D08BF03460A402260236103
:104E18002268002342F001022260A360E360A360DD
:104E2800A36843F40043A36023682360636823F006
:104E3800784323F400436360236823F4003323603A
:104E4800236843F001032360BDE8F8837047BDE899
:104E5800F8830549084B0A6B22F020020A639AE797
:104E68008C2C00200058004000100240300E5000EA
:104E78007A25E000FFE0CF00200000101749184B0A
:104E8800184A194810B4D1F8884044F47004C1F89D
:104E980088401C6844F001041C605C6822405A6029
:104EA8001A6822F0847222F480321A601A6822F496
:104EB80080221A605A6822F4FE025A60DA6A22F0E6
:104EC8000F02DA621A6B002410404FF00062186378
:104ED8009C608A605DF8044B704700BF00ED00E0FD
:104EE800001002400CC07FF8CCFC00FF2DE9F04F09
:104EF8002DED028B93B002901DF08CFBB84B1D7802
:104F080025B113B0BDEC028BBDE8F08FB54B1B6823
:104F18005C05F6D5B44FB54E3B68002B5CD0B44C5D
:104F28003168D4F810218A1A7C2A55D994F81421AA
:104F3800DFF80C839FEDAF8AC4F81011013284F8B2
:104F48001421A8F138094FF0240A5E2098475046EA
:104F58003B689847B9F81430F8EC016A07EE103A44
:104F6800F8EEE66AB8EEC77A0AF1010AC6EE877A61
:104F78005FFA8AFA67EE887AFDEEE77ACDED037A72
:104F8800BDF90CB05FFA8BF017F050FACBF307209D
:104F980017F04CFABAF1270F3B68D6D15E20984734
:104FA8003B6830209847D4F818815FFA88F017F0EA
:104FB8003DFAC8F3072017F039FA3B685E20984796
:104FC80094F8143113F0030800F07681580701F0C3
:104FD8000F80282B01F04B83874B1B78002B6FD059
:104FE800834C0299D4F82031844ACB1A934200F2B8
:104FF8008B87DFF850A29AF80080B8F1000F34D1FF
:10500800DFF80892D9F8000009F050F9C0B2012879
:105018000FD902287A4F41F0F7833B78002B41F0F3
:105028001886D4F82831029AD31AB3F57A6F81F02A
:10503800738774480268002A42D09AF80030BBB9D6
:10504800714BD9F800001B689B781E3B012B4FF071
:10505800020141F2D286043017F05AF901220023E6
:105068008AF8002084F8343127E0664802683AB3A9
:10507800D4F83031029F40F6B731FB1A8B421FD962
:1050880094F82C31002B01F0BB83013BDBB284F890
:105098002C31002B01F0E38212F8011B94F83471D3
:1050A800026094F835315948CA190133006884F808
:1050B800342184F8353109F0FDF8029BC4F8303109
:1050C800534BD6F800801B7843B1524F386828B14B
:1050D800514B1B78013B012B41F234804F4B1B781D
:1050E80063B14F4F3B684BB1414CD6F800B0D4F890
:1050F8004C31ABEB0303632B00F26586DFF8488184
:1051080098F80030022B01F080823D4F97F87430F8
:10511800032B00F05787434B1B7873B1424D2B6824
:105128005BB1334C08F0CAFED4F8583144F61F621C
:10513800C31A9342834600F213813C4B1B78002B21
:1051480040F084803A4B1B784BB1294C029AD4F832
:10515800A83203F5C333A0339A4280F09586354BC5
:105168001B78002B3FF4CDAE214E334C334D06F265
:10517800C927206809F09AF800283FF4C2AE2068D1
:1051880009F090F82B7880465A1E33B120682A70AF
:1051980009F08CF80028F2D1B3E603223946781ECC
:1051A80026F021FC96F8C83296F8C92286F8CB82F8
:1051B80083F47F4383F0FF039B1A1FFA88F89BB29E
:1051C800B8EB132FD5D196F8CA22DBB29A42D0D1C8
:1051D800781E16F019FE2B7818442870C9E700BF0E
:1051E800F13E00206C490020983E0020B056002077
:1051F800341E002000007A44065100203F0D0300B1
:1052080000000020903E00208C3E0020883E0020B8
:1052180008510020083C002010510020185100209F
:10522800D441002020510020245100206451002046
:10523800895100202A51002030510020345100208B
:10524800783F0020943E00208A5400203A4C22786F
:10525800002A40F0FA85394E3478002C5FD1384D59
:105268002878002841F08284364C374DD4F8A012B3
:105278002A78364B93FBF2F3029A0B449A42FFF4D6
:1052880061AF114694F8A432314AC4F8A012D65C32
:10529800F70701F1A286B10701F15C86720701F1F7
:1052A800F78594F8A4322978013393FBF1F201FBD6
:1052B800123384F8A43245E7D4F8102141F2883338
:1052C8009A4201F257823B685E2098473B68142057
:1052D8009847204B204AB3F9043082FB03124FEA67
:1052E800E378C8EBA2080FFA88F85FFA88F017F09D
:1052F8009DF8C8F3072017F099F83B685E20984797
:105308003B681C209847002017F090F8002017F001
:105318008DF83B685E20984794F8143156E60F4D97
:10532800286E002841F0F3818046064B029A86F8E1
:105338000080C3F8A02205E7F85000206D51002036
:105348006C510020341E002088510020A0860100E6
:1053580074510020883F00206766666690510020DF
:1053680094F85E31002B41F0BC81DB4B1A6802F0E7
:105378000803002B48F603414AF60B404BF60F434F
:1053880049F6074704BF03460F4612F0040F4FF0D3
:10539800190118BF1F46920684F85E1103D547F419
:1053A800804747F02007CD4B5A79C7F30909002AEF
:1053B80041F065869B79002B41F05A869846642017
:1053C8004FF0FF3A4FF0000C0A970B97ADF834C036
:1053D800CDF83AC0CDF83EC0CDF842C0CDF83090F7
:1053E800ADF83680ADF838A08DF846000AAF0FCF7B
:1053F800DFF800E384F805C0AEE80F0097E80F0077
:10540800AEE807002EF8023B71464FF0010C1B0C6A
:10541800FE271F20C82201F81E39A770A27184F840
:1054280007C0E07094F86E01207180F0F10383EA00
:105438000313DAB2130983F0E70343EA022383EA8A
:10544800C2031BB283EA0312D2B2C3F3072383EA6F
:10545800121343EA022383EAC2031BB283F0C80291
:1054680082EA0212D2B2C3F3072383EA121343EA91
:10547800022383EAC2031BB283EA0C0787EA0717F1
:10548800FFB2C3F3072282EA171242EA072200EBAF
:105498000C0382EAC7070EEB0C0084F86E312780F4
:1054A80011F8013B7B4083EA0313DBB21A0982EA55
:1054B800172242EA032282EAC3031BB29FB2814247
:1054C8002780EDD183F07C0383EA0313DBB24FEA34
:1054D800131E8EEA172E8EEA032E8EEAC30E0FFADB
:1054E8008EFE1FFA8EFADFF810C2A4F800A05FFA49
:1054F8008EFE4FEA1A2A84F828A084F827E00CF5D3
:10550800CB7804F12209DCF80000DCF80410DCF8A0
:105518000820DCF80C3047460FC70CF1100CCC45BE
:10552800B846F0D1DCF8000038606D4F9CF80430C4
:1055380088F8043007F1270884F8BDE184F8BEA193
:1055480017F8011F286808F0B5FEB845F8D194F897
:105558005F31002B41F0CA806249326809780A201D
:1055680084F85F01002901F01B825F4F0129388808
:10557800069041F2A1860229B7F802E001F096856B
:10558800B8880590032901F0A086F88804900429BA
:1055980001F0B1860529388901F0A8860629B7F8EF
:1055A8000A9001F09F860729B7F80C8001F09786CA
:1055B800FB89039394F86E110A920B4683F030022C
:1055C80082EA0212D2B217094849079387F07A078C
:1055D80047EA02270988237187EAC202444FC1EBD0
:1055E800012187FB013A069B4FF0000C63F30F0C77
:1055F800059B6EF31F4C4FF0000E63F30F0E049BD8
:10560800CDF82CC012B28A440027C91763F31F4E85
:10561800C1EB6A2A039BCDF830E082EA021160F3FD
:105628000F070020C9B268F30F00C2F3072269F31D
:105638001F4782EA111263F31F404FF000090D97CC
:105648008DF83DA00E908DF83C9042EA01220DF1B4
:10565800280C82EAC107BCE80F003FB287F0C808EF
:1056680088EA0818DFF88CE084F805905FFA88F873
:10567800C7F30727AEE80F0087EA181747EA082399
:105688009CE8030083EAC8031BB283F023024EF8A8
:10569800040B82EA0212D2B2C3F30723079F83EAFC
:1056A8001213704643EA022383EAC20207F1010C8F
:1056B80020F814194FF023081621FE27C82384F870
:1056C8006EC1228084F807800EF1020EA770E17087
:1056D800A371114612E000BF7051002078510020DC
:1056E800CB1F0020903F0020404500207050002034
:1056F800030820803C1E0020361E002010F8013BC5
:105708004B4083EA0313DBB21A0982EA112242EA08
:10571800032282EAC3031BB299B270452180EDD1FE
:1057280083F0F40383EA0313DBB24FEA131E8EEA15
:10573800112E8EEA032E8EEAC30E0FFA8EFE1FFA82
:105748008EF8E44FA4F800804FEA182C5FFA8EFE1A
:1057580084F81EE084F81FC07968BA683868FB6866
:1057680007F5CB78A8E80F0038697969BA6904F2B7
:105778009717A8E8070004F2B51884F8B5C184F8AB
:10578800B4E117F8011F286808F094FDB845F8D16E
:1057980094F866C1BCF1000F40F0B387CE4B94F883
:1057A8006E71B3F90010B3F90220B3F904309FED1C
:1057B800CB6ADFF844E384F805C007EE103A336893
:1057C8000A9387F06A0383EA031306EE901AD9B2A4
:1057D8000B0983F0D50343EA012383EAC1031BB213
:1057E80083EA03115242C9B207EE902AC3F3072392
:1057F80083EA111343EA0123F8EEE77AF8EEE66A42
:10580800B8EEC77A83EAC1031BB267EE867A66EE02
:10581800866A27EE067A002083F0C808CDED0C7A58
:10582800CDED0B6A8DED0D7A0E900F90109088EAF1
:1058380008160DF12809F6B2C3F30728B9E80F00D6
:1058480088EA161848EA062888EAC6080FFA88F887
:10585800AEE80F0088F01E0699E8070086EA0616EB
:10586800F6B2C8F3072383EA161343EA06238EE841
:10587800070083EAC6061C20C8214FF005084FF030
:105888001E0CFE237A1CE070A17184F8668184F8EE
:1058980007C0A370AEF1100127710EF10C0026802D
:1058A80084F86E2111F8013B734083EA0313DBB2DD
:1058B8001A0982EA162242EA032282EAC3031BB2C9
:1058C8009EB281422680EDD183F0270383EA031339
:1058D800DBB24FEA131E8EEA162E8EEA032E8EEAEC
:1058E800C30E0FFA8EFE1FFA8EFC7A4FA4F800C082
:1058F8005FFA8EFE4FEA1C2C84F825C084F824E059
:1059080007F5CB7804F1220938687968BA68FB682A
:1059180046460FC610374F45B046F5D1704E3B8806
:10592800A8F8003006F1240784F8BAE184F8BBC16E
:1059380016F8011F286808F0BDFCB742F8D194F8A2
:1059480067A1BAF1000F40F0D686664B1B680522A6
:1059580013F0140F84F8672141F00C80DFED627AB0
:1059680094F86EC15C4B614AB3F90410B2F9062091
:105978005F4E6048CDED0C7A8CF0220383EA031366
:10598800DFB23B0983F0590343EA072383EAC703DD
:10599800B2F5FA6F1BB2A8BF4FF4FA6283EA031795
:1059A800FFB2B2F57A7FC3F3072383EA1713B8BFB0
:1059B8004FF47A724FF0640E43EA0723A2F57A7225
:1059C8000EFB02F283EAC70386FB02E680FB01E0D6
:1059D8001FB2D217C9174FF00008C2EBA612C1EBCD
:1059E800A00187F0C806ADF83A20ADF83810CDF818
:1059F8002880CDF82C80CDF834800DF1280E86EA69
:105A08000616BEE80F00F6B2C7F3072787EA16178F
:105A180047EA062787EAC606374FDEF800E084F82B
:105A280004C00FC736B286F04A0383EA0313DBB219
:105A3800C6F3072181EA13113A4641EA03210CF122
:105A4800010C81EAC303142042F810E9FE264FF046
:105A58004A0E002184F86EC14FF0C80CE070238014
:105A6800043784F807E0A670617184F806C0184608
:105A780012F8011B414081EA0111C9B20B0983EAFE
:105A8800102343EA012383EAC10109B288B2BA426A
:105A98002080EDD181F0140181EA0111C9B24FEAE9
:105AA800111E8EEA102E8EEA012E8EEAC10E0FFA12
:105AB8008EFE1FFA8EF6074F26804FEA16295FFAE8
:105AC8008EFE84F81D9084F81CE079683868BA68FE
:105AD800FB6813E0361E0020883F002088C3E43AA4
:105AE800CB1F00207051002000000000404500201E
:105AF800D34D6210676666663C1E0020B7F81880B2
:105B080007F5CB7CACE80F0038697969ACE803008D
:105B180004F29716ACF8008084F8B391B04684F884
:105B2800B2E104F2B31918F8011F286808F0C2FBA3
:105B3800C145F8D1C94BCA4A1B781278013B12F00B
:105B48000100DBB214BFC0214021172B03D8C54A7E
:105B5800134493F830A0C44B1A8893071ABF002344
:105B680041F01001012312F4027F18BF022312F042
:105B7800100F18BF062312F0200F18BF102300289B
:105B880041F0BC814FF0030C94F86E910A9389F0B0
:105B9800460383EA0313DAB2130983F0920343EA54
:105BA800022383EAC2031BB283EA0310C0B2C3F321
:105BB800072282EA101242EA002282EAC00212B2E6
:105BC80082F0C80E8EEA0E1E5FFA8EFEC2F307221E
:105BD800002382EA1E1203208DF82CA08DF82FC016
:105BE8008DF82D3042EA0E2C8DF82E108DF83000ED
:105BF8000AAA07CA8CEACE0E0FFA8EFEDFF878A240
:105C0800E3718EEA0E1CAAE803005FFA8CFCCEF35F
:105C1800072E8EEA1C1E4EEA0C2181EACC0C94F861
:105C280008E08AF800200FFA8CFC8EEA0C0E8EEA47
:105C38000E1E5FFA8EFECCF3072282EA1E1242EA9B
:105C48000E22607AA17A94F80BC0637182EACE02C0
:105C580012B2504080EA001E5FFA8EFEC2F307209F
:105C680080EA1E1040EA0E2080EACE0000B24140D1
:105C780081EA0111C9B2C0F3072282EA111242EA8D
:105C8800012282EAC10212B28CEA020C8CEA0C1CD4
:105C98005FFA8CFCC2F3072282EA1C1242EA0C2249
:105CA80094F80CE0607BA17B94F8108084F8049051
:105CB80082EACC0212B28EEA020E8EEA0E1E5FFA59
:105CC8008EFEC2F3072282EA1E1242EA0E2282EAFE
:105CD800CE0212B2504080EA0010C0B2C2F30722CE
:105CE80082EA101242EA002282EAC00212B251404D
:105CF80081EA0111C9B2C2F3072282EA111242EA0B
:105D0800012282EAC102E17B13B281EA030282EA3C
:105D18000212D2B2C3F3072383EA121343EA02231F
:105D280083EAC2031BB288EA030282EA0212D2B2F1
:105D3800C3F3072383EA121343EA022383EAC20365
:105D48001BB283F0320282EA0212D2B2C3F30723F3
:105D580083EA121343EA022383EAC2031BB29AB20C
:105D68004FF0FE0C4FF0090EC82009F10101DBB21B
:105D780084F802C084F803E04FEA122CA07184F87A
:105D88006E11228084F812C0637438687968BA6822
:105D9800B7F80C900AF5C47EAEE807000AF5CC7A8D
:105DA8008EF80280AEF8009084F8A8C184F8A73174
:105DB80016F8011F286808F07DFAB245F8D1C4F832
:105DC80058B1FFF7BAB9DFF8B4A0DFF8B480DFF84C
:105DD800B490412016F04CFABAF9023088FB03203F
:105DE800DB17C3EBA00080B216F028FABAF900302E
:105DF80088FB0320DB17C3EBA00080B216F01EFA65
:105E0800BAF9043088FB0320DB17C3EBA00080B28B
:105E180016F014FA99F80010386808F04BFA94F85C
:105E2800503113F0010800F01385104AC4F84CB142
:105E38000133DBB2A2FB0312D20802EB8202A3EB0E
:105E4800420384F85031FFF759B9094B09491868DA
:105E580008F000FA00232370FFF7FDB93C38002052
:105E6800FE56002044BC020872500020CDCCCCCC99
:105E780068510020B85000203C1E0020883F0020B8
:105E88006766666642460020114694F8AC32B14A0D
:105E9800C4F8A81202EB8302926C42B312AD04F26A
:105EA800B323AD4E45F8203D002104F2C5233180CF
:105EB8000B9380211523A52784F8B232284684F84D
:105EC800B11284F8B072904728463188FEF7B7F9C6
:105ED8000A9DA24804F52C716D1A152DA8BF152529
:105EE8002A4623F065FB9E4A94F8AC3215709D4A09
:105EF800013382FB0312A2EBE37202EB42029B1A0C
:105F080084F8AC32FFF72BB9974A984B92F80BE01C
:105F18003068D4F824211B889549801A4FF47A7286
:105F2800DFB202FB0EF21B0A8F770F7590424FF01B
:105F38000007CB774B758F700F7180F00C848D4BF9
:105F4800DFF83C821B68029F8B4AC4F8207188FBEB
:105F5800037CDB171068DFF840E29268C3EB6C1330
:105F6800D4F818C188FB0C878EFB00988EFB029E24
:105F7800D217C2EBAE0203F5FA734FEAEC7E9BB27E
:105F8800CEEB671EC0170CF5EA47C0EBA800303708
:105F98008B761B0A0EF1780E3F120CF1300CCB7683
:105FA8004FEA20281312087781F81D8081F82020F5
:105FB80081F8213081F824E081F8237081F822C02B
:105FC800FFF717B8DFF8D491D9F8000008F066F9A0
:105FD80000283FF4A0A8D9F80000012108F05AF9D8
:105FE8000222002387F8742088F80030FFF793B85E
:105FF8003B685E2098473B68022098475F4B604AA1
:106008009B6A323382FB0328DB17C3EB68185FFAFD
:1060180088F016F00BFAC8F3072016F007FA3B6869
:106028005E2098473B6803209847564B1B78D90752
:1060380040F1D48321F0F0F8534B9FED547AD3ED1F
:10604800037A67EE877AFCEEE77ACDED037ABDF83E
:106058000C30002800F0D586D8B24FEA132816F085
:10606800E5F9404616F0E2F9DFF8348198F8053092
:10607800002B40F0A8840AA9454816F09BF93B6814
:106088005E2098473B6813209847BDF928805FFA3F
:1060980088F016F0CBF9C8F3072016F0C7F93B686B
:1060A8005E2098473B681B209847BDF92A805FFA15
:1060B80088F016F0BBF9C8F3072016F0B7F93B686B
:1060C8005E2098473B68232098474E2016F0AEF98B
:1060D800002016F0ABF90AA92D4816F06BF93B68B9
:1060E8005E2098473B6812209847BDF928805FFAE0
:1060F80088F016F09BF9C8F3072016F097F93B686B
:106108005E2098473B681A209847BDF92A805FFAB5
:1061180088F016F08BF9C8F3072016F087F93B686A
:106128005E2098473B6822209847452016F07EF964
:10613800002016F07BF93B685E20984794F81431EC
:10614800FEF747BF134CDFF85C904FF0010B4FF0A0
:10615800000A32E044BC020874500020F42D0020EC
:10616800092E002056555555BC3C0020B43C002053
:10617800385100202C220020103C0020043600203A
:106188001F85EB51FE560020CC3C0020CDCC4C3E68
:1061980080969800341E002067666666E8540020E2
:1061A80078510020000000201B2B00F044820D2BAA
:1061B80000F00F8289F801B0386808F077F80028F5
:1061C80038D0386808F06EF883B27E2B32682AD04F
:1061D80099F801100029EFD194F83621002AE3D06C
:1061E8007D2B00F0078294F844E1BEF1000F04D043
:1061F80080F02003DBB284F84411511CC9B2224458
:10620800092984F8361182F8383100F0E981082923
:10621800D2D8B4F84221134403EB132303F0FF034D
:10622800A4F84231C8E784F836A184F837A189F880
:1062380001A0C1E794F8453133B194F8393184F8B5
:106248004501302B00F0FB8594F83721C04BDFF86F
:1062580038C3DFF830B3DFF834E3DFF834A30127BD
:10626800002A3EF43BAF3168A1EB0801012900F296
:10627800AB8194F84691B9F1000F40F0E58194F8AC
:10628800471133F8110010B984F84771E8E7013174
:10629800B0F5826F84F8471100F0DC801ED9B0F5A4
:1062A800E26F00F09A8034D9B0F5046F00F0A38053
:1062B800B0F5116F00F02181B0F5E46FD0D1A54A97
:1062C800176C918A642303FB07F393FBF1F116F033
:1062D80005F8002384F83731FEF700BFB0F5007FDA
:1062E80000F095802DD8B0F5807F00F02081B0F5C2
:1062F800887FB5D1DCF800104907B1D5D4F818115A
:106308004FF4887015F0EAFF002384F83731FEF760
:10631800E5BEB0F5C06F00F08D80B0F5E06F9FD19D
:106328008C4A906B918A642303FB00F34FF4E0607E
:1063380093FBF1F115F0D2FF002384F83731FEF713
:10634800CDBEB0F5047F00F02581B0F5806F87D110
:1063580094F848310133DBB2032B00F2508142F24A
:10636800107184F8483101FB03F17B4B1B88002B2B
:1063780040F043810131794B1B78DF07784B1B884C
:1063880048BF0431D80748BF0A319A0748BF1431BB
:106398001F0648BF2831D80548BF28315A0748BFCB
:1063A80064311F0748BFC831980548BF01F5C87157
:1063B8009A0648BF01F57A71DF0648BF01F5FA6110
:1063C800580648BF01F57A614FF4806015F086FFE2
:1063D800002384F83731FEF781BE5E4AD76B918A75
:1063E800642303FB07F393FBF1F115F077FF84F8BF
:1063F8003791FEF773BE5B4BB3F9041001EB8101D3
:10640800490015F06BFF84F83791FEF767BE9EF8D8
:10641800061000293FF424AF534B54491B6881FBF5
:106428000321DB17C3EBA10115F058FF84F837915E
:10643800FEF754BE9EF8061000293FF411AF4A4BF0
:106448004FF4C060996815F049FF002384F837318C
:10645800FEF744BEDCF8001011F020097FF400AF0D
:1064680043490868010600F1D4849BF80C10002900
:106478003FF4F6AE94F84911032900F23686DFE8B6
:1064880001F0322819023B4B1B6859799A79DB795C
:1064980001F1407101EB022101EB0341002384F873
:1064A80049314FF4826015F019FF002384F8373121
:1064B800FEF714BE304B1A68137A507992781B0491
:1064C80003EB002313444A1C84F8492103EB0161C0
:1064D800E7E7294B1A68D379107952781B0403EB44
:1064E80000231344EFE7244B1A689379D078127885
:1064F8001B0403EB00231344E5E79EF8051000296D
:106508003FF4AEAE9AF8001000293FF4A9AE1B4B39
:106518001B8803EB83035B004FF4116093FBF1F1DD
:1065280015F0DCFE002384F83731FEF7D7BDDCF820
:10653800001048077FF594AE114B4FF4807019682E
:1065480015F0CCFE002384F83731FEF7C7BD00BF35
:1065580044BC0208403F0020E03E0020FE560020D8
:1065680072500020883F0020103C00206766666655
:106578006C490020045D0020183F0020B43C002036
:106588002C220020BC3C00207051002078510020B3
:10659800CA3C00209EF8051000293FF461AE9AF825
:1065A800001000293FF45CAE9A4B5B7B002B00F097
:1065B800AF84994B1B8893FBF1F101EB81014900F2
:1065C8004FF4047015F08AFE002384F83731FEF783
:1065D80085BD84F836B184F83831A4F84221EBE55A
:1065E800B4F84221C2F1FF0293427FF4E3AD84F88C
:1065F80045B1DFE584F844B1DEE50231BBE60123AD
:1066080084F8483142F21071AFE607F057FC834B2B
:106618001B68C01A40F6B833984200F2B681DFF81A
:1066280020B29BF804303A2B00F01A83002388F834
:106638000030FEF770BD386807F038FE00287FF498
:10664800B9AD84F837B1B7E57549062015F066FC91
:10665800002384F8460184F83731FEF73FBD94F8EB
:10666800341194F835316F484A1CFEF71EBD4FF0BF
:1066780000083B68D6F8009084F814815E2098479B
:106688003B68694C17209847404615F0CFFE674B8A
:10669800A3FB09239B0BA4FB03125209C2EB0212B2
:1066A800A3EB8203D8B215F0C1FE3B685E20984781
:1066B8003B68182098475E4BA3FB09239B09A4FB62
:1066C80003125209C2EB0212A3EB8203D8B215F0EF
:1066D800ADFE404615F0AAFE3B685E209847FEF7DF
:1066E8007BBC013B84F85E31FEF731BF013B84F887
:1066F8005F31FFF74DB80AF1FF3A84F867A1FFF759
:106708005EBB0CF1FF3C84F866C1FFF718B90024A2
:10671800484FA0464FF0500902E0DBB283F31188DE
:1067280015F804A0601C5146284415F09BFC00286D
:1067380040F040810AF101031C44EFF3118389F30F
:1067480012882A6E9442E8DB0022DBB22A6683F3C1
:106758001188FEF7EABD384B32681B78C4F824214B
:10676800013B012B3FF6EBAB102202238A700B7121
:10677800FFF7E5BB3B68DFF8CCB0DFF8CC905E20D4
:1067880098473B6810209847DBF8003089FB032ABC
:10679800DB17C3EB6A1A5FFA8AF015F047FECAF3F3
:1067A800072015F043FE3B685E2098473B68212090
:1067B8009847DBF8003089FB0329D8176422C0EB1F
:1067C800691002FB10300028B8BF4042C0B215F073
:1067D8002DFE404615F02AFEFEF775BDDFF86C80E9
:1067E800164BB8F80890A3FB09394FEA99095FFAE4
:1067F80089F015F01BFE4FEA192015F017FE35E455
:1068080015F0BAFDFEF759BC15F0A6FD01233B7043
:10681800FEF70FBCBC3C0020B43C00209054002084
:10682800DFC20108883E00208988888873B2E7455E
:10683800D34D62109D250208B73E0020CDCCCCCCAC
:10684800785400202C2200201F85EB51785100201D
:10685800B64B1B88DA0515D4D80600F12F849906A3
:1068680000F13F845A0600F14E84180700F16B844A
:10687800D90700F1648413F0020F0CBF4FF004082D
:106888004FF00C08AA4BAB4A1B78D27803F00103EF
:106898000AB143F002035320039315F0E9FCA64A1A
:1068A800128802EB820202EB8202900080B215F09D
:1068B800C5FC002015F0C2FCA04AA149128838681E
:1068C800C2EBC212520081FB023111444FEAE27A54
:1068D800CAEB612A5FFA8AFA514607F0EBFC99F88D
:1068E8000020039B386848EA03088AEA020A002164
:1068F80089F800A007F0DEFC4146386807F0DAFCAA
:1069080099F80030386888EA0303DBB2194689F839
:10691800003007F0CFFC94F85031002B7FF485AAA3
:106928004F2015F0A5FC19F091F919F08FF919F01D
:106938008DF90121386807F0BDFC824A99F80030CA
:1069480092F80080386808F0010883F00103414696
:1069580089F8003007F0AEFC99F80030386888EA0A
:106968000303194689F8003007F0A4FC94F8503165
:10697800FFF75BBA744B9FED757AD3ED007AF8EEAA
:10698800E77A67EE877AFEF7EBBF714AB2F85231C1
:1069980000210133A2F8523188F80010FEF7BBBB82
:1069A800884689460846049105918E4606910391CA
:1069B800FEF700BE39463A2015F0B0FA40EA08085A
:1069C8005FFA88F8B6E6DFF898B19BF800A0BAF14C
:1069D800000F3FF450AB584AB4F81CE111883B68EB
:1069E80003924FEA0E1E64201FFA8EFE00FB01A1DF
:1069F8004FEA4A00B1FBF0F14EEA012E1FFA8EFE73
:106A0800C1F303215E204EEA010998473B6806203E
:106A180098475FFA89F015F009FD4FEA192015F03B
:106A280005FDB4F81C31039A4A49B2F800904A7A35
:106A380001339BB2012A93FBFAF00AFB1033A4F846
:106A48001C3100F06D836E2343484A7B03FB09F336
:106A580080FB03014FEAE379C9EBA1092AB11FFAC8
:106A680089F99BF8003099FBF3F93B68DFF8F4A04B
:106A78005E2098471FFA89F93B683A209847AAFB95
:106A8800093A4FEA5A1A1FFA8AFB5FFA8BF015F097
:106A9800CDFC4FEA1B2015F0C9FC3B685E209847E7
:106AA8003B683B209847642303FB1A939BB22B480F
:106AB800053380FB0320DB17C3EBA000C0B215F041
:106AC800B5FC002015F0B2FC3B68DFF89CA0DFF8AD
:106AD8008C905E2098473B6828209847DAF8003069
:106AE80089FB0329DB17C3EBA9095FFA89F015F0C5
:106AF8009DFCC9F3072015F099FC3B685E20984778
:106B08003B6804209847B8F80830002B40F0FF8213
:106B1800DAF8083083F310085FFA88F015F086FC7D
:106B2800C8F3072015F082FCFFF7A5BA72500020C1
:106B3800FE560020BC3E0020B43C002070500020CF
:106B480003082080C43200202C2200200AD7233CCE
:106B5800341E0020BC3C0020310CC33067666666DA
:106B6800CA3C00201F85EB51103C0020B849B94BA6
:106B78000093A1F13F06B84BB84A099101F8404C7F
:106B88000AA8B7490896FDF731FC089E731C0893BC
:106B98003470089B2922591C08911A70089BEA2214
:106BA800591C08911A70089BC822591C08910AA8F8
:106BB8001A7021F065FD471C0AA93A46089822F088
:106BC800F7FC089AD31901330893D455089B5A1C2B
:106BD80008921C70089B5A1C08921C70089B5A1C2F
:106BE80008921C70089B5A1C08921C70089B5A1C1F
:106BF80008921C70089B5A1C08921C70089B5A1C0F
:106C080008921C70089B5A1C08921C70089B5A1CFE
:106C180008921C70089B5A1C08921C70089B5A1CEE
:106C280008921C70089B5A1C08921C70089B012231
:106C3800991812A808911A7050F8283D9B1B3370B8
:106C48001BF078FC874B029A2C70C3F8A022FEF741
:106C580079BA029BC4F8283187F80080FEF7E9B9B1
:106C68009BF80240C4B1013CE4B201345C4459468B
:106C7800002211F8013B534083EA0313DBB2120AE6
:106C8800DF0042EA03228C4287EA131382EA0302F6
:106C9800EFD1002A7FF4CAAC734A744F744B128840
:106CA8007449704CFA61DFF8E0911A6809689B68CA
:106CB800FA62B4F85221F866FB64D9F80000F96367
:106CC800FA6505F07BFD824600287EF41FAA0221A2
:106CD800D9F8000007F0DEFA94F854319BF8032045
:106CE8000492642B4FF0040287F8742040F0548219
:106CF80094F85531072B08BF84F855A194F85531FD
:106D0800069307EB031ADAF804100391084621F0FA
:106D1800B7FCDAF8081005915FFA80FA084621F006
:106D2800AFFC5FFA80FB069B5348039903900AEB7C
:106D38000B020832C27123F00F0282724E4A03F02E
:106D48000F0353734C4B0BEBCA009873184652460B
:106D58000F3022F02DFC494B05990AF1090018441F
:106D68005A4622F025FC0398C37903F1010ACBB1F6
:106D7800013B5FFA83FC0CF1080CDFF810E1844456
:106D88000023073010F8012B5A409300D10883EAFA
:106D9800420301F0180153404EFA01F25340844572
:106DA800DBB2EFD1354A04980AF8023018F01CFF1C
:106DB80094F855310022013384F8553184F8542170
:106DC800039BDDF80CA09B785BB11AF80510D9F885
:106DD800000007F06FFA01359AF80230EDB2AB42C5
:106DE800F3D894F854310322013384F8543187F8E6
:106DF800742088F80020FFF7E7B807F04BFAFEF791
:106E08002DB91F4A1268D2067FF526A98046FFF7DA
:106E180026B91023042218460AA98DF82A908DF85D
:106E28002B908DF82C908DF82D908DF828308DF8BA
:106E3800292015F035FA84F83791FEF74FB9062165
:106E4800104815F00FF984F84601FFF7FDB900BFA7
:106E5800B8500020113F002084E102088CE10208AC
:106E680098E10208341E0020B43C002000000020F5
:106E7800103C00202C220020AC410020B241002010
:106E88006C4900206E1F0020E85400200007090EFE
:106E9800AF4BB04A0B93A3F140071268002103F8E7
:106EA800401C2123BB70D30040F10F81AA4903265F
:106EB800AA4B1B88580500F10581DA0700F12081EB
:106EC80003F00203A64A002B1CBF03261146DFF875
:106ED800C0823246404622F06BFB06EB080312A83C
:106EE8000133A8F1020140F8203D00225B1A06F8A0
:106EF80008207B701BF01EFBFEF7D3B9994AD278A5
:106F0800002A0CBF4FF0040C4FF0050CFEF73CBEF6
:106F1800954B1988FFF751BB0123D9F800003B7046
:106F280007F0C0F90746D9F8000007F0BBF97F065B
:106F38007EF47FA88E287EF47CA89AF80030002B77
:106F48007EF493A8894B8A4A1A602D2384F82C3141
:106F5800FEF776B87E4B844A0B9312AFA3F13D003F
:106F680047F8200D1188DFF81482A3F140020020B1
:106F78004FF00A0E03F8400C082382F801E0384667
:106F88009370FDF738F9D8F800307A49DA1781FBA1
:106F98000313C2EBA30399B23846FDF72CF90EF0A0
:106FA8005BF8D8F808800A9B4FEA1842591C0A91E6
:106FB8001A700A9B4FEA1822591C0A911A700A9BE8
:106FC8005A1C0A9283F800800A9B5A1C0A9218706D
:106FD80038461BF0AFFAFEF761B9DFF8B8819FEDCC
:106FE800668AB8F902305A4A0B9207EE903AF8EEE0
:106FF800E77A12AF67EE887AA2F14003FDEEE77AEE
:10700800A2F13D0147F8201D02F8400C0822CDED01
:10701800037A5A701E229A70BDF80C103846FDF794
:10702800EAF8B8F9003007EE903AF8EEE77A384611
:1070380067EE887AFDEEE77ACDED037ABDF80C109D
:10704800FDF7D9F8B8F9043007EE903AF8EEE77A88
:10705800384667EE887AFDEEE77ACDED037ABDF81B
:107068000C10FDF7C8F838461BF064FAFEF713B9A0
:10707800424B9046B3F900A06420FEF7A3B93A4901
:107088009A790B8803EB830303EB83034FEA8308A6
:107098001FFA88F8002A40F01F814FF0FF330FFADB
:1070A80083FA0DF0D9FF40B2FEF78CB9984699469D
:1070B8001846049305930393FEF77CBA4FF03408FF
:1070C800FFF7E0BB03262E4901E72E4B2E4A1B682B
:1070D800214903F48003002B0ABF11460326042626
:1070E800E6E64FF02408FFF7CDBB4B1CDBB2042BC0
:1070F80084F849314FEA01617FF4D3A9FFF7CEB98B
:1071080022490426E3E64FF01008FFF7BBBB0DF059
:10711800A3FF15F08BF9002015F088F9FEF7ABBF37
:107128003B685E2098473B68392098475FFA89F0AA
:1071380015F07CF94FEA192015F078F9C4E44FF0FE
:107148000808FFF79FBB4FF02008FFF79BBB00BF65
:10715800B8500020C837002068E1020872500020AB
:1071680080E10208BC3E0020B43C0020903E002094
:10717800385100206766666658A08B41103C002095
:1071880074E102086C4900206CE1020878E1020809
:107198007B500020883F002097F875A059491AF0C5
:1071A8000F0F04BF0AF1010A5FFA8AFABAF1070F52
:1071B80028BF4FF0010A4FEA0A1B07EB0B035FFADF
:1071C8008BFC187C504B03930A18002392F8241068
:1071D8004D4A937202F10D0307EB0B024CEA0000D3
:1071E80001291870D26803F1010E0CD90239C8B20E
:1071F800811C1944734603F8012B8B424FEA122273
:10720800F9D101308644BB4422F060030AF1010A37
:107218009BF811205FFA8AFA1343BAF1080F8EF827
:1072280000300EF1010344D04FEA0A1B07EB0B01B3
:10723800364A087C334901449A1A91F8241002EB23
:10724800010E0CF1100CBEF1130F5FFA8CFCC3DDBC
:107258005FFA82FB0BF10603DBB20398DFF8B8E0B4
:1072680043F04002C27103F1010CD3B10BF1050BDD
:107278005FFA8BFB0BF1080B834400230EF101002E
:1072880010F8011B59408B0083EA4103CA084B40A0
:107298001F4902F0180241FA02F253408345DBB25B
:1072A800EED104980CF80E3087F875A018F09CFC05
:1072B80086E5164A9A1ACBE79846994618460493E3
:1072C80005939E460393FEF775B998469946184666
:1072D80004930393FEF76EB90E4B1B68DFE6039326
:1072E800FEF768B998460393FEF764B9984699463D
:1072F8000393FEF75FB99846994618460393FEF73D
:1073080059B900BF44BC0208AC410020B941002073
:107318000007090E103C0020B24100202DE9F04F73
:107328002DED0C8B3C4B1B7895B0012B0A9001F08E
:1073380049873A4C94F80021002A41F0EF80072B46
:10734800374D01F00D87002305936B683448984743
:10735800002800F06981B5F8B470002285F855203E
:10736800002F40F03F87B5F93E00AA6AB5F93C60A6
:10737800696AB5F94030DFF8B4B0821AE86A6A631E
:10738800711A1B1A2963274895F85610AB630FF03A
:10739800B7F9DBF80030990040F1F08095ED0D7AEF
:1073A800D5ED0C7A204A94ED725AD4ED735A94EDC7
:1073B800746AD4F8D4311268F8EEC76A95ED0E7A7B
:1073C800F8EEE77AB8EEC77A013377EE857A36EECB
:1073D800A58A77EE068A9342C4ED727A84ED738AA1
:1073E800C4ED748AC4F8D43101F03C840A4B1F7888
:1073F800142F03F0D9800023D4F8DC610693062EFD
:1074080000F2AF80DFE816F01F170B173C16A01626
:1074180014006118FA1700BFA43C002000210020C6
:10742800D846002008470020582F00206C4900202B
:10743800D84B1A78D4F8E0E1DFF8CCC39FEDD67AC0
:107448004FEACE000CEB000383ED007A002A7DD0D2
:10745800D249B0EE476AF0EE476A0023F1EC017AB0
:10746800013367EEA77A05EE903AB4EEE77AF1EECB
:1074780010FAF8EEE55AB8BFB0EE677A9A4276EE9F
:10748800A76AA7EEA56AE9D1F5EEC06A0CEB00037E
:10749800F1EE10FA83ED007A58DDC6EE265AC04B9D
:1074A800C04A1288F7EE007A75EEE75AD3ED007AF3
:1074B80065EEA77AFDEEE77A17EE903A812B43F353
:1074C800FC869342A8BF134607EE903AF8EEE77A97
:1074D800B54B00EB0E0103EB810393ED057AD3ED79
:1074E800003A93ED066A93ED014AD3ED046AD3EDB1
:1074F800034A93ED025AA3EEA77AA4EE276A66EE32
:10750800C76AA7EE646ABDEEC77AE5EE276A17EE8A
:10751800101A812983ED056AC3ED066A43F3CA860A
:107528008A42A8BF0A4607EE902AF8EEE77AFCEEF0
:10753800E77ACDED077ABDF81C300CEB000293809A
:10754800BEF1000F02D1132F04F05083152F42F023
:10755800EC856044DFF8B482838828F81E30D4F8BC
:10756800DC61924B013683FB06239A19F317C3EBB0
:10757800A203C3EBC303F61AC4F8DC618C4B1B7877
:10758800002B01F0D3818B4EDFF88492DFF87CA2C8
:1075980006F5BC780027884BD5ED087A1B78172BA1
:1075A80001F0398496ED007AB8EEC78A082B28EEE8
:1075B800278A07D1B0EE480A069322F06DF9069B98
:1075C8002AF81700DBF8002092000BD5002F04F0F2
:1075D8009F87B0EE480AD5F8143208F17000984732
:1075E800B0EE408AB0EE480AD5F83431A8F1700000
:1075F8009847D5F8A431404698476F4B1B78032B22
:10760800B0EE408A01F01484D6F8F800D5F8B83006
:10761800B0EE480A98470137032F08F12408A9EC6F
:10762800010A06F10406B6D1634B93F80090B9F14C
:10763800070F00F0928694F8E431002B40F09A8608
:107648005E4B5B79002B40F0C78501235A4A84F8CA
:10765800E4311278072A02F0D28100230B93584BA9
:1076680094ED7A9A93ED007A564BD4ED41CA1B6893
:107678000593F7EE007A37EEC9CA534B06932CEE02
:1076880007CA524B0893B4EEE7CA514B0993002539
:10769800504BDFF88091DFF880B1DFED4F8A9FED26
:1076A8004FAADFED3DBADFED4E9A9FED4EBADFED02
:1076B8004EAADFF86881DFF868A14C4F0793F1EE16
:1076C80010FA88BFB0EE67CA2E46494B99ED008A7A
:1076D8002B44D3ED007AF5EE407AF1EE10FA17D08C
:1076E800444B2B44D3ED006A38EE667AB0EEC76A95
:1076F800F4EEC67AF1EE10FA08D5B5EEC07AF1EEDE
:1077080010FACCBF37EEA68A36EEE78A83ED008AF8
:10771800069B1A88930700F08580022E00F082806D
:107728000599354B91F82E102B4407EE901A93EDDE
:10773800007A4B42F8EEE76A07EE903A26EE877A2F
:10774800F8EEE77AB4EEE77AF1EE10FA0AD407EE2B
:10775800901AF8EE677AF4EEC77AF1EE10FA88BF5D
:10776800F0EE477A254B264903EB460331F916001C
:10777800B3F90C30C01A07EE100AB8EEC77AD00772
:10778800E7EE687A40F12C861E4B93ED008A27EECF
:10779800888A47E05E2F00200000000000210020BA
:1077A800602F00205C2F0020943100209324499200
:1077B800542F002008470020A43C0020C446002085
:1077C800B4260020183F00207250002078000020C6
:1077D800FE5600205C490020CDCCCC3DAE47813F11
:1077E8000000C84200003443610BB63BEC35002072
:1077F800A8260020EC220020A0220020003800202B
:10780800883F0020902600207C310020A83C0020E2
:107818006049002038220020A0250020F8350020EB
:10782800E0350020079B94F8F8212B44D3ED01DACA
:1078380038EE6DDA002A38D0D54BD4F8FC210A99F5
:107848001B688A1A9A4230DD022E04F0AA85D14BB1
:107858001B68990741F15E80CF4BD049DFF8ACE354
:1078680031F916C09EED008ADFF8A4E3C7ED00BA2F
:1078780003EB460028EE288AB0F90C00A0EB0C00B8
:1078880007EE900AF8EEE77ADEF8000027EE888A1D
:10789800824238EE6DDA01F39B82F7EE007AB4EE9D
:1078A800E79AF1EE10FA01F16A82BD4B2B4493ED91
:1078B800000A2CEE800A022E20EE0D0AAAEC010A1C
:1078C80004F02D85089BDBED007A93ED007AB54B2B
:1078D800D7ED006A93ED006AB34B67EE277A2B4425
:1078E80027EE8C7AD3ED007A67EE277AF0EE665AA7
:1078F800EDEE275AB1EE467AB4EEE57AF1EE10FADB
:1079080008DCF4EEC65AF1EE10FA8CBFB0EE467AF7
:10791800B0EE657A94ED7A6AF7EE007AB4EEE76A2B
:10792800F1EE10FAACBF0123002343B1F0EEE66A92
:10793800F0EEC77AF4EEE67AF1EE10FA01D587EDAB
:10794800007A022E04F08D84984A994B52F826004A
:107958001B68B0EE6D0A9847964A974B52F8260076
:107968001B689847059B93F8373023B1069B1B8803
:10797800002B00F09985B0EE6B8A904B9BED007A56
:1079880038EE400A2B4493ED008A83ED000A059BEC
:1079980030EE480A93F84830C0EE077A33B3099BB3
:1079A8001B78D80740F1128594F8F831B7EE007AC1
:1079B800B4EEC79AF1EE10FAC0F2E484002B40F05E
:1079C800E4847F4A92ED007AF0EEE76AF4EEC76A43
:1079D800F1EE10FA0ADD7B4A92ED007AF0EECD6AFC
:1079E800F4EEC76AF1EE10FA02F3F385764B94F8D9
:1079F80008222B4493ED007A2CEE877A67EE277ADB
:107A0800C8ED007A2AB94AED01BAC7ED00BAC8ED47
:107A180000BA0136032E09F1040908F1040807F138
:107A2800040705F104057FF450AE684B1B78072B5B
:107A380001F01284012B01F0E787002594F8103239
:107A4800002B40F03187624A624B10681B6810F4C3
:107A5800805E93F82C3040F093875F4A5F4992ED3F
:107A6800006A498B5E4A84ED886A92ED007A5D4A25
:107A780084ED897A07EE901AF8EEE76AD2ED037A78
:107A8800594A84ED866A37EE467A77EEE67AD2ED81
:107A9800006A84ED857A012284F82822C7EEA65A66
:107AA8005249534A91ED005A52499FED536A91ED5C
:107AB800004A5249DFED526AD1ED004A92ED007A50
:107AC80035EE045AF7EE007AF4EEE75A35EE245A0A
:107AD800F1EE10FA88BFF0EE675A25EE065AF4EE7A
:107AE800E65AB1EE476AF1EE10FAB4EEC65AB8BFDC
:107AF800F0EE665AF1EE10FAC4ED8B5A01F184816A
:107B0800B4EEC75AF1EE10FA88BFB0EE475A374ABA
:107B1800DFED396AD2ED017A364A92ED014A374AE9
:107B280077EE847AD2ED014A77EEA47A67EEA67AE8
:107B3800B4EEE76AF1EE10FA08DCB4EEE77AF1EE9B
:107B480010FA8CBFB0EE676AB0EE476A274ADFEDDD
:107B58002A6AD2ED027A274AD2ED024A294A77EEFA
:107B6800A47A92ED007A67EEA67AB1EE473AF4EE7F
:107B7800C37AF1EE10FA08D4F4EEC77AF1EE10FAEF
:107B88008CBFB0EE473AB0EE673A1F4A527841E0F0
:107B9800BC2600207051002000380020883F0020BB
:107BA80064260020D826002070260020A825002062
:107BB800A4250020FC250020F82500200023002013
:107BC800CC260020C82600207C260020A43C0020CB
:107BD8006C490020183F002068360020B84E00206D
:107BE800D0370020CC3C002098270020E03500202A
:107BF800DC260020EC3500206F12833AF83500208F
:107C080000000000E02600203C38002090260020DC
:107C1800B82600200AB9B1EE433A002B41F0F084AF
:107C2800F7EE003AF04E3278002A03F03380EF4B3B
:107C3800DFEDEF7AD3ED024AD3ED016A93ED037AD3
:107C480066EE244AE5EE264AE3EE074A63EEA44AC6
:107C5800F4EEE74AF1EE10FAB4BFB0EE674AB0EEC0
:107C6800644A98BFF0EE647A012ACDED0C4A03F01D
:107C7800368093ED067AD3ED052AD3ED076A26EE12
:107C8800077AA5EE227AA3EE267A23EE877AB4EE57
:107C9800E77AF1EE10FAB4EEC47A8CBFF0EE676AB8
:107CA800F0EE476AF1EE10FA88BFF0EE676AB4BFEB
:107CB800F0EE447AF0EE477A022A8DED0D7A00F064
:107CC800DE8093ED0A7AD3ED092A93ED0B4A26EE6E
:107CD800077AA5EE227AA3EE047A23EE877AB4EE29
:107CE800E67AF1EE10FAB4EEE77A8CBFB0EE664AA7
:107CF800B0EE474AF1EE10FA98BFF0EE446AA8BF1A
:107D0800F0EE477A032A8DED0E7A00F0B88093EDF5
:107D18000E7AD3ED0D2A93ED0F4A26EE077AA5EEDB
:107D2800227AA3EE047A23EE877AB4EEE67AF1EEAD
:107D380010FAB4EEE77A8CBFB0EE664AB0EE474A66
:107D4800F1EE10FA98BFF0EE446AA8BFF0EE477A59
:107D5800042A8DED0F7A00F0928093ED124AD3ED4C
:107D6800112A93ED137A26EE044AA5EE224AA3EED1
:107D7800074A23EE844AB4EEE64AF1EE10FAB4EE6E
:107D8800E74A8CBFB0EE667AB0EE447AF1EE10FAAC
:107D980098BFF0EE476AA8BFF0EE447A052A8DED49
:107DA800104A6CD093ED164AD3ED152A93ED177A45
:107DB80026EE044AA5EE224AA3EE074A23EE844A99
:107DC800B4EEE64AF1EE10FAB4EEE74A8CBFB0EE34
:107DD800667AB0EE447AF1EE10FA98BFF0EE476A90
:107DE800A8BFF0EE447A062A8DED114A47D093EDEC
:107DF8001A4AD3ED192A93ED1B7A26EE044AA5EE0A
:107E0800224AA3EE074A23EE844AB4EEE64AF1EE8C
:107E180010FAB4EEE74A8CBFB0EE667AB0EE447A58
:107E2800F1EE10FA98BFF0EE476AA8BFF0EE447A78
:107E3800072A8DED124A22D093ED1E7AD3ED1D2A22
:107E480093ED1F4A26EE077AA5EE227AA4EE037A6E
:107E580027EE237AB4EEE67AF1EE10FAB4EEE77A7A
:107E68008CBFB0EE666AB0EE476AF1EE10FA8DED9F
:107E7800137A98BFF0EE466AA8BFF0EE477A77EE1D
:107E8800E67AF7EE006AF4EEE67AF1EE10FAC4ED5F
:107E98007A7A43F3938686EEA77A022ADDED0D7A85
:107EA80067EE244A67EE877ACDED0C4ACDED0D7A60
:107EB8002DD0DDED0E7A67EE877A032ACDED0E7AA6
:107EC80025D0DDED0F7A67EE877A042ACDED0F7A9B
:107ED8001DD0DDED107A67EE877A052ACDED107A90
:107EE80015D0DDED117A67EE877A062ACDED117A85
:107EF8000DD0DDED127A67EE877A072ACDED127A7A
:107F080005D0DDED137A27EE877A8DED137A394B9C
:107F18001F6817F0805701F06E81F6EE005AC4ED25
:107F28008B5A002A02F0AB86334B94ED895A93F8AA
:107F3800039094F928320999D4ED884A91F800C041
:107F4800DFF8C0802D49DFF8C0A0B1F9061098ED20
:107F5800007A059106EE903ABDEEC55A284B9AF87C
:107F680000A0B3F81AB094ED856AD4ED867A15EEC0
:107F7800103ABDEEE45A00F0100800F480000CF04E
:107F8800010CF8EEE66A15EE101A0690B9F1000F2A
:107F980041F06A83B8F1000F41F07381DFF84C803B
:107FA8009DED0C5A98ED007ADFF860E025EE877AAF
:107FB800A6EE857AB0EE675AA6EE075ABDEEC57AE8
:107FC80017EE107A17EE100A9F42A8BF1846B9425A
:107FD800C8BF084607EE100AB8EEC77A012A8EED28
:107FE800007A00F0F18013E0BC440020082700204C
:107FF80000000000C8370020BC3E0020404500209B
:10800800B84E0020E4260020904B00204036002087
:1080180098ED047A9DED0D5A25EE877AA6EE857ABD
:10802800B0EE675AA6EE075ABDEEC57A17EE107A7B
:1080380017EE100A9F42A8BF1846B942C8BF0846A3
:1080480007EE100AB8EEC77A022A8EED017A00F020
:10805800BB8098ED087A9DED0E5A25EE877AA6EE3C
:10806800857AB0EE675AA6EE075ABDEEC57A17EEC6
:10807800107A17EE100A9F42A8BF1846B942C8BF27
:10808800084607EE100AB8EEC77A032A8EED027A80
:1080980000F09A8098ED0C7A9DED0F5A25EE877ABC
:1080A800A6EE857AB0EE675AA6EE075ABDEEC57AF7
:1080B80017EE107A17EE100A9F42A8BF1846B94269
:1080C800C8BF084607EE100AB8EEC77A042A8EED34
:1080D800037A79D098ED107A9DED105A25EE877ABB
:1080E800A6EE857AB0EE675AA6EE075ABDEEC57AB7
:1080F80017EE107A17EE100A9F42A8BF1846B94229
:10810800C8BF084607EE100AB8EEC77A052A8EEDF2
:10811800047A59D098ED147A9DED115A25EE877A94
:10812800A6EE857AB0EE675AA6EE075ABDEEC57A76
:1081380017EE107A17EE100A9F42A8BF1846B942E8
:10814800C8BF084607EE100AB8EEC77A062A8EEDB1
:10815800057A39D098ED187A9DED125A25EE877A6E
:10816800A6EE857AB0EE675AA6EE075ABDEEC57A36
:1081780017EE107A17EE100A9F42A8BF1846B942A8
:10818800C8BF084607EE100AB8EEC77A072A8EED70
:10819800067A19D098ED1C7A9DED135A65EE875A28
:1081A800E6EE855AE6EE257AFDEEE77A17EE900AB6
:1081B8008342A8BF03468142C8BF0B4607EE903AE8
:1081C800F8EEE77ACEED077ABCF1000F40F079833C
:1081D800002A40F0718374E3C14B1B78013BDBB28A
:1081E800FFF734BABF4B07934FF47A761B68B6FB98
:1081F800F3F3C3EB4316BC49DFF81C8391F801A0E5
:10820800BA49B8F9060091F8009003EB8603DE003E
:10821800B6B2B74202F0AA82D5F88810B5F93CE0A8
:10822800EB6E4A1C07EE90EA7344012AC5F88820D1
:10823800EB66F8EEE77A02F0A482D5ED1E5AD5ED8A
:10824800206A07EE102A37EEE56AB8EEC75A012F02
:1082580086EE057A37EE257A77EEC77A85ED1F7AAE
:10826800E7EE866A85ED1E7AF0EE667AC5ED216A3C
:10827800C5ED206A02F06A86D5F89C10B5F93EE093
:108288002B6F4A1C07EE90EA7344012AC5F89C201C
:108298002B67F8EEE77A02F08D82D5ED235AD5EDFB
:1082A800256A07EE102A37EEE56AB8EEC75A012F9D
:1082B80086EE057A37EE257A77EEC77A85ED247A49
:1082C800E7EE866A85ED237AF0EE667AC5ED266AD2
:1082D800C5ED256A02F06286D5F8B010B5F940E020
:1082E8006B6F4A1C07EE90EA7344012AC5F8B02068
:1082F8006B67F8EEE77A02F07682D5ED285AD5ED6D
:108308002A6A07EE102A37EEE56AB8EEC75A012F37
:1083180086EE057A37EE257A77EEC77A85ED297AE3
:10832800E6EE276A85ED287AF0EE667AC5ED2B6AC7
:10833800C5ED2A6A02F05B86A8F806006B4B013F80
:1083480093F80090A5F8B47007990023B9F1070FC6
:108358004B608B60CB607FF46EA905F0AFFD059B89
:10836800DFF8B481C01A94F8E431A8F80000002BB3
:108378003FF466A9013B84F8E43115B0BDEC0C8BE1
:10838800BDE8F08F002B3FF431ABD4F8FC310A9AEA
:10839800D31A574A12689A427FF728AB554B93ED88
:1083A800007AB0EECDDAB4EEC7DAF1EE10FA12D4F4
:1083B800514B99ED007AD3ED006AB0EEC77AB4EE6E
:1083C800E67AF1EE10FA7FF711AB04E094F8F83191
:1083D800002B3FF40BAB002384F8F831FFF706BB02
:1083E800B1F9002094ED6B7AB1F90200D4ED6C6A12
:1083F800424982EAE273A3EBE273F4EEC76A80EAC9
:10840800E072F1EE10FAA2EBE072B8BFF0EE476A44
:108418009342B8BF134607EE103A0B78B8EEC77A06
:1084280027EE287A002B40F0EE82354B93ED006A58
:10843800B4EECA6AF1EE10FA41F13282F7EE005A50
:1084480075EEC65A3BEE477A65EEAA5A2D4BA7EE53
:10845800256A93ED007A26EE076AB5EEC06AF1EE5A
:1084680010FA40F2C486C9EE865AB7EE007AB0EE2A
:10847800476AA6EEE56AF0EE466AF4EEC76AF1EEE0
:1084880010FA88BFF0EE476AF5EEC06AF1EE10FA0E
:10849800B8BFF0EE6B6A1C4B93ED007A67EE877AF3
:1084A800A7EEA68AFFF7BEB9184B194A2B4493EDDD
:1084B800007AD2ED007A174B67EE277AF7EE006A5A
:1084C800F4EEE67AF1EE10FA93ED007A88BFF0EE5A
:1084D800667A67EE877A27EE888AFFF74EBA00BF7A
:1084E800F43700205C490020C4460020A43C00204A
:1084F800BC260020C8260020D02600209C2600206C
:10850800A42600209826002094260020AC220020D3
:108518008C26002088260020A83C0020072B02F08B
:10852800D98300230793CF4ECF4D336806935A055E
:1085380001F11382CD4BCE491F68B1F906807A89C3
:108548009045C0F28F82B8F5FA6F81F27382387A5B
:10855800A8EB020303FB00F3C2F5FA6293FBF2F304
:10856800C3F1640307EE903AF8EEE77A9FEDC17A1B
:1085780067EE877AC4ED417ADFF82093DFF820A30D
:10858800B9F818B0B1F900309AF904209AF8000047
:108598009AF801C0A3EB0B0686EAE67E002AAEEB4A
:1085A800E67E14BF01224FF0FF32BEF5FA7FA8BF66
:1085B8004FF4FA7E704580F20186AEEB000607EEB6
:1085C800906AF8EEE77AAC4E5B45C6ED007A03DABE
:1085D800F1EE677AC6ED007AB1F902E0AEEB0B0373
:1085E800002BB8BF5B42B3F5FA7FA8BF4FF4FA730C
:1085F8009842059380F2B9851B1A07EE903AF8EE77
:10860800E77ADE45C6ED017A03DAF1EE677AC6ED60
:10861800017AB1F90410A1EB0B0383EAE370A0EB34
:10862800E370B0F5FA7FA8BF4FF4FA706045CCBF8D
:10863800A0EB0C0C4FF0000C02FB0CFC07EE90CAF0
:10864800F8EEE77A5945069BC6ED027ABCBFF1EE13
:10865800677AC6ED027A13F48053059300F0898592
:10866800B8F5FA6F4246A8BF4FF4FA62B2F57A7FBE
:1086780094F80831B8BF4FF47A72A2F57A72002BD9
:1086880040F090857D49DFF81CE281FB0230D3176A
:10869800C3EB6013581C6FF0630C3EF910003EF9F1
:1086A80013E00CFB0323A0EB0E0003FB00F381FB9C
:1086B8000321DB17C3EB61139E440FFA8EFE07EE0E
:1086C80090EA059BB8EEE78A86ED038A002B41F015
:1086D80069816B4B1B8813F0400B40F0E086694AB8
:1086E800126812F0140F03D013F4027F41F0A9812D
:1086F800654A12789AB1B9F81A2042450FDB634AE5
:108708001278012A02F09B80192A02F098800E2A1A
:1087180005D0082A03D00022B260C4F8402194F89A
:10872800462112B19B0742F06E8294F84C31002B1F
:1087380041F0BB8099F81E20002A00F09383022A9A
:1087480002F0A080032A01F06E83514A518899F8FB
:108758001F200232D2B2002B02F08680002902F0DC
:1087680083804C480068B1FBF0FA0FFA8AFAA4F843
:108778007CA1AAB307EE90AAF8EEE77AF7EE006AB2
:1087880086EEA77A012AD6ED007AD4ED646A77EEF0
:10879800E67A67EE877AC4ED607A21D0D6ED017A61
:1087A800D4ED656A77EEE67A022A67EE877AC4ED39
:1087B800617A15D0D6ED027AD4ED666A77EEE67A5C
:1087C800032A67EE877AC4ED627A09D0D6ED037A78
:1087D800D4ED676A77EEE67A67EE877AC4ED637A56
:1087E8002D490978092903F0CC82BAF1000F40F32A
:1087F8003F8392B394ED647AD4ED607A77EE877A0A
:10880800012AC4ED647AC6ED007A21D094ED657A28
:10881800D4ED617A77EE877A022AC4ED657AC6EDDF
:10882800017A15D094ED667AD4ED627A77EE877A7C
:10883800032AC4ED667AC6ED027A09D0D4ED677AC8
:1088480094ED637A77EE877AC4ED677AC6ED037A9A
:10885800013A022AB8BF0222D2B2002B18BF022264
:1088680007E300BF6C490020D8460020045D0020C3
:10887800404500200AD7233CCC3C00201F85EB5103
:108888007250002070510020071C00203C38002046
:10889800903F002024380020A43C0020B84E00203F
:1088A800F8370020085D0020099BD84E1B78D907AF
:1088B80000F1DD80327822B19200D549D54820F008
:1088C80077FED54B1B68002B40F0A282D34B1B7858
:1088D8009BB1307870B1DFF83C83DFF87C930027D8
:1088E800F8B2D9F80030B8EC010A98473078013767
:1088F8008742F5DBCA4B1B689847CA4B1B78072B86
:1089080000F07E84012384F8003115B0BDEC0C8B97
:10891800BDE8F08FC44BC7ED00BA1B689342BEF6A2
:10892800BCAF002384F8F831FEF7BFBFBF4EDFF8B5
:108938002C9306F5F47806F51577F6EC017A95EDA3
:10894800080AD5F81432F8EEE77A404627EE800A8E
:108958009847A8F1E000D5F834319847A8F170009D
:10896800D5F8A4319847D6F8F400D5F8B830984728
:1089780008F124084745A9EC010ADED1FEF754BEE8
:10898800099A1278D20703D4A94A128BA4F81C2298
:10899800A84AA949128891ED037A07EE902AF8EEC1
:1089A800E77AB4EEE77AF1EE10FA41F22B81A349A7
:1089B800098807EE901AF8EEE77AB4EEE77AF1EE56
:1089C80010FAC1F2A0809E499E4AD1ED006A92ED4C
:1089D800006A9D49C4ED886ABCEEC75A76EE665AAD
:1089E80015EE102AC4ED866AC4ED855A84ED896AAD
:1089F800A4F81C220122D1ED006A84F8282277EE1F
:108A0800677AFFF74BB8914B93ED005AB5EEC05A11
:108A1800F1EE10FA40F3EB838D4BD3ED004AF5EEFF
:108A2800C04AF1EE10FA40F3E28334EEC77A66EEFC
:108A3800E95A87EE246AC5EE856AB7EE007AB4EE85
:108A4800C76AF1EE10FA88BFB0EE476AB5EEC06AA1
:108A5800F1EE10FA76EE876AB8BFB0EE6B6A66EE92
:108A6800266A0AE54FF07E53C4F8043184E533786A
:108A7800002B3FF426AFD4ED6C3A94ED6B6AD4ED3D
:108A8800867A744A94ED857AD2ED005A94ED694A53
:108A9800D4ED684ADFF8C881DFF878E1F4EEC63A29
:108AA800F3EE046AF1EE10FA37EEA65A01F10C81E2
:108AB80098ED026A26EE446AF0EE674AE6EE074A47
:108AC800F4EEC54A34EEE66AF1EE10FA48BFB0EEAD
:108AD800656A012B8EED006A3FF4F3AE98ED066AE5
:108AE80026EE446AF0EE674AE6EE074AB4EEE45A28
:108AF80034EEE66AF1EE10FA88BFB0EE656A022B32
:108B08008EED016A3FF4DDAE98ED0A6A26EE446AFE
:108B1800F0EE674AE6EE074AF4EEC54A34EEE66A36
:108B2800F1EE10FAB8BFB0EE656A032B8EED026A5B
:108B38003FF4C7AE98ED0E6A26EE446AF0EE674A37
:108B4800E6EE074AB4EEE45A34EEE66AF1EE10FABD
:108B5800C8BFB0EE656A042B8EED036A3FF4B1AE70
:108B680098ED126A26EE446AF0EE674AE6EE074A86
:108B7800F4EEC54A34EEE66AF1EE10FAB8BFB0EE8C
:108B8800656A052B8EED046A3FF49BAE98ED166A74
:108B980026EE446AF0EE674AE6EE074AF4EEC54A66
:108BA80074EEE66AF1EE10FAB8BFF0EE656A062BCD
:108BB800CEED056A3FF485AED8ED1A6A66EEC46A52
:108BC800F0EE674AE6EE874AB3EE046AB4EEE45A7A
:108BD80074EEC66AF1EE10FAC8BFF0EE656A072BAC
:108BE800CEED066A3FF46DAED8ED1E6A26EEC44A95
:108BF800E4EE077AF4EEC57A77EEC67AF1EE10FA6B
:108C080048BFF0EE657ACEED077A5AE6BC440020FC
:108C1800E8260020403600209C250020984E0020A1
:108C28008C4B0020A43C0020B826002008470020D8
:108C3800B84E00209C270020CC3C00209E27002016
:108C480088270020D0370020A4270020982600205D
:108C5800A0260020E4260020844B00206049002044
:108C68000827002007EE103A744BDFF8F0811B78D4
:108C7800C4F8D471B8EEC77AB7EE005A132B85EE54
:108C8800079AB8F90400B4F8D86195ED080A01F01C
:108C9800D4846B4B6B4A93ED001AD3ED053A93EDF0
:108CA800122A93ED173AD3ED091AD3ED0E4A93ED34
:108CB800016A93ED064A93ED0A7AD3ED0F5AD3ED84
:108CC800132AD3ED186A93ED045AD3ED030A67EE1D
:108CD800897A69EE288A29EE088AE1EE273A02EBBA
:108CE80086070021A2EE283AC4F8C811C4F8CC11AE
:108CF800E1EE884AA6EE274AE7EE085A93ED167A7F
:108D080093ED0D6A93ED021AD3ED0C1AC7ED003AF4
:108D1800E2EEA86A25EE635A27EE437A93ED0B2A12
:108D2800D3ED152AC7ED204AA0EEE34A26EE646A81
:108D3800D3ED143A83ED054AA1EE275AF0EE477AAF
:108D4800E1EEE45AA2EE086AE2EEC36AE3EEA87A1C
:108D580083ED065AC3ED0E5A83ED0F6A87ED403A4C
:108D6800C3ED176AC3ED187AC4F8D011731C03F069
:108D78001F03A4F8D831A8F80400FEF737BB0799F9
:108D8800314BD1ED017A93ED007AF0EEE77AF4EE0B
:108D9800C77AF1EE10FA7EF588ADD1ED027AF0EEE1
:108DA800E77AB4EEE77AF1EE10FA7EF77EADD1ED10
:108DB800037AF0EEE77AB4EEE77AF1EE10FA7EF78E
:108DC80074AD224B1B689B077FF5ABAD2049214B47
:108DD800B3F90C20B1F900E01F48AEEB020E0068B1
:108DE8008EEAEE72A2EBEE728242BEF65EADB3F987
:108DF8000E30B1F90220D21A82EAE273A3EBE273D1
:108E080098427EF752AD8CE5B0EE465AFEF77FBE2B
:108E180008F048FA5AE596ED007A05EB4702B8EEF5
:108E2800C78A928F2AF8172028EE278AFEF7CABB2E
:108E380020F032FD2AF81700FEF7E6BBA43C00201C
:108E4800003200207C2F0020C42600207051002012
:108E5800883F002000380020C0260020A83C0020C1
:108E68000AD7233CA4F87C219246002B00F06581A8
:108E780002223B785FED066AB97807EE903AF8EE81
:108E8800E77AB0EE007A67EEA67AE14BF4EEC77A9D
:108E9800F1EE10FA187840F3E48337EEC77ADFED85
:108EA800DD6AB0EE676AA7EE266AB0EE467A9FEDF5
:108EB800DA6AD6ED006A66EE866AB0EEE66AC4ED56
:108EC800686A84ED6B6A99B105EE901AB8EEE55AB6
:108ED800DFEDD25A66EEA64A25EE255AF7EE005A7D
:108EE80075EEC55A64EE864AE4EE855A66EEA56AC2
:108EF800DFEDCB5A7B7927EE257A27EE267ACBB1A0
:108F0800DFEDC66ADFEDC75A26EE266A06EE903A0E
:108F1800F8EEE66A26EE266AB4EEE56AF1EE10FA95
:108F280000F3A586F7EE005A35EEC66AC5EE866AE6
:108F380027EE267A0C289FEDBC8ADFEDBC6A00F08C
:108F48001786B4EEC87AF1EE10FA98BFB0EE478AE9
:108F5800B4EEE68AF1EE10FAB8BFB0EE668A84ED98
:108F68004E8A002A00F0DE80B0EE007AF4EEC77A6E
:108F7800F1EE10FA05DD37EEC77ADFEDA66AE7EE07
:108F8800267A96ED017ADFEDA46A27EE267AB0EE0E
:108F9800C76A84ED697A84ED6C6A99B106EE901A15
:108FA800DFED9E5AF8EEE66A27EE075A66EEA56AE6
:108FB800F7EE005A75EEE65A25EE065AE5EE265A01
:108FC80027EE257ADFED966ABB7967EEA67A67EE1B
:108FD800877AABB107EE103AB8EEC77ADFED8F5A51
:108FE800DFED906A27EE067A27EE257AB4EEE67A68
:108FF800F1EE10FA40F32D86DFED8D6A67EEA67A62
:109008000C2800F0D285DFED886A9FED887AF4EEAF
:10901800E67AF1EE10FA88BFF0EE667AF4EEC77AD7
:10902800F1EE10FAB8BFF0EE477A012AC4ED4F7A94
:1090380078DD7B78DFED796A07EE903AF8EEE77A2B
:10904800B0EE007A67EEA67A7B7AF4EEC77AF1EE94
:1090580010FA05DD37EEC77ADFED6E6AE7EE267A9D
:1090680096ED027ADFED6C6A27EE267AB0EEC76AD3
:1090780084ED6A7A84ED6D6A9BB106EE903ADFED75
:10908800675AF8EEE66A27EE075A66EEA56AF7EE23
:10909800005A75EEE65A25EE065AE6EE855A27EE90
:1090A800257ADFED5F6AFB7967EEA67A67EE877A45
:1090B8000BB307EE103AB8EEC77ADFED585ADFED7A
:1090C800596A27EE067A27EE257AB4EEE67AF1EEAB
:1090D80010FA0CDCB5EEC07AF1EE10FA01F1BA83A1
:1090E800B7EE006A36EE477AC6EE076A01E0DFEDB2
:1090F800506A67EEA67A0C2800F03085DFED4A6AE0
:109108009FED4A7AF4EEE67AF1EE10FA88BFF0EEB7
:10911800667AF4EEC77AF1EE10FAB8BFF0EE477A45
:10912800C4ED507A092800F00D8599F82160002EC9
:1091380040F0A484002384F84C313E4B1B7823B9BB
:109148003D4EB378002B41F0F083314B1B78072B51
:1091580000F04C850022072B84F800217EF4F3A848
:1091680004F0ACFE0590FEF7F0B8DFED347AFFF7B7
:1091780048BAB9F81A209045C0F25984B8F5FA6F80
:10918800D4BFC2EB0803C2F5FA634FF47A7101FB4E
:1091980003F194F80801C2F5FA63B1FBF3F2002871
:1091A8003FF470AA94F80931254902FB03F281FBC8
:1091B8000213D217C2EB6312FFF764BADFED1F7A0E
:1091C800FFF701BA1F4B204C1A68204BDFF8848048
:1091D80094F80001D2691B88A8F80020A8F802308A
:1091E80000287FF49EA90590194DFEF7AEB8DFED73
:1091F800136AFFF750B943023EF58FAEFEF791BEF2
:1092080004F05CFE134B401BD880FFF77BBB00BF0C
:10921800A43C0020D7A368416F12033B0AD7233C24
:1092280000004843A4707D3F00C0F94400C0F9C461
:109238000000C842F13E0020703400200000000009
:109248001F85EB511C530020002100208828002096
:10925800D8460020A83C002004F030FED64B0B9ADC
:109268001B78DFF89083801A012BA8F8020000F021
:10927800CD83072B7EF4E1AB04F020FE0546FEF714
:10928800DDBBDFF87483BCF1000F41F03A8598ED3F
:10929800007A9DED0C5ADFF864E325EE877AA5EE97
:1092A800267AB0EE675AA7EE065ABDEEC57A17EED3
:1092B800107A17EE100A9F42A8BF1846B942C8BFD5
:1092C800084607EE100AB8EEC77A012A8EED007A32
:1092D8003FF4F2AA98ED047A9DED0D5A25EE877AAF
:1092E800A5EE267AB0EE675AA7EE065ABDEEC57A05
:1092F80017EE107A17EE100A9F42A8BF1846B94217
:10930800C8BF084607EE100AB8EEC77A022A8EEDE3
:10931800017A3FF4D1AA98ED087A9DED0E5A25EE10
:10932800877AA5EE267AB0EE675AA7EE065ABDEE02
:10933800C57A17EE107A17EE100A9F42A8BF184692
:10934800B942C8BF084607EE100AB8EEC77A032A22
:109358008EED027A3FF4B0AA98ED0C7A9DED0F5A83
:1093680025EE877AA5EE267AB0EE675AA7EE065A5A
:10937800BDEEC57A17EE107A17EE100A9F42A8BF05
:109388001846B942C8BF084607EE100AB8EEC77AB1
:10939800042A8EED037A3FF48FAA98ED107A9DED9A
:1093A800105A25EE877AA5EE267AB0EE675AA7EE10
:1093B800065ABDEEC57A17EE107A17EE100A9F42CC
:1093C800A8BF1846B942C8BF084607EE100AB8EE4B
:1093D800C77A052A8EED047A3FF46EAA98ED147ABE
:1093E8009DED115A25EE877AA5EE267AB0EE675ADA
:1093F800A7EE065ABDEEC57A17EE107A17EE100AD8
:109408009F42A8BF1846B942C8BF084607EE100ACF
:10941800B8EEC77A062A8EED057A3FF44DAA98ED84
:10942800187A9DED125A25EE877AA5EE267AB0EEC7
:10943800675AA7EE065ABDEEC57A17EE107A17EEF0
:10944800100A9F42A8BF1846B942C8BF084607EE8F
:10945800100AB8EEC77A072A8EED067A3FF42CAACE
:1094680098ED1C7A9DED135A65EE875AE6EE855AFB
:10947800E6EE257AFDEEE77A17EE900A8342A8BF5A
:1094880003468142C8BF0B4607EE903AF8EEE77AEA
:10949800CEED077A002A7FF40FAAFFF712BA474ADF
:1094A8004748B2F90420B4F81011DFED466A9FED81
:1094B800467A80FB02E0D217C2EBA002521A12B21F
:1094C80007EE902AF8EEE77A67EEA67A77EE876AD3
:1094D800BDEEE66A16EE102A2032402A41F2DD81FE
:1094E800DFED3A6ABDEEE77A17EE102A2032402AFD
:1094F80001F2CF819FED367AF4EEC77AF1EE10FAD9
:1095080042F36883DFED335A9FED336A01E0F0EEF2
:10951800477AF4EEC67AF1EE10FA37EEE57AF6DC21
:10952800DFED2E7AB4EEE77AF1EE10FA42F14E83CF
:10953800DFED285A9FED2A6A01E0B0EE677AB4EEB3
:10954800C67AF1EE10FA77EE257AF6D49FED1E7AF8
:10955800F4EEC77AF1EE10FA00F38C859FED217ACC
:10956800F4EEC77AF1EE10FA44BF9FED1C7A77EE5D
:10957800677A67EEA75A9FED1C5A9FED1C6A9FED0C
:109588001C7AA5EE856A27EEA55AA5EE867AE5EE41
:10959800077A96ED016AD6ED005A27EEC67A65EE8F
:1095A800A77AA5EEA67AE6EE267A86ED007AC6EDCB
:1095B800017AFFF794B800BFA43C0020883F002040
:1095C8006766666635FA8E3CDB0FC93F000000000F
:1095D800DB0F4940DB0FC940E4CB1641DB0F49C024
:1095E800E4CB16C1DB0FC9BF92E741B99730083CFD
:1095F80015A82ABEA83C00200827002040360020D5
:10960800DC4B5A79002A3EF40BABDB4A1278002A6D
:109618003EF406AB1B78DFEDD94A07EE903AD84BFB
:10962800B8EE677A1B8807EE902A06EE903AF8EEB5
:10963800E77AF8EE666A67EE277AB7EE007AC7EE41
:10964800A63AF4EEE43AF1EE10FA88BFF0EE643A86
:10965800F4EEC73AF1EE10FAB8BFF0EE473AFEF76B
:10966800E1BAB0EE677A22E4B8F1000F00F0E583C2
:10967800DFF82883BCF1000F41F0FA87BAF1000F38
:1096880041F0508698ED005ADDED0C4ADFF810E302
:1096980025EE855ABDEEC77A17EE101AB0EE457A58
:1096A800A4EEA67AB0EE675AA7EE065ABDEEC57AC2
:1096B80017EE107A17EE100A9F42A8BF1846B94253
:1096C800C8BF084607EE100AB8EEC77A012A8EED21
:1096D800007A3FF4F1A898ED047A9DED0D5A25EE35
:1096E800877AA5EE267AB0EE675AA7EE065ABDEE3F
:1096F800C57A17EE107A17EE100A9F42A8BF1846CF
:109708008F42B8BF084607EE100AB8EEC77A022A99
:109718008EED017A3FF4D0A898ED087A9DED0E5AA7
:1097280025EE877AA5EE267AB0EE675AA7EE065A96
:10973800BDEEC57A17EE107A17EE100A9F42A8BF41
:1097480018468F42B8BF084607EE100AB8EEC77A27
:10975800032A8EED027A3FF4AFA898ED0C7A9DEDBE
:109768000F5A25EE877AA5EE267AB0EE675AA7EE4D
:10977800065ABDEEC57A17EE107A17EE100A9F4208
:10978800A8BF18468F42B8BF084607EE100AB8EEC1
:10979800C77A042A8EED037A3FF48EA898ED107AE2
:1097A8009DED105A25EE877AA5EE267AB0EE675A17
:1097B800A7EE065ABDEEC57A17EE107A17EE100A14
:1097C8009F42A8BF18468F42B8BF084607EE100A46
:1097D800B8EEC77A052A8EED047A3FF46DA898EDA5
:1097E800147A9DED115A25EE877AA5EE267AB0EE09
:1097F800675AA7EE065ABDEEC57A17EE107A17EE2D
:10980800100A9F42A8BF18468F42B8BF084607EE05
:10981800100AB8EEC77A062A8EED057A3FF44CA8EE
:1098280098ED187A9DED125A25EE877AA5EE267ADC
:10983800B0EE675AA7EE065ABDEEC57A17EE107A53
:1098480017EE100A9F42A8BF18468F42B8BF0846B5
:1098580007EE100AB8EEC77A072A8EED067A3FF4AB
:109868002BA898ED1C7A9DED135A65EE875AE6EE03
:10987800855AE6EE257AFDEEE77A17EE900A8342DE
:10988800A8BF03468142D8BF194607EE901AF8EEE2
:10989800E77ACEED077A002A7FF40EA8FFF711B811
:1098A800384B93ED006AFEF7D8BD374A3749D2F8EE
:1098B800EC20096844F620608242A8BF0246B2F54F
:1098C8007A7FB8BF4FF47A7292B2C806A4F84E21D4
:1098D80041F120830599002940F0C4832C49D1F82F
:1098E80000C0BCF932E02B48D4F85011A0FB0202AA
:1098F8009009642292FBF0F2142AFDEEC87A04EB78
:109908004108A8BF142201318A42C4F8501117EE49
:10991800900ADCBF0021C4F8501104EB4101A8F8FB
:109928005401B1F9542107EE902AF8EEE77A38EE9F
:10993800678AFDEEC87ACDED057ABDF9141081EA83
:10994800E172A2EBE172724502F32981124A1146D3
:109958004FF07E520A60FEF7EDBEAB68002B3EF476
:10996800E9AD05F150012846984733680693FEF79C
:10997800E1BD00BF78510020CA3C0020713DAA3FDC
:10998800B43C00209826002068100020C83700202A
:10999800183F0020D34D62107800002008270020CF
:1099A800403600201D21B448FAF73DFE00283EF459
:1099B80090AEB24BDB78002B7EF48BAEDFEDB07A45
:1099C800B04938EE678ACBF5FA62FDEEC87A12B272
:1099D800CDED087ABDF920301B0381FB0301DB17AD
:1099E800C3EBA11302FB03F343F30F335B4407EE0E
:1099F800903AB8EEE78A86ED038AFEF76ABE04F06D
:109A08005DFA0B90FDF72BBEDFF8B88204F056FA2A
:109A18009D4AD4F80C321268C4F80C02C31A9A1A78
:109A28000546A8F80430A8F80620FEF707B8194636
:109A3800FFF7AFBB3B7AC3F1640307EE903AFEF73A
:109A480093BD924A127812F0100201F03A8494F809
:109A58001411D4F8182196ED017A00290CBF0121C0
:109A68004FF0FF3102FB01F207EE902AF8EEE77A99
:109A780077EE877AC6ED017AFEF73ABE1E217E4858
:109A8800FAF7D1FD00283FF455ABBBF1000F7FF486
:109A980051AB94F8B831B34242F0F8807C4BD4ED26
:109AA8006F7A93ED010AD4ED505A9FED7A6ADFED93
:109AB8007A6A27EEE57A67EE887AA0EE087AE5EE0C
:109AC800807AB4EEC67AF1EE10FA88BFB0EE467A24
:109AD800B4EEE67AF1EE10FAF4EEC67AB8BFB0EE5C
:109AE800667AF1EE10FA88BFF0EE467AF4EEE67A7E
:109AF800F1EE10FAB8BFF0EE667A84ED4E7AC4ED56
:109B0800507AFFF717BBB4F81C12914240F27685E1
:109B18006249634AD1ED007A92ED007A6149C4ED59
:109B2800887A77EE676AC4ED867A0122C4ED856A81
:109B380084ED897AD1ED006ADFED5B7A84F828221A
:109B4800FDF7ACBFFDEEC87ADFF8788117EE903AE2
:109B5800A8F804A0A8F80630FFF7E7BABDEEE77A40
:109B6800DFF8608117EE103AA8F80430FFF7C6BA9C
:109B7800B4EEC87AF1EE10FA98BFB0EE478ABDEE9F
:109B8800C77AB4EEE68ADFF83C81F1EE10FA17EEF8
:109B9800103AB8BFB0EE668A84ED4E8AA8F8003055
:109BA800002A7FF4E1A9FFF7C0BA9FED3A7ADFED0A
:109BB8003A6ADFF81081F4EEC77AF1EE10FA98BF2E
:109BC800B0EE677AFDEEE77AB4EEE67AF1EE10FAD7
:109BD80017EE903AB8BFB0EE667A012A84ED4F7A54
:109BE800A8F802303FF725AAFFF79FBA04F066F9F4
:109BF800079ADFF8D0802D4B801A1B78A8F804004C
:109C0800FFF7A8BA2A4A2B49D2ED006A2A4A91EDF1
:109C1800006A1278C4ED886A84ED896A002A40F0E7
:109C2800D48476EEC65AF0EE466ABCEEC76A23497B
:109C3800C4ED855A16EE102AC4ED866AA4F81C22D3
:109C4800FF22D1ED006A84F8282277EEC77AFDF763
:109C580025BFB5EEC07AF1EE10FA00F1F785B7EE40
:109C6800006A36EE477AC6EE076AFFF7C7B9DFED36
:109C7800146AFFF75DB900BFC8370020BC3E00205A
:109C880000007A44D34D621024380020C4320020EA
:109C98007800002000C0F94400C0F9C488270020DB
:109CA800D0370020A427002000000000A43C00209A
:109CB800683600208C270020904B0020A027002029
:109CC8000000C842A83C002098ED016A26EE646AAC
:109CD800B0EE674AA6EE074AB4EEC45A34EE666A96
:109CE800F1EE10FAC8BFB0EE656A012B8EED006A7E
:109CF8003EF4E7AD98ED056A26EE646AB0EE674A71
:109D0800A6EE074AB4EEC45A34EE666AF1EE10FACB
:109D1800C8BFB0EE656A022B8EED016A3EF4D1AD84
:109D280098ED096A26EE646AB0EE674AA6EE074A1D
:109D3800B4EEC45A34EE666AF1EE10FAC8BFB0EE5B
:109D4800656A032B8EED026A3EF4BBAD98ED0D6A91
:109D580026EE646AB0EE674AA6EE074AB4EEC45A25
:109D680034EE666AF1EE10FAC8BFB0EE656A042BED
:109D78008EED036A3EF4A5AD98ED116A26EE646A8D
:109D8800B0EE674AA6EE074AB4EEC45A34EE666AE5
:109D9800F1EE10FAC8BFB0EE656A052B8EED046AC5
:109DA8003EF48FAD98ED156A26EE646AB0EE674A08
:109DB800A6EE074AB4EEC45A74EE666AF1EE10FADB
:109DC800C8BFF0EE656A062BCEED056A3EF479ADA4
:109DD800D8ED196A66EEE46AB0EE674AA6EE874ADD
:109DE800B3EE046AB4EEC45A74EE466AF1EE10FAA1
:109DF800C8BFF0EE656A072BCEED066A3EF461AD8A
:109E0800D8ED1D6A66EEE44AE4EE877AF4EEC57A88
:109E180077EEC67AF1EE10FAB8BFF0EE657ACEEDBD
:109E2800077AFEF74EBD99F82020C2EB421102EBEB
:109E38008102D20091B2FEF78ABCDFF8A885BAF198
:109E4800000F41F0EB8098ED005ADDED0C4ADFF889
:109E580098E525EE855ABDEEC77A17EE101AB0EED2
:109E6800457AA4EEA67AB0EE675AA7EE065ABDEE7A
:109E7800C57A17EE107A17EE100A9F42A8BF184647
:109E8800B942C8BF084607EE100AB8EEC77A012AD9
:109E98008EED007A3EF498A998ED047A9DED0D5A5E
:109EA80025EE877AA5EE267AB0EE675AA7EE065A0F
:109EB800BDEEC57A17EE107A17EE100A9F42A8BFBA
:109EC80018468F42B8BF084607EE100AB8EEC77AA0
:109ED800022A8EED017A3EF477A998ED087A9DED75
:109EE8000E5A25EE877AA5EE267AB0EE675AA7EEC7
:109EF800065ABDEEC57A17EE107A17EE100A9F4281
:109F0800A8BF18468F42B8BF084607EE100AB8EE39
:109F1800C77A032A8EED027A3EF456A998ED0C7A98
:109F28009DED0F5A25EE877AA5EE267AB0EE675A90
:109F3800A7EE065ABDEEC57A17EE107A17EE100A8C
:109F48009F42A8BF18468F42B8BF084607EE100ABE
:109F5800B8EEC77A042A8EED037A3EF435A998ED57
:109F6800107A9DED105A25EE877AA5EE267AB0EE86
:109F7800675AA7EE065ABDEEC57A17EE107A17EEA5
:109F8800100A9F42A8BF18468F42B8BF084607EE7E
:109F9800100AB8EEC77A052A8EED047A3EF414A9A1
:109FA80098ED147A9DED115A25EE877AA5EE267A5A
:109FB800B0EE675AA7EE065ABDEEC57A17EE107ACC
:109FC80017EE100A9F42A8BF18468F42B8BF08462E
:109FD80007EE100AB8EEC77A062A8EED057A3EF427
:109FE800F3A898ED187A9DED125A25EE877AA5EE1A
:109FF800267AB0EE675AA7EE065ABDEEC57A17EE76
:10A00800107A17EE100A9F42A8BF18468F42B8BFB1
:10A01800084607EE100AB8EEC77A072A8EED067AC8
:10A028003EF4D2A898ED1C7A9DED135A65EE875A36
:10A03800E6EE855AE6EE257AFDEEE77A17EE900A07
:10A048008342A8BF03468142D8BF194607EE901A3B
:10A05800F8EEE77ACEED077ABCF1000F7EF431AC6A
:10A06800FEF7B6B8DA49D1F800C0BCF832E04FEADA
:10A078005E0E38E49FEDD77A77EE677AFFF779BA04
:10A08800DFF86893D4ED017A94ED006AB9F800001E
:10A09800D9F8143077EEA77AF0EE006AB0EE677A56
:10A0A800A6EE267A013804EBC002D6EE267A083AE4
:10A0B8001033F6EE003A27EE237A67EEA37A84EDA2
:10A0C800207AC4ED217AC44CA64604F1800192EDB1
:10A0D800027A92ED036ADEED036ADEED027A53ED51
:10A0E800014A13ED025A37EE674A76EEC65A77EE02
:10A0F800277AE4EE845A0138A2F10802E5EE047AE0
:10A108000EF1080E03F1080336EE267A01F1080174
:10A11800E4EE877AE5EE475A67EEA37A25EEA37A4E
:10A12800C1ED007A81ED017AD1D1142F7DF419AAFD
:10A1380003F0C4FE069BDFF8B882C01AA8F8020034
:10A14800D4F8DC61FDF70DBADFF8A89299F8002081
:10A15800900802F00D80DFF8A0C200F101084FEA74
:10A1680048180CEB080E0CF12003ACF1700113ED4C
:10A17800076A53ED056A13ED037A53ED017A53ED3F
:10A18800025A13ED084A53ED064A13ED045A26EE17
:10A19800066A66EEA66A27EE077A67EEA77AA4EE45
:10A1A800046A20339E45E4EEA46A01F11001A5EE8D
:10A1B800057AE5EEA57AF1EEC65AB1EEE66AF1EE59
:10A1C800C76AB1EEE77A41ED085A01ED076A41ED39
:10A1D800066A01ED057ACAD1A8F12008C44404EB47
:10A1E800001012F0030318BF0CF1080C0FD05CED3F
:10A1F800017A1CED027A67EEA77A013BE7EE077A4F
:10A208000CF1080CB1EEE77AA0EC017AEFD1142F2B
:10A2180001F0F1850136C4F8DC61FDF70BB9DFF810
:10A22800CC916D48D9F80820B9F80C101EF0C8F97F
:10A238006A4B1F78142F01F04487D4F8DC6101368B
:10A24800C4F8DC611EE7DFF8A491B9F800E0D9F89A
:10A2580004C04FEA5E084FEA880204EB8E065FEA04
:10A26800DE0E04EB020300F0A08010320EF1010EA6
:10A278005B4803EB0E1E324410330CF1100706F155
:10A28800100151ED032A51ED043A10ED043A10ED96
:10A29800032A51ED026A11ED016A10ED020A10ED70
:10A2A800018A12ED044A12ED035A53ED044A53EDA4
:10A2B800035A13ED027A53ED017A52ED020A12EDB8
:10A2C800011A73EE238A72EE221A40ED048A40EDD9
:10A2D800031A70EE268A78EE061A40ED028A40EDDF
:10A2E800011A74EE848A75EE851A43ED048A43EDEB
:10A2F800031A77EE208A77EE811A43ED028A43ED3E
:10A30800011A73EE633A75EE655A17ED035A32EE89
:10A31800623A74EE644A65EE631A17ED044A23EE56
:10A32800052A64EE652AE3EE041A10339E4524EEEE
:10A33800843AA3EE842A00F1100007F11007A5EE75
:10A34800853A01F1100102F11002E4EE852A41ED8F
:10A35800071A01ED082A02ED073A42ED082A57EDDF
:10A36800055A17ED065A70EE666A38EE466A30EE00
:10A37800C77A71EE677A26EE253A65EEE63A25EE5B
:10A38800674A67EE054AE6EE053AA6EE853AA7EE75
:10A39800254AE7EEA54A01ED063A41ED053A02EDF8
:10A3A800064A42ED054A7FF46CAF1FFA88F8624608
:10A3B800414609481BF028FC4146D9F8042030469C
:10A3C8001BF022FC054B1B78142B7FF4B9AEAFE6CB
:10A3D800183F0020DB0F494000210020A43C00204A
:10A3E800102100200827002040360020642F00207C
:10A3F800A83C00205E2F002080210020D4F8E081B6
:10A40800B4F8D8A1C74BCAF120095FFA89F90AEB59
:10A41800481E03EB8E0E5FEA990301F013840133A3
:10A428001801C149C14A0EEB000C0EF1100313EDDF
:10A43800024A13ED035A13ED016A13ED047A51ED44
:10A44800024A51ED035A51ED016A51ED047A64EE66
:10A45800244A65EE255A66EE266A67EE277A103397
:10A468009C4542ED024A42ED035A42ED016A42ED33
:10A47800047A01F1100102F11002D8D1AC49A0F11F
:10A488001002964401EB020C224419F0030309D090
:10A49800BEEC017AFCEC017A67EE277A013BE2EC2C
:10A4A800017AF5D1BAF1000F41F07B80142F7DF4C9
:10A4B80058A803F003FD069BDFF8A882D4F8DC61F6
:10A4C800C01AA8F80200FDF74CB8D4F8E091994AF0
:10A4D800994BDFED9A7AD3ED008A994B4FEAC9017F
:10A4E8000A44F8EE688A928809EE102A643AC82A63
:10A4F800A8BFC82268EEA78AF8EE497A782AB8BFBA
:10A50800782268EEA78A07EE902A4944B0EE680AD6
:10A5180003EB8108B8EEE78A1FF00AFAB8EEC99A89
:10A52800F0EE409AB0EE680A1FF064F938EE097A46
:10A5380079EE487A28EE098A67EE877AB7EE006ADC
:10A5480088EE277A142FF8EE007A77EE076A60EE25
:10A55800277A89EEA67A77EE065A36EE477AC6EE5D
:10A56800256A67EEA67A27EE267AC8ED006A88ED96
:10A57800047AC8ED026AC8ED017AC8ED037A01F0E1
:10A588002C84704B704A09F1010983FB0938A8EB48
:10A59800E97808EB48080136A9EB08081778C4F8E9
:10A5A800DC61C4F8E0812BE703F088FC664B069079
:10A5B8001F78142F05BFDFF8AC81D4F8DC61D4F81C
:10A5C800DC61A8F80060FCF71ABF76EE665AFFF760
:10A5D8002CBB5E4A99ED007AD2ED006AB0EEC77ADC
:10A5E800B4EEE67AF1EE10FA7DF500AA01220A9996
:10A5F800C4F8FC1184F8F821FDF7CBBE544A55493C
:10A60800D2ED007A544A91ED007A1278C4ED887A36
:10A6180084ED897A002A01F0BC8277EE676A4F4997
:10A62800C4ED867AC4ED856AFF22D1ED006ADFEDBC
:10A638004E7A84F82822FDF731BA494FDFF8E490C2
:10A64800D7ED005A97ED055A97ED016A97ED064A3E
:10A65800D7ED044AD7ED036A97ED027A67EE897A57
:10A6680009EB8603A5EEA75AA6EE274A64EEC54A6B
:10A67800A6EEC54AE7EE274A20EE050A87ED054A09
:10A68800C7ED064A29EE088A69EE288A83ED005A42
:10A698001FF002F9D7ED0E5AD7ED176A97ED091A90
:10A6A800D7ED121A97ED0F5A97ED187A97ED0A2AF7
:10A6B800D7ED132A97ED0D6AD7ED167A97ED0C3A78
:10A6C800D7ED0B3A97ED154AD7ED144AE1EE085A43
:10A6D800002109EB8602E8EEA16A00B2C4F8C811AD
:10A6E800A2EE085AC4F8CC11C4F8D011A8EEA27A88
:10A6F80026EE656A67EEE67AA3EE655AA3EE886AE7
:10A70800A6EEC47AE8EEA47A87ED0E5AC2ED205A76
:10A7180087ED0F6AC2ED406A87ED177AC7ED187AA0
:10A72800FEF724BB7C2F00200C31002010210020D4
:10A73800FC3000207C3100205C49002027D4D23630
:10A74800F048002056555555A43C0020D02600203E
:10A75800683600208C270020904B0020A02700207E
:10A7680000320020A83C002000000000B5F93C3071
:10A778006A6207EE903A0122F8EEE77AEB66C5F8CE
:10A7880088200023012FC5ED1F7AC5ED1E7AC5F874
:10A79800803001F02782B7427DF46EADB5F93E30C6
:10A7A8002B6707EE903A00220123F8EEE77AAA62B7
:10A7B800C5F89C300023012FC5ED247AC5ED237A16
:10A7C800C5F8943001F00A82B7427DF485ADB5F939
:10A7D80040306B6707EE903A00220123F8EEE77AE3
:10A7E800EA62C5F8B0300023012FC5ED297AC5ED1E
:10A7F800287AC5F8A8307DF49FAD1FED258AB9F1F8
:10A80800030F2BD0BAF1000F09D007EE90AAF8EE8B
:10A81800E77AF4EEC87AF1EE10FA01F1AE84C04A94
:10A828006B6F1268A8F80600002103EB560393FB30
:10A83800F6F6EE6291621163D162FDF77FBDB94A07
:10A84800927B002A3DF467AFFDF769BFF7EE006A17
:10A85800FEF7D4BBF7EE006AFEF74BBCB0EE480A31
:10A868001FF01AF800B2CDE7B4F87CA10AF1FF3A5C
:10A878000FFA8AFABAF1000FA4F87CA13DF7B9AF34
:10A88800FEF7F3BAB4F84E2102F57A7291B2FDF7E9
:10A898005EBFDFEDA57AFEF77CBEF4EEC77AF1EE77
:10A8A80010FA41F3B882DFEDA15A9FEDA16A01E0E9
:10A8B800F0EE476AF4EEC66AF1EE10FA36EEE57A83
:10A8C800F6DCDFED9C6AB4EEE67AF1EE10FA41F1BF
:10A8D8008082DFED965A9FED986A01E0B0EE667AC5
:10A8E800B4EEC67AF1EE10FA77EE256AF6D49FED4B
:10A8F800937AF4EEC76AF1EE10FA40F3CE849FED36
:10A90800907A77EE666A66EEA65A9FED8E5A9FEDAC
:10A918008E6A9FED8E7AA5EE856A26EEA55AA5EE7B
:10A92800867AE5EE076AFEF7DDBD894F3A78013A87
:10A938000A2A1CD8DFE812F0B0005C012201D90015
:10A948001B001B009B008A00660051000B00814A17
:10A95800814952680968C8328A4203D31DF0E8F871
:10A9680028B1B378032B01F0C88401233B70F37836
:10A97800002B3EF4EAAB794B1B78D80740F1958061
:10A98800DFF8D481D4F8C421D8F800309A4200F214
:10A9980098803B78012B3EF4D8AB94F8C021002A6C
:10A9A8003EF4D3AB0B2B0DD801229A4040F603019D
:10A9B80012EA01060CD112F4C06F03D0093B012B37
:10A9C80041F2C185634BD8F800205A600B233B70D5
:10A9D800002384F8C031FEF7B8BB614B1B78002B0D
:10A9E80001F07B831A201CF0EBFB002841F07583F3
:10A9F80094F8C031002B41F0708309233B700DF0AF
:10AA080091FBB4E71A201CF0DBFB0028F7D0554B6C
:10AA18001B88002BF3D1544B4520D3F800801DF040
:10AA2800A9F80E201DF0A6F840461DF049F9DDF8FA
:10AA3800288040461DF044F94C4A4D4B12681A6074
:10AA480040460A233B700DF0A5F8D8E71DF052F8F0
:10AA58000DF0A2FB00288AD01DF06AF8002886D0E5
:10AA6800424A434B12681A600A233B707FE71DF085
:10AA780041F8404B002105208DE80300A3F10802AE
:10AA8800029153200EF084F800287FF470AF314A09
:10AA9800082310603B706AE7304B1B78DB0701F135
:10AAA800D383F378002B3EF450AB08F013F9002859
:10AAB8003FF466AF284B1B6803F59C530833C4F872
:10AAC800C4313B78012B7EF440AB94F8C031002BA5
:10AAD8007EF43BABB378032B01F0E7840EF022F948
:10AAE800012384F8C031FEF730BB1DF003F8224A79
:10AAF8000292A2F10C03262101930091A2F10A030C
:10AB08005021163A49200EF043F800287FF42FAF61
:10AB1800104B4FF0FF310722186059603A7026E752
:10AB28001C5300206857002000000000DB0FC940BC
:10AB3800E4CB1641DB0F49C0E4CB16C1DB0FC93F9C
:10AB4800DB0F494092E741B99730083C15A82ABE67
:10AB58006D340020D4370020B0560020FE56002067
:10AB680090380020945D0020905D0020A45D0020B6
:10AB78009C5D0020B8BE0208FEBC0208DFF8A48372
:10AB88001CF0B8FFE64AD8F80430126864339342E0
:10AB9800BFF4EDAE40201CF093FF00287FF4E7AE31
:10ABA800D8F80030DFF89CA3DFF87CB34FF04009F9
:10ABB8000FE01CF0DFFFDBF80020D8F80030013A86
:10ABC8000133B9F10109CBF80020C8F8003001F0D1
:10ABD80010841AF803301846002BEAD100234FF0EE
:10ABE800FF32C8F800300423C8F804203B70BEE6E2
:10ABF800CB4BCC4A1B685360CB490023136003221C
:10AC08000B603A70B3E6C94BDFEDC97A93ED080AD9
:10AC18000892B4EEE70AF1EE10FA40F218851EF039
:10AC2800D1FED4ED527A20EE270A1EF035FEB0F59B
:10AC3800617F089A00F3518607EE900AF8EEE76AFA
:10AC4800DFEDBC7A66EEA76A07EE902AB8EEE77ADF
:10AC5800FDEEE67A17EE903A2033402B41F242821D
:10AC68009FEDB50A1EF018FE00B207EE900AF8EE46
:10AC7800E77A38EE278A86ED038AFDF756BD099BE9
:10AC880093F800C00CF0010CBCF1000F7DF419AE74
:10AC9800FDF79EBAA94BDFEDAA7A1F68C4ED7A7A50
:10ACA80017F0805740F0328310F4800700F0AC8131
:10ACB8000027B6EE007A67EE877AF4EEE75AF1EEEF
:10ACC80010FA48BFF0EE675A40F12083C4ED8B5A62
:10ACD800FDF727B903F0F2F80790FDF724BC74EEEE
:10ACE800677AB7EE007AF4EEC77AF1EE10FAC4ED9F
:10ACF8007A7A40F3638784EEA77A8DED0C7AFDF7B4
:10AD080006B9BEF1000F00F02E8698ED007A9DED91
:10AD18000C5ADFF834E225EE877AA5EE267AB0EEF3
:10AD2800675AA7EE065ABDEEC57A17EE107A17EEE7
:10AD3800100A9F42A8BF1846B942C8BF084607EE86
:10AD4800100AB8EEC77A012A8EED007A3DF4B9AD43
:10AD580098ED047A9DED0D5A25EE877AA5EE267AB0
:10AD6800B0EE675AA7EE065ABDEEC57A17EE107A0E
:10AD780017EE100A9F42A8BF1846B942C8BF084636
:10AD880007EE100AB8EEC77A022A8EED017A3DF472
:10AD980098AD98ED087A9DED0E5A25EE877AA5EEC6
:10ADA800267AB0EE675AA7EE065ABDEEC57A17EEB8
:10ADB800107A17EE100A9F42A8BF1846B942C8BFBA
:10ADC800084607EE100AB8EEC77A032A8EED027A13
:10ADD8003DF477AD98ED0C7A9DED0F5A25EE877A04
:10ADE800A5EE267AB0EE675AA7EE065ABDEEC57AEA
:10ADF80017EE107A17EE100A9F42A8BF1846B942FC
:10AE0800C8BF084607EE100AB8EEC77A042A8EEDC6
:10AE1800037A3DF456AD98ED107A9DED105A25EE63
:10AE2800877AA5EE267AB0EE675AA7EE065ABDEEE7
:10AE3800C57A17EE107A17EE100A9F42A8BF184677
:10AE4800B942C8BF084607EE100AB8EEC77A052A05
:10AE58008EED047A3DF435AD98ED147A9DED115AD6
:10AE680025EE877AA5EE267AB0EE675AA7EE065A3F
:10AE7800BDEEC57A17EE107A17EE100A9F42A8BFEA
:10AE88001846B942C8BF084607EE100AB8EEC77A96
:10AE9800062A8EED057A3DF414AD98ED187A9DEDED
:10AEA800125A25EE877AA5EE267AB0EE675AA7EEF3
:10AEB800065ABDEEC57A17EE107A17EE100A9F42B1
:10AEC800A8BF1846B942C8BF084607EE100AB8EE30
:10AED800C77A072A8EED067A3DF4F3AC98ED1C7A12
:10AEE8009DED135A65EE875AE5EE265AE6EE257A69
:10AEF800FDEEE77A17EE902A9342A8BF13468A42DE
:10AF0800A8BF194607EE901AF8EEE77ACEED077A51
:10AF1800FDF7D7BC0699C9003EF5DCACFDF70ABCC5
:10AF2800B0560020D4370020845D0020103A00205D
:10AF38008FC2753CD06D393A00000000C837002038
:10AF48000000008098BC020840360020012A40F327
:10AF5800498607EE101AB8EEC77AC7EE876AB1EECF
:10AF6800E68AB9F1030F13D0BAF1000F09D007EE42
:10AF780090AAF8EEE77AF4EEC87AF1EE10FA01F149
:10AF8800FC80EB6E03EB560393FBF6F36B6202E473
:10AF9800B0EE480A1EF080FC00B2E5E7012A40F353
:10AFA8001D8607EE101AB8EEC77AC7EE876AB1EEAB
:10AFB800E68AB9F1030F14D0BAF1000F09D007EEF1
:10AFC80090AAF8EEE77AF4EEC87AF1EE10FA01F1F9
:10AFD800D4802B6F03EB560393FBF6F3AB62FFF7BA
:10AFE800F3BBB0EE480A1EF057FC00B2E4E7012AB2
:10AFF8007FF703AC07EE101AB8EEC77AC7EE876A78
:10B00800B1EEE68AFFF7FBBBB6EE007AF4EEC75A5C
:10B01800F1EE10FA3FF74DAEFCF783BF98ED005AFA
:10B028009DED0C4ADFF844E625EE855AFDEEC73A59
:10B03800A4EE265AB0EE674AA5EE064A13EE901A19
:10B04800F4EEC44AF1EE10FAB0EE445A88BFB0EEFE
:10B05800475ABDEEC55A15EE100A15EE107A9842F9
:10B06800A8BF1F468142C8BF0F4605EE107AB8EE4A
:10B07800C55A012A8EED005A3DF4A6A898ED045A47
:10B088009DED0D4A25EE855AA4EE265AB0EE674A84
:10B09800A5EE064AF4EEC44AF1EE10FAB0EE445AB0
:10B0A80088BFB0EE475ABDEEC55A15EE100A15EE28
:10B0B800107A9842A8BF1F468842B8BF0F4605EECF
:10B0C800107AB8EEC55A022A8EED015A3DF47CA8D2
:10B0D80098ED085A9DED0E4A25EE855AA4EE265A9B
:10B0E800B0EE674AA5EE064AF4EEC44AF1EE10FA4D
:10B0F800B0EE445A88BFB0EE475ABDEEC55A15EEB9
:10B10800100A15EE107A9842A8BF1F468842B8BFA9
:10B118000F4605EE107AB8EEC55A032A8EED025A8C
:10B128003DF452A898ED0C5A9DED0F4A25EE855A2C
:10B13800A4EE265AB0EE674AA5EE064AF4EEC44AD3
:10B14800F1EE10FAB0EE445A88BFB0EE475ABDEEA1
:10B15800C55A15EE100A15EE107A9842A8BF1F4678
:10B168008842B8BF0F4605EE107AB8EEC55A042AD1
:10B178008EED035A3DF428A898ED105A9DED104A1B
:10B1880025EE855AA4EE265AB0EE674AA5EE064A81
:10B19800F4EEC44AF1EE10FAB0EE445A88BFB0EEAD
:10B1A800475ABDEEC55A15EE100A15EE107A9842A8
:10B1B800A8BF1F468842B8BF0F4605EE107AB8EE02
:10B1C800C55A052A8EED045A3CF4FEAF98ED145A80
:10B1D8009DED114A25EE855AA4EE265AB0EE674A2F
:10B1E800A5EE064AF4EEC44AF1EE10FAB0EE445A5F
:10B1F80088BFB0EE475ABDEEC55A15EE100A15EED7
:10B20800107A9842A8BF1F468842B8BF0F4605EE7D
:10B21800107AB8EEC55A062A8EED055A3CF4D4AF1A
:10B2280098ED185A9DED124A25EE855AA4EE265A35
:10B23800B0EE674AA5EE064AF4EEC44AF1EE10FAFB
:10B24800B0EE445A88BFB0EE475ABDEEC55A15EE67
:10B25800100A15EE107A9842A8BF1F468842B8BF58
:10B268000F4605EE107AB8EEC55A072A8EED065A33
:10B278003CF4AAAF98ED1C5A9DED134A65EE855A29
:10B28800E6EE845AE6EE257AF4EEE74AF1EE10FA95
:10B29800C8BFF0EE477AFEF7CFBE9FEDEF7AF4EE27
:10B2A800C76AF1EE10FA44BF9FEDEC7A77EE666A52
:10B2B800FFF729BB8223FCF740B9DFEDE97AFCF7F9
:10B2C80007B99AF803E0BEF1000F00F02083B4F943
:10B2D8001CE19AF80200A8EB0E0C8CEAEC71A1EBC9
:10B2E800EC71814240F39E84F045C8BF404207EEAE
:10B2F800900AF8EEE77A012138EE278AC4F820216F
:10B3080084F8241186ED038AFDF7F2B9B7EE007AC6
:10B3180077EE677AF4EEE75AF1EE10FA88BFF0EEAE
:10B32800675AD3E498ED005A9DED0C4ADFF83CE3E8
:10B3380025EE855AFDEEC73AA4EE265AB0EE674AC6
:10B34800A5EE064A13EE901AF4EEC44AF1EE10FA8E
:10B35800B0EE445A88BFB0EE475ABDEEC55A15EE56
:10B36800100A15EE107A9842A8BF1F468142C8BF3E
:10B378000F4605EE107AB8EEC55A012A8EED005A2E
:10B388003DF49AAA98ED045A9DED0D4A25EE855A8A
:10B39800A4EE265AB0EE674AA5EE064AF4EEC44A71
:10B3A800F1EE10FAB0EE445A88BFB0EE475ABDEE3F
:10B3B800C55A15EE100A15EE107A9842A8BF1F4616
:10B3C8008842B8BF0F4605EE107AB8EEC55A022A71
:10B3D8008EED015A3DF470AA98ED085A9DED0E4A7B
:10B3E80025EE855AA4EE265AB0EE674AA5EE064A1F
:10B3F800F4EEC44AF1EE10FAB0EE445A88BFB0EE4B
:10B40800475ABDEEC55A15EE100A15EE107A984245
:10B41800A8BF1F468842B8BF0F4605EE107AB8EE9F
:10B42800C55A032A8EED025A3DF446AA98ED0C5AE5
:10B438009DED0F4A25EE855AA4EE265AB0EE674ACE
:10B44800A5EE064AF4EEC44AF1EE10FAB0EE445AFC
:10B4580088BFB0EE475ABDEEC55A15EE100A15EE74
:10B46800107A9842A8BF1F468842B8BF0F4605EE1B
:10B47800107AB8EEC55A042A8EED035A3DF41CAA78
:10B4880098ED105A9DED104A25EE855AA4EE265ADD
:10B49800B0EE674AA5EE064AF4EEC44AF1EE10FA99
:10B4A800B0EE445A88BFB0EE475ABDEEC55A15EE05
:10B4B800100A15EE107A9842A8BF1F468842B8BFF6
:10B4C8000F4605EE107AB8EEC55A052A8EED045AD5
:10B4D8003DF4F2A998ED145A9DED114A25EE855ACE
:10B4E800A4EE265AB0EE674AA5EE064AF4EEC44A20
:10B4F800F1EE10FAB0EE445A88BFB0EE475ABDEEEE
:10B50800C55A15EE100A15EE107A9842A8BF1F46C4
:10B518008842B8BF0F4605EE107AB8EEC55A062A1B
:10B528008EED055A3DF4C8A998ED185A9DED124ABA
:10B5380025EE855AA4EE265AB0EE674AA5EE064ACD
:10B54800F4EEC44AF1EE10FAB0EE445A88BFB0EEF9
:10B55800475ABDEEC55A15EE100A15EE107A9842F4
:10B56800A8BF1F468842B8BF0F4605EE107AB8EE4E
:10B57800C55A072A8EED065A3DF49EA998ED1C5A25
:10B588009DED134A65EE855AE6EE845AE6EE257A75
:10B59800F4EEE74AF1EE10FAC8BFF0EE477AFEF78C
:10B5A8006AB9304B4FEA890E5FEA9A0901EB0E0C33
:10B5B80003EBC818A64400F0518609F101094FEAC7
:10B5C800091908EB090008F110030CF110010EF13C
:10B5D800100213ED024A13ED035A13ED016A13ED3D
:10B5E800047A51ED024A51ED035A51ED016A51EDC9
:10B5F800047A64EE244A65EE255A66EE266A67EEFA
:10B60800277A1033984242ED024A42ED035A42ED3E
:10B61800016A42ED047A01F1100102F11002D8D159
:10B62800A9F11009C8440CEB0901CE441AF0030A29
:10B638003EF43CAFB8EC017AF1EC017A67EE277A78
:10B64800BAF1010AEEEC017AF4D1FEF72FBFDFED73
:10B65800067AFFF70EBB00BFDB0FC9BFDB0F49C07F
:10B66800000002437C2F002000000000403600202C
:10B6780098ED005A9DED0C4A25EE855AA4EE265AFF
:10B68800B0EE674AA5EE064AB0EE445ABEF1000F86
:10B6980000F0E283BAF1000F06D0F4EE444AF1EE6E
:10B6A80010FAC8BFB0EE475ABDEEC77A17EE10CAF7
:10B6B800BDEEC57A05EE10CA17EE101A8C4500F3D8
:10B6C800B3859942A8BF194607EE101AB8EEC77A93
:10B6D800DFF8A4E5012A8EED007A3DF4F2A898ED92
:10B6E800047A9DED0D4A25EE877AA4EE267AB0EE0F
:10B6F800674AA7EE064AB0EE447ABAF1000F00F0A6
:10B708008285F4EEC44AF1EE10FA40F37C85614676
:10B718009942A8BF194607EE101AB8EEC77A022A4E
:10B728008EED017A3DF4CDA898ED087A9DED0E4A8C
:10B7380025EE877AA4EE267AB0EE674AA7EE064A87
:10B74800B0EE447ABAF1000F00F05285F4EEC44A24
:10B75800F1EE10FA40F34C8561469942A8BF1946AC
:10B7680007EE101AB8EEC77A032A8EED027A3DF476
:10B77800A8A898ED0C7A9DED0F4A25EE877AA4EEDD
:10B78800267AB0EE674AA7EE064AB0EE447ABAF1D6
:10B79800000F00F02285F4EEC44AF1EE10FA40F3EF
:10B7A8001C8561469942A8BF194607EE101AB8EEE3
:10B7B800C77A042A8EED037A3DF483A898ED107AAF
:10B7C8009DED104A25EE877AA4EE267AB0EE674AF8
:10B7D800A7EE064AB0EE447ABAF1000F00F0F28400
:10B7E800F4EEC44AF1EE10FA40F3EC846146994253
:10B7F800A8BF194607EE101AB8EEC77A052A8EEDCB
:10B80800047A3DF45EA898ED147A9DED114A25EE70
:10B81800877AA4EE267AB0EE674AA7EE064AB0EE1B
:10B82800447ABAF1000F00F0C284F4EEC44AF1EE93
:10B8380010FA40F3BC8461469942A8BF194607EE46
:10B84800101AB8EEC77A062A8EED057A3DF439A8A3
:10B8580098ED187A9DED124A25EE877AA4EE267A9D
:10B86800B0EE674AA7EE064AB0EE447ABAF1000F86
:10B8780000F09284F4EEC44AF1EE10FA40F38C849E
:10B8880061469942A8BF194607EE101AB8EEC77A62
:10B89800072A8EED067A3DF414A898ED1C7A9DEDE2
:10B8A800134A65EE875AE4EE265AE5EE867ABAF12F
:10B8B800000F00F06884F4EEE47AF1EE10FA40F13B
:10B8C800628462469A42A8BF1A4605EE102AB8EE6C
:10B8D800C55A8EED075AFCF7F4BF07EE902ADFED44
:10B8E800DC6AB8EEE77A66EEA65A9FEDDA5A9FED63
:10B8F800DA6ADFEDDA7AA5EE856A26EEA55AE5EE74
:10B90800867AE5EE276A26EE870AFFF7ABB9B4F91F
:10B918001CC19AF80210A8EB0C0282EAE270A0EBB4
:10B92800E270884240F3708102EBD272012152101A
:10B93800C4F8302184F8341184F82411D4F818217B
:10B948006244B2F5FA6FA8BF4FF4FA62B2F57A7F93
:10B95800B8BF4FF47A7207EE902AB8EEE78A86ED00
:10B96800038AFCF7C5BE98ED005ADDED0C4A25EEBA
:10B97800855AA4EEA65AF0EE674AE5EE064ABDEEF1
:10B98800E45A15EE10EA714500F359819E45A8BFA7
:10B998009E4605EE10EAB8EEC55A002F00F07A85EB
:10B9A800DFF8D4E2012A8EED005A3CF48AAF98ED14
:10B9B800045ADDED0D4A25EE855AA4EEA65AF0EE9E
:10B9C800674AE5EE064ABDEEE45A15EE10CA61452F
:10B9D80000F3CB819C45A8BF9C4605EE10CAB8EE83
:10B9E800C55A002F00F0F685022A8EED015A3CF464
:10B9F80068AF98ED085ADDED0E4A25EE855AA4EE9B
:10BA0800A65AF0EE674AE5EE064ABDEEE45A15EE90
:10BA180010CA614500F3DA819C45A8BF9C4605EE33
:10BA280010CAB8EEC55A002F00F0C985032A8EED5A
:10BA3800025A3CF446AF98ED0C5ADDED0F4A25EE5C
:10BA4800855AA4EEA65AF0EE674AE5EE064ABDEE20
:10BA5800E45A15EE10CA614500F3B5819C45A8BFAC
:10BA68009C4605EE10CAB8EEC55A002F00F0458571
:10BA7800042A8EED035A3CF424AF98ED105ADDEDFC
:10BA8800104A25EE855AA4EEA65AF0EE674AE5EE6E
:10BA9800064ABDEEE45A15EE10CA614500F36B8103
:10BAA8009C45A8BF9C4605EE10CAB8EEC55A002FA3
:10BAB80000F01885052A8EED045A3CF402AF98ED83
:10BAC800145ADDED114A25EE855AA4EEA65AF0EE79
:10BAD800674AE5EE064ABDEEE45A15EE10CA61451E
:10BAE80000F346819C45A8BF9C4605EE10CAB8EEF7
:10BAF800C55A002F00F08D84062A8EED055A3CF4B5
:10BB0800E0AE98ED185ADDED124A25EE855AA4EEFE
:10BB1800A65AF0EE674AE5EE064ABDEEE45A15EE7F
:10BB280010CA614500F32A819C45A8BF9C4605EED2
:10BB380010CAB8EEC55A002F00F0C984072A8EED46
:10BB4800065A3CF4BEAE98ED1C5ADDED134A65EE7C
:10BB5800855AE6EEA45AE6EE257AFDEEE77A17EE68
:10BB6800902A914203DC9A42A8BF1A46114607EE72
:10BB7800901AF8EEE77A002F7FF4C8A9069B002BED
:10BB88007FF4C4A9059B5B45B8BFF0EE477AFFF781
:10BB9800BDB977EEC76AF0EE477AFEF740BDBCF84C
:10BBA80034209FED2F7A07EE902AF8EEE77A2D4A97
:10BBB80067EE877AC2ED007AFCF7BCBD2A4B1F6896
:10BBC80017F080577FF475A8FFF76EB8F0EE477A44
:10BBD800FDF7BCBCB0EE677AFDF7A2BC9FED2A8AE0
:10BBE800FFF7E7B99FED288AFFF7BBB99FED1F0A5A
:10BBF800DFF8888025EE800A1DF04EFED4F8DC615F
:10BC0800A8F80600FBF7ADBC94F82421002A3FF4FD
:10BC180095AED4F82C2184F834E184F824E1C4F8F2
:10BC280028218BE694F8241129B1D4F82C1184F832
:10BC38002421C4F82811D4F81821724481E605EEAD
:10BC4800101AA8E60A490B4A8C46FEF71EBC00BF2C
:10BC580084F9223F92E741B99730083C15A82ABEDB
:10BC68006F12833A78000020C83700200000C842CD
:10BC7800FC3000200021002040360020A83C002095
:10BC880035FA8E3CDB0FC93F0000000007EE906AD2
:10BC9800F8EEE78A5FED067A1FED060A84F8B861C8
:10BCA80068EEA78A38EE800AFDEEC07A17EE903A61
:10BCB8002033402B40F2B5821FED0D0A584BFDEEA4
:10BCC800E87A83ED010A17EE903A2033402B00F210
:10BCD800A582DFED547AF4EEE78AF1EE10FA40F32C
:10BCE8009583DFED516ADFED517A01E0F0EE478A86
:10BCF800F4EEE78AF1EE10FA38EEE67AF6DCDFEDDC
:10BD08004C7AB4EEE77AF1EE10FA40F17C839FEDBD
:10BD1800466ADFED486A01E0B0EE677AB4EEE67A8B
:10BD2800F1EE10FA77EE067AF6D49FED437AF4EE48
:10BD3800C77AF1EE10FA40F37B829FED3A7A77EEFC
:10BD4800677A27EEA76ADFED3D5ADFED3D6A9FED82
:10BD58003D7AE6EE256A67EE865AA6EE267AE5EE85
:10BD6800877AC4ED6F7AFDF79EBE05EE101A36E6A7
:10BD780005EE101ABBE605EE101A96E605EE101A47
:10BD8800D7E696ED000A059306921DF085FD2E492B
:10BD9800DFF8BCE0D1F8EC10DFF8B880069AA8F814
:10BDA80000008EFB013EC917C1EBAE1107EE901AD9
:10BDB800F8EEE77A059BFDEEE77A17EE901AA8F8F9
:10BDC8000210FCF712BD05EE101A4CE605EE101A2B
:10BDD80027E6F0EE476AFEF78ABD02F06FF8069B89
:10BDE800DFF87080D4F8E091D4F8DC61C01AA8F8C4
:10BDF8000200FEF7C6BB02F061F8144BDFF854806E
:10BE08001F78069B99F80020D4F8DC61C01AA8F8BE
:10BE18000400FEF7FFB9B0EE667AFEF752BD00BF28
:10BE280078000020DB0F4940DB0FC940E4CB164106
:10BE3800DB0F49C0E4CB16C1DB0FC93F92E741B91C
:10BE48009730083C15A82ABE68100020A43C0020A2
:10BE5800D34D6210A83C0020BAF1000F06D0F4EED2
:10BE6800444AF1EE10FAC8BFB0EE475ABDEEC74AD1
:10BE7800BDEEC55A14EE10CA15EE101A8C4514EE14
:10BE8800109A00F337829942A8BF194605EE101A96
:10BE9800B8EEC55A002F00F01083DFF8ECE5012A50
:10BEA8008EED005A3CF40DAD98ED045A9DED0D4A07
:10BEB80025EE855AA4EE265AB0EE674AA5EE064A44
:10BEC800B0EE445ABAF1000F00F00B82F4EEC44A07
:10BED800F1EE10FA40F3058261469942A8BF19466F
:10BEE80005EE101AB8EEC55A002F00F05E83022A3C
:10BEF8008EED015A3CF4E5AC98ED085A9DED0E4ADA
:10BF080025EE855AA4EE265AB0EE674AA5EE064AF3
:10BF1800B0EE445ABAF1000F00F0DA81F4EEC44AE8
:10BF2800F1EE10FA40F3D48161469942A8BF194650
:10BF380005EE101AB8EEC55A002F00F02C83032A1C
:10BF48008EED025A3CF4BDAC98ED0C5A9DED0F4AAB
:10BF580025EE855AA4EE265AB0EE674AA5EE064AA3
:10BF6800B0EE445ABAF1000F00F0A981F4EEC44AC9
:10BF7800F1EE10FA40F3A38161469942A8BF194631
:10BF880005EE101AB8EEC55A002F00F0FA82042AFE
:10BF98008EED035A3CF495AC98ED105A9DED104A7D
:10BFA80025EE855AA4EE265AB0EE674AA5EE064A53
:10BFB800B0EE445ABAF1000F00F07881F4EEC44AAA
:10BFC800F1EE10FA40F3728161469942A8BF194612
:10BFD80005EE101AB8EEC55A002F00F0C882052ADF
:10BFE8008EED045A3CF46DAC98ED145A9DED114A4F
:10BFF80025EE855AA4EE265AB0EE674AA5EE064A03
:10C00800B0EE445ABAF1000F00F04781F4EEC44A8A
:10C01800F1EE10FA40F3418161469942A8BF1946F2
:10C0280005EE101AB8EEC55A002F00F0E882062A6D
:10C038008EED055A3CF445AC98ED185A9DED124A20
:10C0480025EE855AA4EE265AB0EE674AA5EE064AB2
:10C05800B0EE445ABAF1000F00F01681F4EEC44A6B
:10C06800F1EE10FA40F3108161469942A8BF1946D3
:10C0780005EE101AB8EEC55A002F00F0B682072A4E
:10C088008EED065A3CF41DAC98ED1C5A9DED134AF2
:10C0980065EE855AE6EE845AE6EE257ABAF1000F87
:10C0A80040F0E680FDEEE77A17EE902A944540F3DB
:10C0B800E68007EE909AF8EEE77A002F7EF426AF36
:10C0C8005CE501F0FBFEDA4BDFF8C0831F78069BC6
:10C0D800C01AA8F80200FEF7B0B80A980BF05AFD8B
:10C0E800FEF78DBCDFEDD37AF4EEE76AF1EE10FAD5
:10C0F80040F33A82DFEDD05A9FEDD06A01E0F0EECE
:10C10800676AF4EEC66AF1EE10FA76EEE57AF6DCC6
:10C11800DFEDCB6AF4EEE67AF1EE10FA40F1218217
:10C12800DFEDC55A9FEDC76A01E0F0EE667AF4EEDE
:10C13800C67AF1EE10FA77EEA56AF6D4DFEDC27A88
:10C14800F4EEE76AF1EE10FA05DDDFEDBA7A77EE84
:10C15800E66AFFF7C8BBDFEDBD7AF4EEE76AF1EEF9
:10C1680010FA44BFDFEDB67A77EEE66AFFF7BBBB9D
:10C17800B74800F1800CFEF734B8A8F80600A5F817
:10C18800B460FCF7E1B8FDEEE77A17EE902A624555
:10C19800FFF69DABFFF796BBBDEEC77A17EE101AF8
:10C1A8006145BFF66EAB07EE10CAFFF76FBBBDEE79
:10C1B800C77A17EE101A6145BFF63EAB07EE10CAF4
:10C1C800FFF73FBBBDEEC77A17EE101A6145BFF601
:10C1D8000EAB07EE10CAFFF70FBBBDEEC77A17EE1E
:10C1E800101A6145BFF6DEAA07EE10CAFFF7DFBADC
:10C1F800BDEEC77A17EE101A6145BFF6AEAA07EE74
:10C2080010CAFFF7AFBABDEEC77A17EE101A61452C
:10C21800BFF67EAA07EE10CAFFF77FBADFED8D7A68
:10C228009FE5F8F719F949E507EE10CAFFF74EBA86
:10C238009FED867AF4EEC77AF1EE10FA44BF9FEDCF
:10C24800807A77EE677A7CE5802013F06BFC08B182
:10C2580012F0C0FC0CF066FDFEF789BB6146FFF7E3
:10C26800E5B994F80832002B7BF4DFABFBF7CBBBC6
:10C27800F4EEE74AF1EE10FA7FF714AF62469A42FD
:10C28800A8BF1A46914614E7BDEEC55A15EE101A16
:10C298006145BFF6EAAE6146EAE6BDEEC55A15EE5F
:10C2A800101A6145BFF6B9AE6146B9E6BDEEC55A8A
:10C2B80015EE101A6145BFF688AE614688E6BDEEF8
:10C2C800C55A15EE101A6145BFF657AE614657E6D6
:10C2D800BDEEC55A15EE101A6145BFF626AE614689
:10C2E80026E6BDEEC55A15EE101A6145BFF6F5AD46
:10C2F8006146F5E514EE101AC8E5DFF89481D8F820
:10C30800000012F049FC544B1B780022022BC8F89D
:10C3180000207EF42AAB12F089FEFEF726BB4F4AB6
:10C328004F4B10681B689847089BDBED007A93ED2C
:10C33800007A4C4BD7ED006A83ED020A4A4B67EE50
:10C34800277A2B4427EE8C7AD3ED007A474B67EE99
:10C35800277AF0EE665AE7EE8D5A93ED006AB1EE51
:10C36800467AF4EEC75AF1EE10FA08D4F4EEC65A3B
:10C37800F1EE10FA8CBFB0EE467AB0EE657A3C4B1F
:10C388001B78012B02D0192B7BF4C4AADFED397A74
:10C39800B4EEE7DAF1EE10FACCBF01230023FBF785
:10C3A800C4BADFED357AF4EEE7DAF1EE10FA27DCFD
:10C3B800DFED327AF4EEE7DAF1EE10FA20D4304B02
:10C3C800D3ED007AB1EE677AB4EEC7DAF1EE10FA7F
:10C3D8002AD4B4EEE7DAF1EE10FA88BFB0EE67DAE5
:10C3E800284BC7ED00BA1B689A427BF756AAFCF7A0
:10C3F800E8BC1AF80330002B7EF4B9AAFEF7EEBBAE
:10C408009FED14DAECE7F0EE477A8EE4B0EE687A46
:10C4180075E4069800287FF46FAB05985845B8BFB7
:10C42800B0EE475AFFF768BBB0EE47DAD8E700BF6F
:10C43800A43C0020DB0F4940DB0FC940E4CB164188
:10C44800DB0F49C0E4CB16C1DB0FC93FDB0FC9BF07
:10C458000021002000000000203800204C26002089
:10C4680060260020E035002070260020D826002015
:10C47800342400200000964200C0F84400C0F8C4EC
:10C48800D4260020B826002040360020A83C0020F2
:10C49800885D0020069800287FF482AA05985845F0
:10C4A800B8BFB0EE475AFFF77BBA802013F03AFBCB
:10C4B80000287CF44AAEFEF711BB069900297FF4E8
:10C4C800ECAC05995945B8BFB0EE475AE5E4069873
:10C4D80000287FF433AB05985845B8BFB0EE475AEB
:10C4E800FFF72CBB069800287FF4E4AA0598584566
:10C4F800B8BFB0EE475AFFF7DDBA069800287FF4B8
:10C50800B7AA05985845B8BFB0EE475AFFF7B0BA72
:10C51800132B05D1B0EE480A1DF0BEF9AAF80000A9
:10C52800B0EE480AD5F814323A4898473A4B1B7887
:10C53800132BB0EE408A7BF455A81DF0ADF9AAF88C
:10C548000200FBF74FB845201BF014FBFF201BF03F
:10C5580011FB32481BF0FAFA30461BF00BFBFEF7D2
:10C5680031BAF0EE676AE9E5F0EE667AD0E5069949
:10C5780000297FF434AD05995945B8BFB0EE475A44
:10C588002DE5069900297FF402AD05995945B8BFF4
:10C59800B0EE475AFBE4069900297FF4D0AC059920
:10C5A8005945B8BFB0EE475AC9E4069900297FF447
:10C5B8009EAC05995945B8BFB0EE475A97E406981E
:10C5C80000287FF433AA05985845B8BFB0EE475AFB
:10C5D800FFF72CBA069800287FF406AA0598584554
:10C5E800B8BFB0EE475AFFF7FFB9069900297FF4A4
:10C5F80046AD05995945B8BFB0EE475A3FE506998B
:10C6080000297FF414AD05995945B8BFB0EE475AD3
:10C618000DE500BFF0480020A43C002004E2020819
:10C6280038B50B4C23688BB15A68821A002A054624
:10C6380004DA0CE05A68AA1A002A07DB9A68226012
:10C6480018461A6890472368002BF3D138BD38BDC7
:10C65800843200200D4B01210022890710B4027298
:10C6680003F1640402D51979815401329C4203F123
:10C67800140308D0072A06DC99798907F3D49C4269
:10C6880003F11403F6D15DF8044B7047BCDC0208D3
:10C6980024230370704700BF0122102302704370E7
:10C6A800704700BF436A8269D154436A0169426B8B
:10C6B80001338B4228BF00234362002A2FD0EFF3B7
:10C6C8001181502383F31288436B1A68D2072CD444
:10C6D80070B45E686EB9456A826A954217D08469FB
:10C6E8001444DC600ED9AA1A5A608562002280F8C8
:10C6F80050201A6842F00102C9B21A6081F3118809
:10C7080070BC70470469A21A5A608662EEE701237A
:10C7180080F85030C9B281F3118870BC7047C26C80
:10C72800136843F0800313607047C9B281F311881E
:10C73800704700BF026B10B462B1036CC2684469F1
:10C74800D11A013B615C5DF8044B08BF13460364D2
:10C75800C8B27047016A4369C4685B5C0131A14291
:10C7680028BF114601625DF8044BD8B2704700BF7C
:10C77800436B13B190F850007047836A406A181AE7
:10C78800B0FA80F040097047416A836A99420AD337
:10C79800CB1A416B026961B14968501E0B44834250
:10C7A8000AD2C01A704702691144CB1A416B00299A
:10C7B800F2D1501EC01A704700207047036B43B176
:10C7C800026C5B6893422FBF981AC0689B1AC01806
:10C7D8007047C269036A9A422FBFD01AC06880188E
:10C7E800C01A70472B2303732A2383700023837591
:10C7F800704700BF03682DE9F041DF691FB13B4670
:10C80800BDE8F0411847002A164611DD04460D46DA
:10C818000E4400E023689B68204698470028F9D01A
:10C82800236815F8011B1B6820469847AE42F1D1D2
:10C83800BDE8F08100233F22027043708370C3700B
:10C84800704700BF08B505F033FE024B024ADA60B4
:10C85800FEE700BF00ED00E00400FA052DE9F0470F
:10C868000569C3681D4028D00F4606464FF00048AA
:10C878004FF00009B5FA85F328FA03F2D2431B3BBF
:10C8880032611540042B16D8DFE803F0312921194D
:10C8980003007B6A002B32D003F1FF3A1FFA8AFAB1
:10C8A800C7F824903C6A34B123682046514698471B
:10C8B8006468002CF8D1002DDCD1BDE8F087386819
:10C8C800716B036889B29847002DD3D1F5E7786872
:10C8D800B16B036889B29847002DCBD1EDE7B868F2
:10C8E800F16B036889B29847002DC3D1E5E7F86872
:10C8F800316C036889B29847002DBBD1DDE7F36A34
:10C908001FFA83FACEE700BF30B50446C06C6171E8
:10C918000368A26823F00103036087B0A37900923B
:10C9280013F004023DD04FF4805213F00203019239
:10C9380044D102934FF480630022039311F0010362
:10C94800059237D1049308238D07694648BF04939D
:10C9580018F07EFE6079E36CA17900F00202002AEB
:10C9680015BF4FF440324FF480324FF400340024A6
:10C9780010F0010F586808BF2246CC074CBF02438D
:10C9880020EA02025A609A6809074CBF42F008027E
:10C9980022F008029A601A6842F001021A6007B091
:10C9A80030BD13F0020301920BD04FF4005513462B
:10C9B8000295C1E7042304930C23C5E74FF4005301
:10C9C800B7E70293B8E700BF10B50446C06CA16092
:10C9D800036823F001030360A37986B013F004020F
:10C9E800009141D04FF4805213F00203019244D1D8
:10C9F80002934FF4806362790393D1074FF00003E9
:10CA08000493059345BF0423049308230C23694624
:10CA1800920748BF049318F01BFE6079E36CA17974
:10CA280000F00202002A15BF4FF440324FF4803262
:10CA38004FF40034002410F0010F586808BF224654
:10CA4800CC074CBF024320EA02025A609A680907E1
:10CA58004CBF42F0080222F008029A601A6842F0BD
:10CA680001021A6006B010BD13F00203019207D04C
:10CA78004FF4005113460291BDE74FF40053B7E756
:10CA88000293B8E7022810B428BF0220064C074BCF
:10CA9800207000EB8001064A5DF8044BC0EBC10032
:10CAA80003EB4000106070470C3F00205433002017
:10CAB800183F002008B516F09FFFF7F77BF9BDE88F
:10CAC800084016F081BF00BF2DE9F04F013085B056
:10CAD800C3B203938E4D8F4F8F4C904E0A2302930F
:10CAE8003220DFF8409217F009FF4FF4FA7A4FF03E
:10CAF800100C4FF47A70D9F80430C3F30803002BF4
:10CB080040F0C880EFF31183002B40F0C380296800
:10CB1800A26800BF2B689942F9D1D7F800E000FB62
:10CB28000EF39B1AB3FBFEF300FB01314FF0010E2D
:10CB38000191D9F80430C3F30803002B40F08E802C
:10CB4800EFF31183002B40F089802B68A16800BFA8
:10CB58002A689342F9D1D7F800B000FB0BF2521AB9
:10CB6800B2FBFBF200FB0323019A9B1AB3F57A7F11
:10CB7800DFD3BAF1010ABED1039B002B40F0C48079
:10CB88004FF47A7ADFF89C9150464FF0100CD9F8A0
:10CB98000430C3F30803002B40F09980EFF31183AE
:10CBA800002B40F094802968A26800BF2B68994246
:10CBB800F9D1D7F800E000FB0EF39B1AB3FBFEF3A4
:10CBC80000FB01314FF0010E0191D9F80430C3F395
:10CBD80008033BBBEFF3118323BB2B68A16800BF9D
:10CBE8002A689342F9D1D7F800B000FB0BF2521A29
:10CBF800B2FBFBF200FB0323019A9B1AB3F57A7F81
:10CC0800E3D3BAF1010AC2D1029B013B02937FF43C
:10CC180067AF4349434B4448444A0860DA6005B06B
:10CC2800BDE8F08FEFF311888CF31288A1682368B0
:10CC3800DB0344BFC6F800E0A1682B6832685FFADE
:10CC480088F888F31188D7F800801A4400FB08F3A5
:10CC58005B1AB3FBF8F300FB0233CDE7EFF311885F
:10CC68008CF31288A1682368DB0344BFC6F800E090
:10CC7800A1682B6832685FFA88F888F31188D7F8BA
:10CC880000801A4400FB08F35B1AB3FBF8F300FBBF
:10CC9800023369E7EFF311828CF31288D4F808E0C5
:10CCA8002368D90303D501233360D4F808E02B683F
:10CCB8003168D2B282F311883A68194400FB02F352
:10CCC800A3EB0E03B3FBF2F300FB01312EE7EFF306
:10CCD80011828CF31288D4F808E02368D90303D5AD
:10CCE80001233360D4F808E02B683168D2B282F3AC
:10CCF80011883A68194400FB02F3A3EB0E03B3FB57
:10CD0800F2F300FB01315DE7184617F09DFC37E7A9
:10CD1800B0560020B456002010E000E0AC560020C9
:10CD2800FC9F002000ED00E0EFBEADDE0400FA0538
:10CD380038B5434B5A899989914224BF00225A81B8
:10CD4800198ADA89914224BF0022DA81DA788AB313
:10CD5800072A2FD03B493C4D91F857000124002168
:10CD68000A282C709C70D9713DD00C2865D0DFED55
:10CD7800377A8ABB364C9FED370AA278002918BF4C
:10CD8800F0EE407A062A04D8334901EB820191ED8E
:10CD9800000A217959B3013A032A4DD8F7EE007AEF
:10CDA80087EE800A1CF078FD2388984228BF184631
:10CDB800208038BDD97921B198780428B8BF0420DB
:10CDC8009870204890F857000A280CD00C28CED12B
:10CDD800DFED227A002ACDD0072ACBD00A282CD121
:10CDE800DFED1F7AC6E70A20DFED1E7AC1E79B78E0
:10CDF800154A07EE103A1178B8EEC77A27EE277A67
:10CE080007EE901AF8EEE77A67EE877AB4EEE70A4B
:10CE1800F1EE10FA10DDC0EE077AFDEEE77A17EEB4
:10CE2800903A102BA8BF1023012BB8BF0123DBB207
:10CE38008B4238BF0B46137038BDDFED0B7A99E78C
:10CE4800C4460020D8460020F43700206F1203396A
:10CE58006C4B00206F120338D8BE02080AD7A339DA
:10CE68000F506E3A5304E9386F12833A2DE9F047B0
:10CE7800B24FB34E16F0C0FDBE421ED2DFF8488353
:10CE8800DFF848934446258862197DB14A450DD29A
:10CE9800052D0BD933886188C3F30B03994200F041
:10CEA800F280144625886219002DEFD1716830464A
:10CEB8001436F6F70BFFBE42E4D3A24A1378A3F167
:10CEC800170102290FD9A04911F83300002840F0B2
:10CED8000681D8000144497829B19C4911F83330BA
:10CEE800002B00F024819A4B5A78022A40F2F180F4
:10CEF800002298495A701A789748022A016000F26D
:10CF0800E48002EB8201954BC2EBC10203EB4203C2
:10CF1800998C5A8C924C9142236001D300225A84F6
:10CF2800904B9A78042A00F0F98032B91A88B2F541
:10CF3800F07F84BF4FF4F0721A808B4DFFF7F8FE34
:10CF48002B688A4A1A40002A00F0F480D80700F1BA
:10CF5800E080590400F1D8801A0700F1D0809B04C2
:10CF680000F1C68014F0C0FE10B9814811F012FA21
:10CF78004020F6F7E1FE8020F6F7DEFE4FF4007061
:10CF8800F6F7DAFE4FF48020F6F7D6FE4FF40010DD
:10CF9800F6F7D2FE4FF00070F6F7CEFE4FF0806045
:10CFA800F6F7CAFE4FF00060F6F7C6FE1AF080F9F1
:10CFB800002130226F481EF030FD206804F058FF31
:10CFC8006D4B266803F1500102E0043399427AD090
:10CFD8001A78002AF9D19C78D8788442F5D2674922
:10CFE800674B91F804E06748674D5C6B674B2860B6
:10CFF800C827642111FB0E71DFF8D4E15960644F32
:10D0080030F8061C634DAEF8001000219960D96015
:10D01800196159619961D96183F8201083F8211049
:10D028003A702E600CB109F0E9FB5B4B9FED5B5A3F
:10D038001B885B4A9FED5B6A55795B4C5B495C4892
:10D04800086006EE903AF8EEE66A1388C5EE265AAE
:10D0580007EE103A53881279C4ED005A07EE903A59
:10D06800B8EEC77A534BF8EEE77A1D725A7227EE7C
:10D07800067A67EE867ABDE8F04783ED017AC3ED5C
:10D08800007A16F0A1BC63799B077FF40AAF716838
:10D0980094F804A03046F6F719FE3388BAEB133F2C
:10D0A80004D01436BE42FFF4EDAE06E7738870680C
:10D0B800AA1FC3F30B039A4204F10601A8BF1A463C
:10D0C8001CF076FAEDE7012289E700221A70234B5B
:10D0D8001EE7204902EB420201EB82010BE7D80070
:10D0E8000C186468002C7FF4F5AE17241470F1E670
:10D0F8003148F6F721FE4020F6F71EFE32E72F48AA
:10D10800F6F71AFE2B682AE72D48F6F715FE2B6866
:10D1180022E72C48F6F710FE2B681AE79A8AB2F530
:10D128007A7FBFF40AAF4FF47A729A8205E7182320
:10D138001370D8E643F001032B6007E7E0160308F5
:10D14800D01203083C3800208CD60208A0BF020881
:10D158000C3F00201C3F0020045D002054330020B9
:10D16800183F00206C4B002090340020096000021A
:10D178004C570020FC23002040380020A03B002012
:10D18800403F00200638002094460020BC3E002086
:10D19800071C00203024002044220020C0C9FB487E
:10D1A8003C23002017B7D138482200205C3A0020E1
:10D1B8003661023D383A0020094000020160000251
:10D1C800092000020860000202F0030800000408B9
:10D1D800E42E002008B516F00FFCF6F7EBFD16F06C
:10D1E800F3FBBDE8084041E638B50D4C0D4DAC42A7
:10D1F80006D2616820461434F6F768FDAC42F8D3CD
:10D20800F7F71EFA084A094B094C1460002209492D
:10D218001A705A7008480860BDE838400FF0DCBF43
:10D22800D0120308E0160308183F00200C3F002026
:10D2380054330020045D00201C3F002008B5FFF790
:10D24800D3FF16F0D9FBF6F7B5FDBDE8084016F098
:10D25800BBBB00BFF0B50C292BD8DFE801F06F2A63
:10D268002A2A4C2A2A2A2B2A2A2A0700046AB2F8D0
:10D278000CE097881668674D24F480540462036AAA
:10D288004468C16923F4005343EA0E3321F4E641AC
:10D29800A84243EA073341EA062100F0B58005F5C4
:10D2A8000065A84200F0B08092684460C1610264E1
:10D2B8000362F0BD046A96899588D2F800E0554F5C
:10D2C80024F480740462036A4468C16923F4007317
:10D2D80043EA062321F07301B84243EA052341EAF1
:10D2E8000E017ED04C4DA8427BD092684460C1614B
:10D2F800C2630362F0BD046A96899588D2F800E09B
:10D30800444F24F010040462036A4468816923F0DE
:10D31800200321F0807143EA061321F4E641B84264
:10D3280043EA051341EA0E2148D03B4DA84245D0B7
:10D3380092684460816182630362F0BD046A9389E4
:10D34800B2F804E01768334E24F001040462056A59
:10D358004468816943EA0E0321F4803125F002050F
:10D368009BB221F07301B04243EA050341EA070189
:10D3780014D0294DA84211D005F54065A8420DD01A
:10D3880005F58065A84209D005F58065A84205D055
:10D3980092684460816142630362F0BDD689158A50
:10D3A800578A23F0080333433D43D68824F4407456
:10D3B80023F00403ADB233432C43E9E7D589178A38
:10D3C800D68823F0800343EA051324F44064558A81
:10D3D80023F0400344EA870443EA061344EA850439
:10D3E800A6E7D589178AD68823F4006343EA05237C
:10D3F80024F44054558A23F4806344EA071443EA2A
:10D40800062344EA051470E7158A24F4804444EAA4
:10D41800851449E7002C0140003401402DE9F04F04
:10D42800C822002183B07948794CDFF80892794DF9
:10D43800794E7A4FDFF800821EF0EFFA7848794982
:10D44800DFF8F8E1DFF8F8C100221359834200F051
:10D45800C280B3F1804F00F0CA80AB4200F0C980AF
:10D46800B34200F0C880BB4200F0C780734500F0AB
:10D47800C680634500F0C580434500F0C480DFF8EE
:10D48800C4A153457AD00AF5806A534508BF0923D9
:10D4980075D01432782AD8D15D4C634D634E614FF4
:10D4A80004F1780802E01434A04564D0A379002B75
:10D4B800F9D023794FEA131909F1FF39B9F1050FAA
:10D4C80003F00F03EFD835F8190040FA03F2D2073A
:10D4D800E9D54FF0010A0AFA03F3013B18401BF0A3
:10D4E800C9FD16F809305249184411EBC002DAD0C8
:10D4F80051F83000DFF850E1217A00F138439B0AF7
:10D508001EF8033003F01F0E5B09022B0AFA0EFA0D
:10D5180063D0032B66D0012B58D093880093B3FABD
:10D5280083F3C3F11F039BB2DA0800EB820203F016
:10D538000703D2F820E09B004FF00F0C0CFA03FC15
:10D548002EEA0C0EC2F820E0D2F820E001FA03F32C
:10D5580043EA0E03136269460023022214348DF84D
:10D5680004208DF805308DF806308DF8073018F056
:10D57800CBF8A0459AD103B0BDE8F08F082309EB9A
:10D58800C3034FF0010B93F804A00AF01F034FEAFE
:10D598005A1ABAF1020F0BFA03F311D0BAF1030FBA
:10D5A80008D0DA457FF475AFD1F814A043EA0A032E
:10D5B8004B616EE7D1F81CA043EA0A03CB6168E728
:10D5C800D1F818A043EA0A038B6162E77B694AEA4B
:10D5D80003037B61A1E70023D1E7BB694AEA0303A0
:10D5E800BB619AE7FB694AEA0303FB6195E70123FC
:10D5F800C5E70223C3E70323C1E70423BFE70523E5
:10D60800BDE70623BBE70723B9E700BF3039002091
:10D61800BCDC020800040040000800400010004084
:10D62800002C014000100240A8DD0208B4DD020809
:10D6380038580020B8DB02080040014000140040C0
:10D648000034014000440140BCDD020803682DE9B4
:10D65800F04F03F13845644EAD0A0124755D05F0BD
:10D668001F066D09022D04FA06F400F0A280032DAE
:10D6780000F0A480012D52D08088B0FA80F4C4F163
:10D688001F04A4B2E50803EB850504F007042E6A1D
:10D69800A4000F27A74026EA07062E622E6A01F08B
:10D6A800030702FA04F47A1E3443012AC1F3810CF9
:10D6B800C1F300182C62C1F3411135D9C60700F136
:10D6C8009780850700F1A380440700F1B180020725
:10D6D80000F1BF80C60600F1CD80850600F1DB8031
:10D6E800440600F1E980020600F1F780C60500F162
:10D6F8000581850500F11381440500F121810205AA
:10D7080000F12F81C60400F13D81850400F14B81B1
:10D71800440400F15981020455D4BDE8F08F334D1B
:10D728006E6934436C61A7E7002422464FF0010E6E
:10D738004FF0030904E00132102A04F10204ECD08E
:10D748000EFA02F636EA0005F5D1D3F808A009FA70
:10D7580004F5ED430AEA050AC3F808A0D3F808B0AF
:10D768000CFA04FA4AEA0B0AC3F808A0B3F804A0B2
:10D778001FFA8AFA2AEA06069E80B3F804A008FA75
:10D7880002F646EA0A06B6B29E801E682E401E6061
:10D79800D3F800A007FA04F646EA0A061E60D3F892
:10D7A8000CA001FA04F605EA0A0A46EA0A05DD6051
:10D7B800C1E70E4DAE693443AC615DE70B4DEE69D0
:10D7C8003443EC6158E71A6822F040421A601A683C
:10D7D80042EA87771F60DA6822F0404242EA8171A4
:10D7E800D960BDE8F08F00BFBCDD02080010024020
:10D7F8001A6822F003021A601A683A431A60DA6853
:10D8080022F003020A438507DA607FF55DAF1A68E4
:10D8180022F00C021A601A6842EA87021A60DA6873
:10D8280022F00C0242EA81024407DA607FF54FAF2A
:10D838001A6822F030021A601A6842EA07121A605F
:10D84800DA6822F0300242EA0112DA6002077FF554
:10D8580041AF1A6822F0C0021A601A6842EA8712B9
:10D868001A60DA6822F0C00242EA8112C606DA605B
:10D878007FF533AF1A6822F440721A601A6842EAD8
:10D8880007221A60DA6822F4407242EA0122850609
:10D89800DA607FF525AF1A6822F440621A601A68C8
:10D8A80042EA87221A60DA6822F4406242EA812258
:10D8B8004406DA607FF517AF1A6822F440521A60FE
:10D8C8001A6842EA07321A60DA6822F4405242EAD9
:10D8D8000132DA6002067FF509AF1A6822F4404285
:10D8E8001A601A6842EA87321A60DA6822F44042FB
:10D8F80042EA8132C605DA607FF5FBAE1A6822F487
:10D9080040321A601A6842EA07421A60DA6822F45A
:10D91800403242EA01428505DA607FF5EDAE1A68C9
:10D9280022F440221A601A6842EA87421A60DA68CA
:10D9380022F4402242EA81424405DA607FF5DFAEF4
:10D948001A6822F440121A601A6842EA07521A60EA
:10D95800DA6822F4401242EA0152DA6002057FF5E1
:10D96800D1AE1A6822F440021A601A6842EA875255
:10D978001A60DA6822F4400242EA8152C604DA6088
:10D988007FF5C3AE1A6822F040721A601A6842EA3C
:10D9980007621A60DA6822F0407242EA016285047E
:10D9A800DA607FF5B5AE1A6822F040621A601A682C
:10D9B80042EA87621A60DA6822F0406242EA8162CB
:10D9C8004404DA607FF5A7AE1A6822F040521A6064
:10D9D8001A6842EA07721A60DA6822F0405242EA8C
:10D9E8000172DA6097E600BF10B50409013C052C06
:10D9F80017D80D4B33F8142000F00F0042FA00F34B
:10DA080013F001030DD0012303FA00F00138104090
:10DA18001BF030FB054A064B125D104403EBC000B7
:10DA280010BD002010BD00BFA8DD0208B4DD02084B
:10DA38003858002001490248FEF710BFD0390020AD
:10DA48000040014001490248FEF708BFA8390020FC
:10DA58000034014001490248FEF700BFA839002000
:10DA68000034014001490248FEF7F8BE8039002021
:10DA78000004004002494FF08040FEF7EFBE00BFAF
:10DA88005839002001490248FEF7E8BE3039002025
:10DA9800002C014001490248FEF7E0BE3039002061
:10DAA800002C01402DE9F04104684A4DA30AAB421D
:10DAB80072D009D8B3F5801F6AD04A3DAB425AD11B
:10DAC8004FF0700E022608E0434DAB4268D0033594
:10DAD800AB4252D14FF0C00E042647794FEA970C5B
:10DAE800002961D0B000634685190227D4F80C805C
:10DAF8009F400CEB4503BFB2384D03F1040C47EAD5
:10DB0800080745F8231045F82C20E760EFF311814A
:10DB1800502282F31288821905EBC202136973B38B
:10DB280013620433821905EBC202576917B11F60EB
:10DB380053690433821905EBC202976917B11F6054
:10DB480093690433821905EBC202D76917B11F60C4
:10DB5800D36904330027CAB21F6082F311883044A6
:10DB680005EBC000036A6BB9E3684FF6FE72134019
:10DB7800E360BDE8F081BDE8F081BDE8F08105EB28
:10DB88000E03CFE7E36843F00103E360BDE8F081EB
:10DB98004FF0480E0126A0E74FF0200E00269CE724
:10DBA8004FF0980E032698E7BF08022306FA03F001
:10DBB800BB40DB43E768094D9BB23B4087190CEB40
:10DBC800470CE3600CF1040345F82C1045F82320BA
:10DBD8009CE700BF4B0010004D00100030390020BA
:10DBE8001F4B98422CD0B0F1804F2BD0A3F5943323
:10DBF800984229D003F58063984227D003F5006343
:10DC0800984225D003F58063984223D003F59033DA
:10DC1800984221D003F5406398421FD003F58063F2
:10DC2800984207D003F58063984208BF092202D0C2
:10DC38000020704708220B4B03EBC203187970478A
:10DC48000022F8E70122F6E70222F4E70322F2E7CE
:10DC58000422F0E70522EEE70622ECE70722EAE7CE
:10DC6800002C0140B8DB02082DE9F04F013085B0E7
:10DC7800C3B203930B4602918B4C8C4E002B00F0E1
:10DC88009A8032208A4D8B4FDFF82C9216F036FEA0
:10DC98004FF4FA7A4FF0100C4FF47A70D9F8043038
:10DCA800C3F30803002B40F0DE80EFF31183002B51
:10DCB80040F0D9802968A26800BF2B689942F9D141
:10DCC800D7F800E000FB0EF39B1AB3FBFEF300FB52
:10DCD80001314FF0010E0191D9F80430C3F3080364
:10DCE800002B40F08780EFF31183002B40F08280F7
:10DCF8002B68A16800BF2A689342F9D1D7F800B011
:10DD080000FB0BF2521AB2FBFBF200FB0323019A51
:10DD18009B1AB3F57A7FDFD3BAF1010ABED1039B10
:10DD2800002B40F0BD804FF47A7ADFF88C91504692
:10DD38004FF0100CD9F80430C3F30803002B75D149
:10DD4800EFF31183002B71D12968A26800BF2B68FB
:10DD58009942F9D1D7F800E000FB0EF39B1AB3FB08
:10DD6800FEF300FB01314FF0010E0191D9F80430A8
:10DD7800C3F3080313BBEFF31183FBB92B68A16846
:10DD880000BF2A689342F9D1D7F800B000FB0BF224
:10DD9800521AB2FBFBF200FB0323019A9B1AB3F55C
:10DDA8007A7FE3D3BAF1010AC4D1029B013B029303
:10DDB800002B7FF466AF05B0BDE8F08FEFF3118854
:10DDC8008CF31288A1682368DB0344BFC6F800E01F
:10DDD800A1682B6832685FFA88F888F31188D7F849
:10DDE80000801A4400FB08F35B1AB3FBF8F300FB4E
:10DDF8000233D2E7EFF311888CF31288A168236805
:10DE0800DB0344BFC6F800E0A1682B6832685FFAFC
:10DE180088F888F31188D7F800801A4400FB08F3C3
:10DE28005B1AB3FBF8F300FB023370E7EFF31182E0
:10DE38008CF31288D4F808E02368D90303D50123AA
:10DE48003360D4F808E02B683168D2B282F31188C5
:10DE58003A68194400FB02F3A3EB0E03B3FBF2F399
:10DE680000FB01317FE7EFF311828CF31288D4F8BD
:10DE780008E02368D90303D501233360D4F808E008
:10DE88002B683168D2B282F311883A68194400FBD2
:10DE980002F3A3EB0E03B3FBF2F300FB013118E727
:10DEA800184616F0D1FB3EE710E000E0AC56002023
:10DEB800B0560020B456002000ED00E0204B5B680F
:10DEC800C3F3080330B4BBB9EFF31183A3B91D4BF7
:10DED8001D4C1868A16800BF1A689042F9D11B4B05
:10DEE8001C684FF47A7202FB04F3591AB1FBF4F17F
:10DEF80030BC02FB00107047EFF31182102383F34C
:10DF0800128811498C680B6813F4803F104B02D0BB
:10DF1800012018608C680B49D2B20D68186882F32A
:10DF280011880A4B19684FF47A72284402FB01F3EE
:10DF38001B1B30BCB3FBF1F302FB0030704700BF82
:10DF480000ED00E0B056002010E000E0B4560020DC
:10DF5800AC5600202DE9F84F8046FFF7AFFF254E5D
:10DF68002549DFF8A0E0254A254D844610274FF4BF
:10DF78007A740120DEF80430C3F30803D3B9EFF351
:10DF88001183BBB90B68D2F808A000BFD1F8009084
:10DF98004B45F7D1D6F800B004FB0BF9A9EB0A09F9
:10DFA800B9FBFBF904FB0393A3EB0C034345E1D353
:10DFB800BDE8F88FEFF3118A87F31288D2F808B01A
:10DFC8001368DB0344BF2860D2F808B00B68D5F8A3
:10DFD80000905FFA8AFA8AF31188D6F800A099446B
:10DFE80004FB0AF3A3EB0B03B3FBFAF304FB0933BB
:10DFF800DAE700BFB4560020B056002010E000E079
:10E00800AC56002000ED00E02DE9F04FDFF830C1FC
:10E01800474A4849484E494D8046102718F1FF386D
:10E02800C0F08480DCF80430C3F30803002B5CD113
:10E03800EFF31183002B58D10B68946800BF086870
:10E048008342F9D1D6F800904FF47A7000FB09FEAC
:10E05800AEEB040EBEFBF9FE00FB03EEDCF8043069
:10E06800C3F308034FF47A740120FBB9EFF311836B
:10E07800E3B90B68D2F808A000BFD1F800904B456F
:10E08800F7D1D6F800B004FB0BF9A9EB0A09B9FBE4
:10E09800FBF904FB0393A3EB0E03B3F57A7FBDD220
:10E0A800DCF80430C3F30803002BDFD0EFF3118A48
:10E0B80087F31288D2F808B01368DB0344BF2860DE
:10E0C800D2F808B00B68D5F800905FFA8AFA8AF39C
:10E0D8001188D6F800A0994404FB0AF3A3EB0B03BC
:10E0E800B3FBFAF304FB0933D5E7EFF3118487F3A5
:10E0F8001288D2F808901368D80303D501232B603F
:10E10800D2F808900B682868E4B284F31188D6F82E
:10E1180000A04FF47A7400EB030E04FB0AF3A3EBA0
:10E128000903B3FBFAF304FB0E3E97E7BDE8F08F53
:10E1380010E000E0B0560020B4560020AC56002095
:10E1480000ED00E030B4EFF31183102282F312885F
:10E158000649074C0A680748013200250A6025600D
:10E16800DBB2026883F3118830BC7047B0560020D8
:10E17800AC56002010E000E01D4B70B59C68E36CC5
:10E18800226BDD69C2B1636B2BB12B0702D5E36C3F
:10E1980008221A6270BD2A06F7D5A26A616A8A4205
:10E1A8001FD0511CA069A162825C2069E66C814283
:10E1B8003285EAD3A362E8E7A906E4D5E26A1AB190
:10E1C800988C80B29047DEE7E1699B8C6069DBB28E
:10E1D8004E1CE6614354E169E368994228BFE26155
:10E1E800D1E7E26C136823F080031360CDE700BF2A
:10E1F8006C2C002070B4EFF31186502383F312883F
:10E20800436B1A68D20720D45D686DB9446A826A84
:10E21800944217D081691144D9600ED9A21A5A6064
:10E228008462002280F850201A6842F00102F1B29C
:10E238001A6081F3118870BC704701698A1A5A60A4
:10E248008562EEE7012380F85030F1B281F311883E
:10E2580070BC704703682DE9F041DF691FB13B4688
:10E26800BDE8F0411847002A164611DD04460D4660
:10E278000E4400E023689B68204698470028F9D0A0
:10E28800236815F8011B1B6820469847AE42F1D158
:10E29800BDE8F08103689B69184700BF03685B69A4
:10E2A800184700BF0368DB68184700BF03685B684E
:10E2B800184700BF03681B68184700BF10B40B4B12
:10E2C8000B4A1C7801238340234052F8200031B9BF
:10E2D800B3FA83F149095DF8044BF5F7EABA191C5A
:10E2E80018BF01215DF8044BF5F7E3BA9C560020EE
:10E2F800A056002008B501210220FFF7DFFF094BD7
:10E308001B7803F00503052B08D000210120FFF737
:10E31800D5FF00210846FFF7D1FFFEE704F05AF9C0
:10E32800F3E700BF0C2A0020054B53F8203033B127
:10E338001A689B88918A0B4218BF1B049361704727
:10E34800A05600202DE9F04F734B744A1C7893B007
:10E3580000F59C412031814607911160002C00F0A6
:10E36800C4846F4A1268904240F2DC816D4A6E495B
:10E378001768DFF8ECB16D4D0492013C03911C70F5
:10E3880007F48057002F40F0DA81694B05931E7817
:10E3980006F00106039B5B7D002B40F07B84049B09
:10E3A8001B68190400F1CB86624B9945AB7800F2E3
:10E3B8005883002B40F05883049BD3F8009019F43D
:10E3C800805A40F03984039BBBF906805B8B9845E3
:10E3D800B4BF4FF000084FF00108574B1B6813F00B
:10E3E800805300F0E081002E00F0E1810399534A48
:10E3F800498C92ED037A07EE901AF8EEE77AB4EEBC
:10E40800E77AF1EE10FA80F25287B8F1000F40F087
:10E41800D6814B4C94F8A020002A40F0D08149497D
:10E42800494A086890F82D000021116051609160F8
:10E43800002840F0C481454A1070002E40F0C58184
:10E44800434B1A78002A50D10399BBF900E04E8B50
:10E45800898BBBF902007645B4BF8024002444F0C0
:10E4680040037145D8BF23469B0843F08004864289
:10E47800B8BF234643F040048142D8BF1C46BBF9CD
:10E4880004E0BBF90600A40844F080037645B8BF51
:10E498001C4644F040037145D8BF23469B0843F00F
:10E4A800800E274CB042C8BF734643F0400E94F824
:10E4B800A2608842B8BF73469E4201F09D80A4F8CE
:10E4C800A42084F8A620234984F8A2300E78002ED0
:10E4D80000F0F2875F2B01F045806F2B00F03F873B
:10E4E800059B1B78DE0740F10187049B1A4A1B68CD
:10E4F800069203F00403002B40F0398410AF174C48
:10E5080000237B6004F15009109340F6330A4FF062
:10E51800190840F2833628E0985400208C530020D4
:10E52800945400206C490020B84E0020BC3E0020C6
:10E53800FE560020404B4C00C8370020CC3C002041
:10E548004C230020183F0020EC3500200823002031
:10E558009C340020071C0020705100204038002007
:10E568004045002004344C4520D0A278E3789A42F4
:10E5780018FB0260F6D26178043118FB03623BF99C
:10E5880011305345A8BF5346B3F5617FB8BF4FF468
:10E5980061739842E6DA9A42E4DB21782429E1D8CB
:10E5A80038460434F6F730F84C45DED1B34BB44A5C
:10E5B8001B7897E8030082E80300002B00F0FB8338
:10E5C8000121AF48F6F72FF8002840F04981EB7891
:10E5D800002B40F04581AB4FA9483C8824F001044A
:10E5E800A4B202213C80F6F71EF8002800F0418111
:10E5F800A20740F1C986DFF8E0A2A34B9AF8001001
:10E6080058680393A30708BF81F00201C1F34001D2
:10E61800F5F74FF924219A48F6F705F830B9059A25
:10E6280013785E0744BF23F004031370069B1B682E
:10E6380013F00A0F40F056813C8891480C21F5F7F9
:10E64800F2FF002800F07381904B1B7844F480742B
:10E65800082B3C8000F074810E2B00F07181049B24
:10E668001B685C0544D58A4B1B79002B00F0DA80C7
:10E6780014218348F5F7D7FF002840F0D88013F01D
:10E68800C9FF012010F0AEFC90B3DFF850820024DF
:10E698004FF0CC0902E0DCB2022C29D809FB04F6C1
:10E6A800631C58F80650002DF5D1C378794A90F9C3
:10E6B800020052F8233001950322009201212A46D4
:10E6C80010F0A0FA034604EB440000EB001004939A
:10E6D80053B1294608EB8000CC221DF09EF9049B1B
:10E6E80048F806300134E4B217F06EFD0028D3D1A3
:10E6F800059B1B78D80740F127816749674A0123A2
:10E708000B701370039B9AF80010186801F0010150
:10E71800F5F7CFF8069B1B685B0700F1858113B0FE
:10E72800BDE8F08F5E4B5F4A1F68049307F480577B
:10E738000392DFF8ACB15C4D002F3FF426AE002108
:10E748004F48F5F770FF00287FF41FAE574B05932D
:10E7580019461B7813F001063FF41CAE544A96780C
:10E7680003F0FE030B70002E3FF414AE514C2278D8
:10E778000B2A0DD80121914040F603060E4041F0C6
:10E78800678211F4C06F03D0093A012A41F21B8352
:10E79800DFF83CA1484ADAF8001051600B2203F078
:10E7A80001062270F6E519F4800F7FF41CAE434C85
:10E7B800002284F8A020B8F1000F3FF430AE404AA0
:10E7C80001211170002E3FF43BAE19F0100F3FF4F9
:10E7D80037AE3C4A1278D2063FF532AEBAF1000F96
:10E7E8007FF42EAE002B7FF42BAE19F4800F7FF44C
:10E7F80027AE354B1B78002B01F06382334B9B7897
:10E80800B8F1000F41F0EF823BB1314A314B126849
:10E818001B689B1A002BC1F27E82284C012384F8C6
:10E82800A1300DE6059B1B78D9077FF528AF4FF47B
:10E838000F7011F077F900283FF45AAF10F0CAF9B9
:10E848004FF40F7011F004F900283FF451AF10F0A5
:10E85800C1F94FF40F7011F0FBF80028EED147E72B
:10E86800069B1B6899077FF5B6AE064F3C8844F0B7
:10E87800010424F00204A4B23C80BCE6F13E00206E
:10E88800C837002072500020A05600203C380020D5
:10E89800BC3C00206CDC0208FF5600204C22002003
:10E8A8006C490020B84E0020BC3E0020FE560020D7
:10E8B800703400206D340020D43700204C23002011
:10E8C80008230020C4320020071C00201C38002028
:10E8D800B0560020F83900209C560020D84100206E
:10E8E800404500200621AE48F5F79DFE3C880028EB
:10E8F80000F0BC84650640F1BA850721A848F5F701
:10E9080092FE00283FF499AEA64BA74AB3F904300B
:10E91800A6493C8882FB0302DB17C3EBA2030B80EA
:10E928009F480C21F5F77FFE00287FF48DAEA04BA1
:10E938001B7824F48074A4B2082B3C807FF48CAE3E
:10E9480024F040043C808AE69A4B93F80090B9F191
:10E95800000F5FD1DFF8A882974E18F8030C3578BE
:10E968004146A8F1030418F001FC002800F0908348
:10E97800002D40F0E28304F10801607918F0F6FBFD
:10E98800002841F0F2808D49A07A18F0EFFB0028AA
:10E9980000F09183022D41F0EC808949E07B18F06A
:10E9A800E5FB002841F0E9808649207D18F0DEFB70
:10E9B800002800F09183042D41F0B6808249607EE2
:10E9C80018F0D4FB002841F0C8808049A07F18F0D7
:10E9D800CDFB002800F09183062D41F0C2807C49D0
:10E9E80094F8230018F0C2FB002840F0AE8679495D
:10E9F80094F8280018F0BAFB002800F09183082D3D
:10EA080040F08D86744994F82D0018F0AFFB00286B
:10EA180040F09183714B01221A7018F02AFE069B70
:10EA28001B685B077FF57BAE032018F0C9FB002845
:10EA380000F0DD853B8813F008047FF470AE0820F1
:10EA480010F0BCFB6648674D6749684A684BBBF8DD
:10EA5800066000682E80086014601C6013B0BDE872
:10EA6800F08F0BB90123AB701B2018F0A9FBDFF85E
:10EA7800948195F8217095F820305E4C8146B24615
:10EA8800052B00F20181DFE813F0BF007F000600CC
:10EA9800FB00FD00F100012F04BF052385F820309D
:10EAA800BAF1000F12D0039BB8F80000B3F91810A0
:10EAB8000022134661F30F0361F30F0260F31F4254
:10EAC80061F31F43CBF80420CBF800304A4E6A6943
:10EAD80033689A4280F0BB8447F230520323EA61DC
:10EAE80085F82030238843F0020323800BF0E0FAF6
:10EAF8003268EB6913440422AB6185F82020012FAA
:10EB080040F0BB853368AA699A4280F0BD803B4BD0
:10EB1800187820B918F054FB002840F0B5802388F5
:10EB280023F0020323803268B8F80230642101FB25
:10EB380003234FF4806000222B6185F82020EA70BF
:10EB480010F034FB95F820309AE718F065FB01289F
:10EB580007D1294EB8F802303268642101FB03233B
:10EB68002B61B9F1000F03D098F80630002B7FD144
:10EB7800012F00F08980204E2A6933689A42C0F03C
:10EB88008685012385F82030012F6FD098F807304B
:10EB9800012B00F0A0800CF00BFD95F820306FE7FA
:10EBA800C8370020883F002067666666102200206C
:10EBB8003C380020FF56002080000020693B0020E0
:10EBC8006E3B0020733B0020783B00207D3B0020FB
:10EBD800823B0020873B00208C3B00204C220020F9
:10EBE8002C2200201C220020282200202022002085
:10EBF80018220020E03E0020B0560020071C00200C
:10EC08005F3B0020A03B0020BAF1000F9DD14FF4DC
:10EC18008060B9F1000F00F0F18210F0CFFA059B87
:10EC28001E7800232B61049BD3F8009019F4805AB6
:10EC380006F001063FF4C7AB1D219948F5F7F3FC30
:10EC480000287FF4C0AB974A039BD2881B8BBBF983
:10EC58000680991A884540F3248513449845B4BF23
:10EC68004FF000084FF00108FFF7B7BB8E4E5AE788
:10EC78000CF09EFC03224FF47A7385F82020EB6198
:10EC8800894E2FE7884E3AE7059B1E7806F0010665
:10EC9800FFF792BB039A013BD27D3BF91330002A60
:10ECA80040F0EA82A3F57A73B3F57A7FA8BF4FF4F0
:10ECB8007A7323EAE37307EE903A9FED7C7AF8EED5
:10ECC800E77A67EE877A7A4AFCEEE77A17EE903AA7
:10ECD8001380FFF769BB0CF06BFC032240F6B833D6
:10ECE80085F82020EB61704EFCE6724F3B78002BD4
:10ECF80000F0E086704BDFF8D481DFF8D4B1DFF89C
:10ED0800D4A1039345465E46049099460EE019F84F
:10ED180004109847032C28DC88B93B782AF8020F9E
:10ED280001349C4205F1040580F2DA80072CE1B237
:10ED38003046DBF80430EADD984700B2EDE738F8F2
:10ED480024206B88801A4FF47A719B1A01FB00F01B
:10ED580040F6CA0290FBF3F00844904240F2EE23DA
:10ED6800A8BF10469842B8BF184600B2D5E7534C22
:10ED780094F8AA3053B1059B1B78D90706D5039B95
:10ED8800BBF906205B8B9A4200F39C84112144480E
:10ED9800F5F749FC002800F0788294F8AE302BB9DA
:10EDA80094F8A83013B93223A4F8AC30012384F8BE
:10EDB800AE30FFF7A3BBDFF820A1DFF820813F4C7E
:10EDC8001F460AF15A064FF0010951461AF8010C7C
:10EDD80018F0CCF9F8B19AF804009AF802309AF8C9
:10EDE80003E000EB400104EB8101013BD1F8B420C2
:10EDF80003EB4303434493420DD094F8E02081F899
:10EE0800B0E009FA00F022EA0000C1F8B430C1F815
:10EE1800B87084F8E0000AF1060AB245D5D128494D
:10EE2800214A284B284C09681B78D2F800A0089181
:10EE38000793A4F1B0090026636853B31F7847B35A
:10EE4800A168AAEB010100290ADB99F8E01001206A
:10EE5800B04021EA00010AF5FA7089F8E010A060D4
:10EE6800079AB2B1217858780431C9B2002840F025
:10EE78002482039A3BF91110108B00F1C80E7145DA
:10EE880040F3D28399F8E0109B783141CA0740F1EA
:10EE980044840136042E04F10C04CDD1FFF790BB55
:10EEA800C837002090270020B0560020AAF1823FE2
:10EEB80070500020EC540020B84E00204C23002055
:10EEC800045D0020B03E0020FC23002020560020D6
:10EED800903F00204A230020763A0020F4BE020822
:10EEE800DDF81090C74A04921146C74A0968A2FB88
:10EEF800092A42F201020A404FEA9A1A059200F0E2
:10EF0800C081C24DC248C34CC34A95F800E000789E
:10EF180084F800E01070BEF1000F04D0BE4A92F8E9
:10EF280000E08EF0010EBD4C0F2084F82400002B69
:10EF380000F0A282BA4B039E0C931B78B6F826C049
:10EF48000B931D463B78B78C039EB64A368B0E96BC
:10EF58002E46A2FB0552520802EB4202B21AD2B266
:10EF6800CDF824C001F48051089294F82580DFF888
:10EF7800C8B2DFF8F0C20A900AF5967276460F9189
:10EF880004F1280500200692CDF83490A646002EFC
:10EF980000F0FF813EF910201FFA82F9B9454FEAC7
:10EFA800400103D3099CA14540F237825CF8202038
:10EFB800924580F0F7813BF90120059C002C40F038
:10EFC8000B82013098422BF8012005F10605DEDBA3
:10EFD8000A99954A8EF824100F290CBF01210021A7
:10EFE800DDF834908EF82580117000F04C828F4D3A
:10EFF8008F4EDFF874A23488DAF80000A9686A68CE
:10F00800E86044F00404401A9042814F3480824CF6
:10F018004FF0010188BF00223970217088BF85F840
:10F028002120002B00F04382049A03991768814E2F
:10F03800B1F824C0B1F818E07F4817F48057344677
:10F0480040F0538239460EE0627802EB820202EB0E
:10F05800820202F2EE2292B20131994220F8022B8A
:10F0680004F102040ED016F81120002A00F0D9810C
:10F07800022AE9D00131028820F8022B994204F1D2
:10F088000204F0D10C9A137801331370FFF77AB9A0
:10F0980008F10501607918F069F800283FF473ACAD
:10F0A800012D40F0628504F10D01A07A18F05EF898
:10F0B800002840F05E856149E07B18F057F8002889
:10F0C8003FF472AC032D40F058855D49207D18F05F
:10F0D8004DF8002840F028855A49607E18F046F817
:10F0E80000283FF472AC052D40F037855649A07FC3
:10F0F80018F03CF8002840F03485544994F823006F
:10F1080018F034F800283FF472AC072D40F01D8346
:10F118004F4994F8280018F029F8002840F0FF8299
:10F128004C4994F82D0018F021F800283FF472ACEF
:10F13800092D3FF46FAC4FF009094B46F2E2374C0A
:10F14800D4F88830A9EB0303002BFFF62DA9424A17
:10F1580094F88C30517C079AC4F8882001333F4AD0
:10F16800039F32F81120B97D03F00F0384F88C3027
:10F17800234492B292FBF1F283F8902094F8901015
:10F1880094F8912094F8923094F89C000A4494F8EA
:10F198009310134494F89420194494F895300A4431
:10F1A80094F89610134494F89720194494F89830DA
:10F1B8000A4494F89910134494F89A20194494F83E
:10F1C8009B300A44134494F89D1094F89F201844E7
:10F1D80094F89E3001440B441A4442F30B12642AFB
:10F1E800F97DA8BF642213B209B1C2F1640307EE26
:10F1F800903A9FED1B7AF8EEE77A62E50FF0D6FFBA
:10F208000DE500BF6C490020D34D62106853002003
:10F2180044140020B03E0020451400204C23002058
:10F2280099540020ABAAAAAAB63F0020BC3E0020F1
:10F23800E03E002054560020404500206E3B002050
:10F24800733B0020783B00207D3B0020823B002060
:10F25800873B00208C3B00207856002094560020E5
:10F2680014AE23419C540020B056002024F04004E2
:10F27800A4B23C80FFF741BBC3F53B6308331BB224
:10F2880010E5A94A92F800E045E694F8A830002B6A
:10F298003FF434A9059B1B7813F001037FF42EA9D2
:10F2A800012284F8A83084F8A920FFF727B99F4CD9
:10F2B800012284F8A020FFF782BA012800F0CA834F
:10F2C80099F8E0200123B34001361343042E89F84E
:10F2D800E03004F10C047FF4AFADFFF771B9059B82
:10F2E800934A1B781060DB0700F1FA8194F8A610A6
:10F2F80000297FF4FAA8B4F9A430322B7FF7F5A8D7
:10F3080094F8A2200120572A84F8A60000F0F1837F
:10F31800049B1B6813F0040302D05A2A00F0E0840F
:10F328005D2A00F07C845B2A00F083845E2A00F06A
:10F338008384562A00F0E384972A00F0B684A72A2B
:10F3480040F038847B49049B0A781B6842F0040229
:10F358000A70794A069203F00403FFF7CCB8B2F5B5
:10F36800FA7FFFF6C2A894F8A620002A7FF4BDA869
:10F37800059B1B780121DF0784F8A61000F1108493
:10F388000AF008FAFFF7B1B844F002043C80FFF72E
:10F3980032B9002F3FD05CF8202092454FEA400157
:10F3A800FFF409AE654A654C525C04EB0109002A7A
:10F3B80000F08F80022A47D199F8012002EB8202DF
:10F3C80002EB820202F2EE2292B2032833DD059CA0
:10F3D80012B2002C3FF4F5AD089C25F81420B8F1C2
:10F3E800000F03D10B9C022C7FF6EBAD6A88B5F8B1
:10F3F8000090B5F804804A449044514A0FFA88F8BE
:10F4080082FB08424F4CA2EBE87224F8018012B24A
:10F418004FF00108D5E53A464100069C4CF82040DB
:10F42800CBE5CAB2022A04D9032A7FF423AE624686
:10F4380012E6724610E6012404FA00F90A9C24EA4E
:10F44800090412B20A94B8E53BF80120BDE73E4B27
:10F458001B78002B7FF440ABBAF1000F3FF43CABB4
:10F46800012F7FF411AC95F82030FFF709BB44F069
:10F4780040043C80FFF741BA3449354A0C91DFF823
:10F48800E0B0012111701B2132480593F5F7CBF844
:10F49800059B00287FF4ABAD2F4DDFF8C0A0EA68CC
:10F4A800DAF80030AB609B1AC82B00F21483049B77
:10F4B8001F6807F48057E5E531462648F5F7B3F8A5
:10F4C80000283FF40CAF84F8A7600AF063F9FFF74F
:10F4D80007B8C2B2022A40F2BB82032AB4D10E9AFC
:10F4E8000F9C002C08BF3A466FE700210FE06278B6
:10F4F80002EB820202EB820202F2EE2292B20131A8
:10F50800994220F8022B04F102043FF4BBAD16F82F
:10F5180011201AB1022AEAD00288F0E7CAB2032AF7
:10F52800FAD87246EBE700BFB03E00204C2300201B
:10F53800FC390020C43200207051002054560020AD
:10F5480056555555BC230020F82200209954002018
:10F55800B63F0020C8370020BC3E0020B05600202F
:10F5680040450020B2F5FA7FFEF6BFAF94F8A6300A
:10F57800002B7EF4BAAF059E3378012113EA01000F
:10F5880084F8A61000F09A82AE4A927823F001031C
:10F598003370002A3EF4A9AFAB4C23780B2B18D854
:10F5A80001FA03F240F603010A427EF49EAF12F418
:10F5B800C06F0ED0093B012B0BD8452018F0DAFAA2
:10F5C800FF2018F0D7FAA14818F0C0FA002018F068
:10F5D800D1FA9F499F4A049B09681B6851600B2216
:10F5E80022709D4A069203F00403FEF784BF0820A8
:10F5F8000FF0DCFDFFF793B8984A99491068B4F901
:10F60800A420C66981FB06018911F617701A00F556
:10F61800FF407F3082423EF756AF891B0A4412B240
:10F62800A4F8A420FEF74FBFC83881423DDA99F804
:10F63800E0109B783141C8073FF52BACC3F10008B7
:10F64800791E162900F2BF80DFE811F0B601CA0161
:10F658009C011401DE01EF018901760161014C0171
:10F668003701BD0014012401EF0189017601E8008A
:10F67800D400C000AD009700830005993268EB699B
:10F688000E781344AB6106F00106FEF795BE0BF049
:10F698008FFF032240F6B83385F82020EB61FFF78F
:10F6A80021BA4FF00108FEF798BE99F8E030012220
:10F6B800B24023EA02030AF5FA7289F8E030A26040
:10F6C800FFF7E7BB00216748F4F7ADFF00287FF498
:10F6D8005DAB322384F8AA00A4F8AC30FFF756BB20
:10F6E800614B1B78002B3EF400AFEB78002B7EF4C7
:10F6F800FCAE94F8A7300133DBB2032B84F8A730B3
:10F708007EF6F3AE594B5B781BB9B8F1000F7EF467
:10F71800ECAE0AF0CDFCFEF7E3BE984690E74FF05A
:10F7280008094B4603EB83031C4486F80090A17834
:10F73800607817F0C7F9059B4D4A1B7801211170B5
:10F74800DA077FF56AA9FEF7DDBF4FF007094B46D8
:10F75800E8E7D9F8E4003B4B90F836109A78414432
:10F768006429A8BF642121EAE17180F83610002AD3
:10F7780040F04B8302F0EAFCA2E5D9F8E400314BF3
:10F7880090F837109A784144FE29A8BFFE2121EA53
:10F79800E17180F83710002AECD0162017F06EFDC2
:10F7A800D9F8E400E6E7089A264B51784144B1F5C8
:10F7B800967FA8BF4FF4967121EAE17151709B784A
:10F7C800002B40F0B082D9F8E400D3E7D9F8E40080
:10F7D80081781C4B4144C829A8BFC82121EAE1719E
:10F7E80081709B78002BC5D0142017F047FDD9F8FD
:10F7F800E400BFE7D9F8E4004178124B4144C82936
:10F80800A8BFC82121EAE17141709B78002BB1D0D3
:10F81800132017F033FDD9F8E400ABE7D9F8E4007A
:10F828000178084B4144C829A8BFC82121EAE171E1
:10F8380001709B78002B9DD0122017F01FFDD9F87E
:10F84800E40097E7703400206D34002004E20208D9
:10F85800B0560020D4370020705100201C530020DF
:10F86800D34D6210C8370020B03E00201C3800205D
:10F878004C220020089AC34B917998784144642916
:10F88800A8BF642121EAE1719171002840F05D82EE
:10F898000D2F98D00898BB4B41799A784144642938
:10F8A800A8BF642121EAE1714171002A8BD00E20A2
:10F8B80017F0E4FCD9F8E4005CE7D9F8E400B14BB0
:10F8C800017A9A784144C829A8BFC82121EAE17180
:10F8D8000172002A3FF44EAF0B2017F0CFFCD9F885
:10F8E800E40047E7D9F8E400A64BC1799A78414487
:10F8F800C829A8BFC82121EAE171C171002A3FF4D3
:10F9080039AF0A2017F0BAFCD9F8E40032E7D9F881
:10F91800E4009C4B81799A784144C829A8BFC82142
:10F9280021EAE1718171002A3FF424AF092017F020
:10F93800A5FCD9F8E4001DE7D9F8E400914B41791A
:10F948009B784144C829A8BFC82121EAE1714171C7
:10F95800002B40F0F481112F7FF43AAF0AE7D9F871
:10F96800E400884B01799B784144C829A8BFC82185
:10F9780021EAE1710171002B40F0DB81102F7FF447
:10F988003BAFF7E6089A11798844B8F1640FA8BF2D
:10F998004FF0640828EAE87882F8048017F088FCB9
:10F9A800784B9B78002B3FF40EAF0320414617F0AD
:10F9B80065FCD9F8E400DDE6089A724B11784144F9
:10F9C800FA29A8BFFA2121EAE17111709B78002B6E
:10F9D8003FF4F9AE012017F051FCD9F8E400C9E66C
:10F9E800089A684B917841446429A8BF642121EAA8
:10F9F800E17191709B78002B3FF4E5AE022017F07F
:10FA08003DFCD9F8E400B5E608985E4BC1799A78D0
:10FA1800414481F30801C171002A3FF4D4AE0520A6
:10FA280017F02CFCD9F8E400A4E6D9F8E400554B0B
:10FA3800C1789B784144C829A8BFC82121EAE1714F
:10FA4800C170002B40F0E5810F2F7FF4E9AE91E6FD
:10FA58000E9ABAE43BF91110987840F633039942AC
:10FA6800A8BF1946B1F5617FB8BF4FF461710C2F7B
:10FA7800A1F561714FF4966393FBF0F391FBF3F1F9
:10FA880056D0182F7FF41CACD9F8E430C9B2C82975
:10FA980093F817E00846A8BFC82086453FF410AC85
:10FAA800384AD8759278002A3FF40AAC384617F0DD
:10FAB800E5FB05E4344A0392FFF714BA049B84F883
:10FAC800A600FA3A1B68A4F8A420304A069203F06C
:10FAD8000403FEF710BD2E4A049B1F68138823F009
:10FAE80004031380012307F4805785F82130FFF7BA
:10FAF800C9BA264A274B069210461A6826494FF477
:10FB08007A73B3FBF2F3C3EB431203EB820302688D
:10FB1800DB005007A1F8B43000F19180049B1B680A
:10FB280003F00403FEF7E7BC4FF004094B46F9E580
:10FB38001A4B5B785FFA81F843453FF4C1AB404606
:10FB480004F0E8FD0F4B9B78002B3FF4B9AB41461E
:10FB5800384617F093FBFFF7B3BB4FF005094B4648
:10FB6800E0E54FF006094B46DCE54FF001094B464E
:10FB7800D8E54FF002094B46D4E54FF003094B4650
:10FB8800D0E500BF70340020B84E0020705100202E
:10FB9800E03E00205C490020D84600200C3F0020B1
:10FBA800049BA4491B680A60A34A069203F0040355
:10FBB800FEF7A1BC0021BB2A109173D0B72A6DD0E3
:10FBC800BE2A69D0BD2A46D0792A00F0F5807A2A63
:10FBD80000F0EB809E2A00F0E2809D2A00F0D88099
:10FBE800AE2A00F0CE80AD2A00F0C480EF2A00F0E3
:10FBF800BE80FD2A00F0AD80FB2A00F00381FE2ABA
:10FC080000F0FD80F72A00F00A817B2A7EF46DACB3
:10FC18004FF4FA61022004F0A7FCFEF766BC874A9D
:10FC280000218748874C0260834A21700692FEF7BC
:10FC380062BC854A0121F4E7844A0221F1E7049B6A
:10FC4800834A1B680A21118003F00403FEF753BCA2
:10FC58000646FEF79FBB4FF6FE737E4A76489689A6
:10FC68000690D089334401449381D18113F0C4FEB6
:10FC7800F4F7A0F813F0A8FEFDF7F8F8049BB4F821
:10FC8800A4201B68FA3A0021A4F8A42003F0040376
:10FC980084F8A610FEF72FBC0223DEE70B464FF6CA
:10FCA800FE71DAE70B460221D7E7049B6A4A1B6814
:10FCB8004FF4C8711180604A069203F00403FEF7FE
:10FCC8001ABCB8F1000F3EF4A8AD644C94F8A1300A
:10FCD800002B3EF4B5AB002384F8A130FEF7B0BB8F
:10FCE80094F8A820002A40F09D8094F8AA20524950
:10FCF800069182F0010284F8AA20FEF7FCBB13F0FB
:10FD08007BFEF4F757F813F05FFEFDF7AFF894F8B1
:10FD1800A220FFF711BB514C0AF0CAF9002384F85E
:10FD2800A130FEF78DBB152017F0A8FAD9F8E4002A
:10FD380020E5102017F0A2FAD9F8E4001EE61120F9
:10FD480017F09CFAD9F8E40005E60D2017F096FAAA
:10FD58009EE50021012004F007FCB4F8A43000223D
:10FD6800963BA4F8A43084F8A620FEF7BEBB002179
:10FD78000846F0E7FF21002019F0CCFB94F8A220F8
:10FD880034E70121002019F0C5FB94F8A2202AE7E6
:10FD98000021FF2019F0BEFB94F8A22020E70120E3
:10FDA80019F0B8FB94F8A22017E72D4A137A43F00C
:10FDB80001031372FEF799BB294A137A23F0010352
:10FDC8001372FEF792BB452017F0D4FEFF2017F000
:10FDD800D1FE244817F0BAFE304617F0CBFE059B3B
:10FDE8001B78FEF7D5BC002B3FF46FAF1E491F4AA6
:10FDF80009684FF47A7000FB0313136065E700216C
:10FE08000320A8E700210220A5E7172017F036FAFB
:10FE1800D9E40F2017F032FAD9F8E40014E60021EB
:10FE2800042098E7044A84F8A81084F8A9000692E8
:10FE3800FEF761BBFC3900207051002054330020CC
:10FE4800183F00200C3F0020A2330020F033002090
:10FE5800225D002000380020245D00204C23002073
:10FE68009C3F002004E20208B0560020F839002028
:10FE7800037903F00C03042B05D0082B0FD0C3B96A
:10FE8800B0F80B0070470C4BB0F80B001B7803EB75
:10FE98008302C3EBC20300EB430080B27047064BFA
:10FEA800B0F80B005B7803EB430300EB830080B2F0
:10FEB80070470020704700BF0C3F0020F3F7D7BE03
:10FEC80020B10078B0FA80F04009704701207047EF
:10FED80008B520211BF0D6FD0346184623B1027849
:10FEE800202A03F10103F8D008BD2DE9F8430D4697
:10FEF80016468146002440F634074FF01908484654
:10FF0800FFF7E6FF814690B119F02AFBB842A8BF77
:10FF18003846B0F5617FB8BF4FF46170A0F56170E5
:10FF280090FBF8F04CB92870337801333370013402
:10FF3800022CE4D14846BDE8F8836870F4E710B5B0
:10FF48000446B0F80900F3F7E5FE01462046FFF73E
:10FF58008FFF4B68184410BD38B505460C46FFF7AF
:10FF6800EEFF2B7903F00303012B00D001D20470BC
:10FF780038BD048038BD0FB413B5084C0849206853
:10FF880004AB53F8042B0193F4F763F92068F3F7F3
:10FF980061FE02B0BDE8104004B070478C28002014
:10FFA800C5FE00082DE9F0410379054603F030004D
:10FFB80020280E4614462BD12A4FDFF8B48000249F
:10FFC8006B799C4201DBBDE8F0812B7903F00303D8
:10FFD800022B11D0032B15D0012B14BF315D3157E3
:10FFE8003846FFF7C8FF6B79013B9C4202DA40466E
:08FFF80017F0ACF80134E3E757
:020000040801F1
:1000000036F814103846FFF7BAFFF0E736F9141047
:100010003846FFF7B4FFEAE703F00303012B06D0ED
:1000200008D2097848B1102813D0BDE8F08191F9C1
:100030000010F7E7B1F90010F4E70C48FFF79FFF55
:100040008CB1B5F90720B5F905100948BDE8F041B4
:1000500095E76A79074B53F83230BDE8F04153F821
:10006000210017F077B8BDE8F08100BF24E3020853
:100070006BE8020848CB0208EAE2020838B50D46F0
:100080000446FFF760FF2A4601462046BDE8384097
:100090008CE7024B01461868F3F7EDBD8C28002071
:1000A000014817F057B800BF760903082DE9F74F4C
:1000B000344C01F010038146884600252746009302
:1000C000314B1868F3F7CAFD94F804B00BF00C0339
:1000D0004B453FD10D2303FB0573B3F80900F3F73C
:1000E0001DFE06462046FFF7C7FE0BF00302012A5D
:1000F00082467168B06835D03CD211F80A2010F8F9
:100100000A00801A42424241009B03B112BB18F020
:10011000200F10D07AB90D2101FB05711B48096829
:100120000192FFF72CFF7168019A51442046FFF7B6
:100130003DFFFFF7B5FF0D2202FB05721448116861
:10014000FFF71DFFB168002251442046FFF72EFF44
:10015000FFF7A6FF0135C42D04F10D04B0D103B0A3
:10016000BDE8F08F11F90A2010F90A00811A4A42FD
:100170004A41C9E731F90A2030F90A00831A5A4284
:100180005A41C1E754C102088C280020ECE2020861
:10019000EDE2020810B5064C0B4602460549206800
:1001A000F4F75BF82068F3F759FDBDE8104077E7F6
:1001B0008C280020C5FE00080FB407B504A951F82B
:1001C000040B0191FFF7E6FF03B05DF804EB04B008
:1001D000704713460A4601460048EDE7F7E2020879
:1001E000F8B5037903F03003102B0AD0202B23D06D
:1001F0003BBBB0F90720B0F905101248BDE8F84044
:10020000DAE74579104E114816F0A4FF06EBC50356
:1002100000241F79BC4202D3BDE8F84040E714B186
:100220000B4816F097FF56F835300A4853F824105B
:10023000FFF7A5FE0134EDE741790748BDE8F84036
:10024000BAE7F8BD10E3020848CB020827E302082A
:10025000EAE2020874E7020837E302080CB407B5C3
:1002600010F0200009D069B92320FFF712FF05A97B
:1002700004980191FFF78EFF012003B05DF804EBB5
:1002800002B070470020F8E70CB4C30607B500D5EC
:1002900051B905A904980191FFF77CFF012003B033
:1002A0005DF804EB02B070470020F8E72DE9F04F4D
:1002B000DFF820B189B08046894616460D461446BF
:1002C0004FF0000A002E71D06A6863689A426BD1C1
:1002D000AF68A368FB1A5F425F4194F90B30049347
:1002E00094F90A300393B4F908300293B4F9063054
:1002F0000193B4F9043000935A46534639464046B8
:10030000FFF7ACFF95F90B30049395F90A3003938E
:10031000B5F908300293B5F906300193B5F9043008
:1003200000935A465346394640460AF1010AFFF700
:10033000ABFFBAF1080F05F10C0504F10C04C1D1B3
:100340000024DFF894A0254696B30027012303FA82
:1003500007FB325959F8043053403BEA030314BFFA
:100360000123002312EA0B0F079306D000972B46B8
:10037000524607994046FFF771FF59F804301BEACF
:10038000030F06D000972B46524607994046FFF7C9
:100390007BFF01370E2FD9D10135082D04F10C0454
:1003A000D2D109B0BDE8F08F002796E73746A9E71C
:1003B0003746012359F80420BB40134206D000976A
:1003C0002B46524601214046FFF75EFF01370E2FB4
:1003D000EFD1E1E748E3020860E302082DE9F04FBE
:1003E000DFF8E8A085B005468846144600270623B6
:1003F0007B4303930026039B334408EB030292F8EC
:10040000C0B0002C5ED02344524693F8C030019314
:10041000ABEB0300D0F1000949EB000900963B4625
:1004200049462846FFF71AFF8DE840083B465246EA
:10043000494628460136FFF727FF062EDBD1013754
:10044000062FD4D1DFF884B008F1E40A00261AF8A8
:10045000019B002C38D0A3195A4693F8E43001933D
:10046000A9EB03014F424F41009606233946284627
:10047000FFF7F4FE8DE840020623144A3946284669
:100480000136FFF701FF0B2EE1D198F8F0606CB157
:1004900094F8F0300193F21A54425441002300932F
:1004A0000A4A072321462846FFF7D8FE0023009377
:1004B00001960723054A21462846FFF7E5FE05B0C9
:1004C000BDE8F08FA146AFE72746D3E775E3020802
:1004D0002DE9FF47DFF86CA0814690460E46154691
:1004E0000027B8F1000F2AD02B8832889A4224D1F5
:1004F00074886A88A21A54425441EA780292AA780F
:100500000192009352463B4621464846FFF7A6FE1D
:10051000F3780293B378019336F8043B0093524684
:100520003B46214648460137FFF7AEFE102F05F146
:100530000405D6D104B0BDE8F0870024DDE74446C9
:10054000E6E700BF89E302082DE9F04FDFF8688095
:100550008FB007468A46164600240DF124095AF842
:1005600024300293494602A80FF048FC16B356F80F
:100570002430029D0393EB1A5D420DF1100B5D4197
:10058000594603A80FF03AFCCDF800B02346424686
:1005900029463846FFF762FE2346CDF800904246D2
:1005A000294638460134FFF76FFE202CD7D10FB013
:1005B000BDE8F08F3546EFE79BE302082DE9F347EE
:1005C000DFF868A081460F46904602260024B8F165
:1005D000000F28D037F8242038F824309A4238F811
:1005E00006201ED1BD5BA91A4D424D4101920093D8
:1005F0005246234629464846FFF730FEBB5B01932F
:1006000037F82430009352462346294648460134A1
:10061000FFF73AFE042C06F10406D8D102B0BDE87B
:10062000F0870025E2E74546E8E700BFA5E30208BA
:100630002DE9F04F2DED088BDFF80C9193B080463B
:1006400092460D461446002695ED008AB5EE408A86
:10065000F1EE10FA71D0D5ED019A95ED029AD5ED33
:10066000038ABAF1000F3FD094ED000A94ED01BA6D
:10067000D4ED02AA94ED03AAB4EE408AF1EE10FA8A
:1006800060D1F4EE4B9AF1EE10FA5BD1B4EE6A9AB7
:10069000F1EE10FA56D1F4EE4A8AF1EE10FA0CBFE0
:1006A000012700270FA8F3F7DDFCB0EE4B0A8346C5
:1006B0000CA8F3F7D7FCB0EE6A0A059009A8F3F787
:1006C000D1FCB0EE4A0A049006A8F3F7CBFC049ADA
:1006D000059B039002920193CDF800B033464A4641
:1006E00039464046FFF7BAFDB0EE480A0FA8F3F7C7
:1006F000B9FCB0EE690A07460CA8F3F7B3FCB0EEFC
:10070000490A834609A8F3F7ADFCB0EE680A0490E5
:1007100006A8F3F7A7FC049B039002938DE88008DA
:1007200033464A46002140460136FFF7ADFD082E0C
:1007300005F1100504F1100486D113B0BDEC088B4F
:10074000BDE8F08F0027ADE7B6E302082DE9F04FD2
:10075000834687B092460C46154600274FF019098C
:100760004FF46178BAF1000F4ED023782A78934283
:100770002B7947D160786978884243D1A078A978ED
:1007800088423FD1E078E97888423BD1217999428B
:1007900038D166796979711A4E424E410593EB78EA
:1007A0000493AB7819FB038303936B78019219FBD5
:1007B000038302936B790093144A3B4631465846B3
:1007C000FFF74CFD23790593E3780493A3780F4A50
:1007D00019FB03830393637819FB03830293237844
:1007E00001936379009331463B4658460137FFF742
:1007F0004BFD0F2F04F1060405F10605B2D107B039
:10080000BDE8F08F0026C9E75646DBE7CAE30208D9
:100810002DE9F04F89B002F11803DFF8E090364F70
:10082000DFF8DCB00793824690460C46164694F9F2
:10083000022099F90630934207D099F90E3093427D
:1008400003D099F9163093424BD1B8F1000F01D182
:1008500045462DE096F9023071799A42328849D1A5
:100860002088904246D1E578F078854242D12579BA
:10087000307985423ED1A579B07985423AD1657902
:10088000681A4542454157F821100491B17957F84B
:1008900021100391317957F821100291F1780092DB
:1008A00057F8211001915A4629465046FFF7D6FCC9
:1008B000627994F9023057F822200492A27957F80D
:1008C00022200392227957F822200292E27857F8E8
:1008D000222001922288009229465A465046FFF76C
:1008E000D3FC079B08369E4204F108049FD109B04F
:1008F000BDE8F08F0025C6E76CDC02089C4E0020A6
:10090000E8E302082DE9F04FDFF8B4A085B0814696
:1009100090460C46154600261927B8F1000F4CD01A
:1009200028782378834246D162786B789A4242D104
:10093000A278AB789A423ED1E178EB78CB1A594253
:1009400059418B4610F0E0F998B1EA784FF46171A3
:1009500017FB02120392AB7817FB031302936B7819
:100960000193037A00935246334659464846FFF7AF
:1009700075FC207810F0C8F998B1E2784FF46171F5
:1009800017FB02120392A37817FB031302936378F9
:100990000193037A00935246334659464846FFF77F
:1009A00073FC0136142E04F1040405F10405B4D1DE
:1009B00005B0BDE8F08F0021C3E7C346D9E700BF0B
:1009C00005E40208F7B50746FFF77EFA044630B1A2
:1009D000002224490120FFF795FF03B0F0BD3846FF
:1009E00018F0C2FD1328054635DC8600781C8DF80A
:1009F0000740FFF771FA1B4C074668B118F0B4FDC9
:100A0000C0B210F067F938B1037804F825309DF8CA
:100A1000073001338DF807303846FFF75DFA074697
:100A200050B118F0A1FD0D2806D8A31958709DF8F3
:100A3000073001338DF80730B11C0DF10702214456
:100A40003846FFF756FA9DF80730042BC5D000232F
:100A500044F82530C1E7132221460348FFF7B9FBCC
:100A6000BBE700BF4038002018E4020808B516F0C4
:100A700071FBBDE80840FFF713BB0148F6E700BF74
:100A80001EE402087FB50346FFF71EFA044630B1A4
:100A9000002218490120FFF7A1FC04B070BD6A468E
:100AA0001549154E184618F0BBFD01AD78B1032C61
:100AB00002D1FFF7E2FFF0E718F056FD6A4645F86D
:100AC00024003146002018F0ABFD0134EEE7032C82
:100AD000EFD101AC70CC32462946E0B212F004F9F5
:100AE0000028E6D033462A4621460448FFF764FB37
:100AF000D3E700BF744F002083E8020875E30208C3
:100B000070B50646FFF7E0F9044628B100220F4908
:100B10000120BDE87040DBE4304618F025FD0F28C9
:100B200005460ADC3046FFF7D7F90146284612F0A1
:100B300003F948B9BDE870409FE721460F220448F9
:100B4000BDE87040FFF745BB70BD00BFF44F00200B
:100B500018E4020870B50646FFF7B6F9044628B156
:100B600000220F490120BDE87040EDE4304618F046
:100B7000FBFC1F2805460ADC3046FFF7ADF90146AD
:100B8000284611F0DBFF48B9BDE8704075E7214603
:100B90001F220448BDE87040FFF71BBB70BD00BFBB
:100BA000744F002018E40208F8B50546FFF78CF9E9
:100BB000064628B1002226490120BDE8F840FDE4A0
:100BC000244928461AF035FF68B9214B4FF47A7151
:100BD0004FF4FA6219805A809980DA8019815A811B
:100BE0009981DA81F8BD284618F0BEFC0328044636
:100BF00027D82846FFF770F9064650B118F0B4FC24
:100C0000012705463046FFF767F928B9BDE8F840E7
:100C100033E705460746F5E718F0A6FC002FF5D0A8
:100C2000A5F2EE2240F2DC539A42EFD8A0F2EE2277
:100C30009A42EBD8064B23F8245003EB84035880E8
:100C4000F8BD314603220448BDE8F840FFF7C1BAB9
:100C5000205600202AE4020830E402082DE9F0477B
:100C6000484E494FDFF8388104462046FFF72CF9FB
:100C7000814628B1002245490120BDE8F047D7E46C
:100C80000522314620461AF017FF40B93F4900229D
:100C90004318103080281A60FAD1BDE8F08704228A
:100CA000394620461AF008FF054620460DBBFFF7DF
:100CB00013F98146002862D017F0E6FC2C465FFA53
:100CC00080FA58F824501DB93148BDE8F047CDE608
:100CD0005246294648461AF0EFFE40B920460FF02A
:100CE0005BF829462B482C4CFFF766FABDE7013428
:100CF000E7E718F039FC0728054639D82046FFF702
:100D0000EBF8064640B3F3F705F9204B03EB051368
:100D100083ED000A01243046FFF7DEF8064638B1BD
:100D2000F3F7F8F8194B03EB051383ED010A0134CF
:100D30003046FFF7D1F8064638B1F3F7EBF8134B1E
:100D400003EB051383ED020A01343046FFF7C4F8C4
:100D500020B9BDE8F04790E60446DCE7F3F7DAF89F
:100D60000A4B032C03EB051585ED030AF1D181E74E
:100D7000494607220948BDE8F047FFF72ABABDE80F
:100D8000F08700BF2AE4020838E402083C4400204F
:100D90003DE402084AE402087809030818E402085E
:100DA00094D30208F7B50746FFF78EF8044630B132
:100DB000002236490120FFF7C9FC03B0F0BD3846D8
:100DC00018F0D2FB0E28054659DC06264643781C4F
:100DD0008DF80740FFF780F82C4C074650B118F00B
:100DE000C3FB032806D8A31958719DF807300133B7
:100DF0008DF807303846FFF76FF8074658B118F0FE
:100E0000B3FB0D2807D806236B43E0549DF8073049
:100E100001338DF80730711C0DF10702214438466B
:100E2000FFF767F8FFF758F8074660B118F09CFB2A
:100E3000182808D8062303FB0543D8709DF807300F
:100E400001338DF807303846FFF746F860B118F0E7
:100E50008BFB0D2808D8062303FB05459DF80730BA
:100E6000287101338DF807309DF80730062BA4D088
:100E7000A2190023A3519380FFF7FFFD9DE70E22E7
:100E800021460348FFF7A5F997E700BF753A002010
:100E900018E402082DE9F04F85B00346FFF714F877
:100EA000064620B1FFF7E9FD05B0BDE8F08F03AAC3
:100EB0004849DFF84C91DFF84CA1DFF84CB11846F7
:100EC00018F0AEFB3446054637464FF0FF38BDB943
:100ED00041484146FFF753F8404B93F906204FFA3B
:100EE00088F082425AD093F90E20824255D093F96D
:100EF000162082426BD09FBB3948FFF7B7FDD3E77E
:100F0000012E0ED0022E11D01EB9284618F02CFB4F
:100F1000804603AA2F49002018F082FB01360546BF
:100F2000D5E7284618F020FB0746F2E74946284651
:100F30001AF010FE20B92B4928461AF00BFE08B112
:100F400044F00104514628461AF004FE28B95946D7
:100F500028461AF0FFFD0028DBD044F00204D8E751
:100F6000002C08BF03240022E4B2019200943B4607
:100F700011460DF04BFE054618B91B48FFF776FDEC
:100F800092E739461948FEF7FAFF1948FFF76EFD58
:100F9000184B294618680EF077FE012553F8355096
:100FA000002DA8D01448FFF761FD54B169798C4237
:100FB00007D012482246FEF7E2FFE1B22846FDF7CD
:100FC0006DF9EB6A002BE0D00023EB62DDE7022530
:100FD000E4E700BF83E8020860E402089C4E0020BA
:100FE00069E4020857E402087FE4020894E4020876
:100FF000D5E4020890280020A9E40208B7E402081A
:1010000054E402085AE402085DE402082DE9F743BB
:101010000346FEF759FF044638B139490022012042
:1010200003B0BDE8F043FFF7F3BB00900190184612
:101030005E1C18F099FA324B93F9022040B28242BA
:101040001A4654D093F90A1081424FD093F91230C6
:10105000834252D025463046FEF73EFF074628B170
:1010600018F082FA0135ADF80000EDB2DFF8948097
:1010700000263846FEF730FF0746C8B118F074FA6C
:1010800081460EF03BF858F82030994510D1022ED9
:1010900019D0032E1CD0431E012EDBB20ED00B2B19
:1010A00003D88DF803000135EDB20136042EE0D1EE
:1010B000052D14D803B0BDE8F043DEE4042BF4D8CA
:1010C0008DF80400EFE70528EFD88DF80600EAE771
:1010D000831EDBB20D2BE8D88DF80500E3E76B46E5
:1010E00003CB2060616003B0BDE8F083012402EB14
:1010F000C4048DF802000125ADE70224F7E700BF24
:101100004C5700206CDC0208F7B50646FEF7DCFE03
:10111000054658B1002401A920460EF04BFB0134CE
:10112000FFF7F2FF122CF6D103B0F0BD304618F0F5
:101130001BFAC4B2112C5CD8701CFEF7CDFE304DEA
:101140000746C0B92F4B13F814108A1E5142514163
:101150002C4B13F81420AA5C002945D003EB440360
:1011600040F2EE215B78192000FB0313214626484C
:10117000FFF722F8D8E7017828461AF087FC50B12B
:10118000224A401B032C8CBF0323002352FA80F019
:10119000C65C032E02D1FFF770FCC5E73846FEF7A8
:1011A0009BFEF0B1022EF6D118F0DEF940F6CA022D
:1011B00080B29042134BA8BF104640F2EE229042FC
:1011C00003EB4403B8BF1046A0F2EE20192290FBB7
:1011D000F2F05870B31E594259410A4B03F814609B
:1011E000B6E7022EF6D1D6E721460948FEF7E4FF1E
:1011F0009AE7112229460748FEF7EBFF94E700BF64
:101200007CD4020854560020F6E402083CBF0208D1
:1012100006E5020830E4020830B4034600F1600538
:10122000064C07CC0C3343F80C0C43F8081C43F86D
:10123000042CAB42F4D130BC704700BF44BF02085D
:101240000121114B817370B40022042440F2DC565A
:1012500032250907C47306804580828103F1640446
:1012600003D581181D790D7101329C4203F11403DD
:1012700008D0072A06DC99790907F2D49C4203F1C9
:101280001403F6D170BC7047BCDC020870B5064E82
:10129000044600F1EA054E2220463146144418F077
:1012A0008BF9AC42F7D170BD50BF02082DE9F04F69
:1012B000AB4E3378192B91B007D80121A94A01FA16
:1012C00003F31A40002A40F06B81A74BA74F02930B
:1012D00006F16408029B1B689C065FD4B7F90050B6
:1012E000A34CA249234601E0B1F90050B3F9042010
:1012F000B3F90600954203F10C0303DBA842024652
:10130000A8BF2A46984521F8022BEDD1DFF8889234
:10131000B9F80C3013B3974DDFF880A205F110082F
:10132000B5F9023000EE103A5046B8EEC00AF1F7B7
:10133000E3FA18F0B5FAB4F90430B4F9062000B2B3
:1013400098420AF1240A04F10C0403DB824213469A
:10135000A8BF034625F8023FA845E1D13378013BF9
:10136000182B00F22D82DFE813F0E8002B022B028D
:1013700054002B022B022B02DB002B022B022B0230
:101380002B022B029E002B022B022B022B022B0284
:101390005400CC002B022B029E00E800F37BFF2BB5
:1013A00003D0754A12789A4279D8B6F90C50F37E78
:1013B0003D80FF2B03D0704A12789A426BD8B6F961
:1013C00018407C80082015F0FFFE002888D096F891
:1013D000F430012B00F0F681684B96F90E20B3F83B
:1013E00002E01888664996F91A3012FB0EF213FBD8
:1013F00000F381FB02E0D217C2EB201281FB030154
:10140000DB171544C3EB21132DB21C443D807C80B7
:1014100066E75C4BB7F908101A6802B111609B6966
:10142000B7F90A2003B11A60029B1B689A0600F103
:1014300029820224D90202D411B0BDE8F08F99F8B4
:101440000F60112EF8D8504B059333F9163000EE8B
:10145000103A751C06F10E07B8EEC00A204608F0D7
:1014600019FFEDB2A61BFFB2DDF8148000E025469F
:101470006C1CA819122DE4B2C0B2DDD038F91530B9
:1014800000EE103AB8EEC00A08F004FFBC42EED1FC
:1014900011B0BDE8F08F3C4A32F9134091E73A4A67
:1014A00032F9135083E7394D002435F9023F00EE3D
:1014B000103AE0B2B8EEC00A013408F0EBFE062C98
:1014C000F3D1029B1B68980602D43278052AB1D169
:1014D000651CA31C2046EDB2DCB2B7F9003000EE6B
:1014E000103AB8EEC00A08F0D5FEB7F9023000EEA7
:1014F000103A2846B8EEC00A08F0CCFE029B1B68E2
:1015000098E7234D002435F9023B00EE103AE0B293
:10151000B8EEC00A013408F0BDFE042CF3D1D0E7C8
:10152000184BB7F906101A6802B111609B69B7F938
:101530000820002B7FF477AF76E799F80E30002B68
:1015400040F0A481134B1B7813F0010340F09E81FF
:101550000C4A1268002A00F0A18113600124B0E750
:1015600034240020324130036C4900203036002002
:10157000382400202E360020903F0020883F002095
:101580001F85EB517857002040450020323600205F
:1015900036360020FE56002068570020F054002008
:1015A000BF4B1B88DF0540F19B81BE4BBE4AD3ED8C
:1015B000006A93ED017AD3ED027ABC4B0593FDEE00
:1015C000E66ABDEEC77AFDEEE77AB3F90650B84B8E
:1015D000118B029316EE900A17EE102A17EE903A2E
:1015E000ADF82400ADF82620ADF82830B14BB24C50
:1015F000B3F90220B3F90030B048D4ED007A9FED82
:10160000B07A059C03F5E16702F5E1624FF47A7365
:1016100003FB02F203FB07F377EEC77A80FB02E7D6
:1016200080FB03E0174418442488D217DB17C2EB71
:10163000E722C3EBE023059FFDEEE77A641AA3F5EA
:10164000FA733846ADF83E30ADF82C4017EE903ABC
:10165000059CB7F802C0B7F804E040893F89ADF8AF
:101660002A30A2F5FA72E389ADF83C20A2896D1AFE
:10167000521AACEB010CAEEB010E7F1A401A591A4C
:10168000904BADF83820ADF83A10ADF83250ADF8C7
:101690002EC00693ADF830E0ADF83470ADF83600EA
:1016A00003F11001002223F8022F9942FBD1737835
:1016B0000493DFF82882844F002B00F0BE800023C3
:1016C000454608F1700BCDF81C8098463EE010AB03
:1016D00003EB4E0434F91C4CABF80040014495F97F
:1016E00002C0012306EB810103FA0EFE774B496825
:1016F0001CFB04F483FB043CE417019B1EEA010F6E
:10170000C4EB6C140CBF01214FF0FF319C420EDB87
:10171000039B02FB03F26D4B83FB02E3D217C2EB88
:101720006313A3EB09031BB2A342A8BF234637F8F8
:10173000102003FB012327F81030049B08F1010857
:10174000984505F107050BF1020B74DAA87900281A
:1017500059D1287895F90520039241000C1806EB21
:10176000840495F904306289248995F803C095F8BA
:1017700001E0121B92B2554C02FB03F384FB03946D
:10178000DB17C3EB64134FEA5209A3EB09031BB247
:101790000193BCF1000F9AD010AB03EB4E0ABBF9DA
:1017A00000403AF91CAC544536DAA444644503DCE5
:1017B000E2455446A8BF644624B2ABF800408DE72A
:1017C00000247EE63B4A96F91AE0108896F90E301E
:1017D0003E49B2F902201EFB00F05B4202FB03F21D
:1017E00081FB00E31B1181FB02E1C017D217C2EBA2
:1017F0002112C11A11441B1A6D1A1A442DB2144435
:101800003D807C806CE51630C0B215F0DDFC002810
:101810009FD1ABF8000090E77FF760AFA4EB0C0C12
:10182000D44503DB6445A8BF6446A2460FFA8AF498
:10183000ABF8004052E7DDF81C80254B25491C78A9
:101840002248069DDDF814E008E03EF912200C3134
:101850001344884525F8023F3FF43CADB5F802C07B
:1018600091F90A30CA7A13FB0CF380FB039CFF2A20
:101870004FEAE373C3EB6C1301D0A242E5D3B1F995
:101880000820E4E703250424022026E6124BB7F9DA
:101890000A201B6813B11A60012412E6012410E625
:1018A00072500020CC3C0020B84E00204045002063
:1018B0006C490020883F002040360020C5B3A2912B
:1018C0000080BB442E360020303600201F85EB51AF
:1018D000903F0020382400207857002098240020D2
:1018E000294A2A4B2A4992ED007AD3ED003AD2EDEB
:1018F000017A93ED014A91ED005AD2ED026AD3EDDF
:10190000024AD1ED015A9FED236A234B029337EE31
:10191000237A77EE847A37EE057A76EEA46A77EE4C
:10192000A57A27EE067A66EE866A67EE867A19460B
:10193000BDEEC77AFDEEE66AFDEEE77A17EE102AF5
:101940000968CDED016A17EE903AADF82420CD0478
:10195000BDF90420ADF82630ADF8282006D40F4A92
:101960000F4B0592198BB2F906503FE60B4B0593CE
:1019700019460B4BB1F90650198B8D42BCBF524230
:10198000ADF8282032E600BFE0350020EC3500201D
:10199000F83500203333333F6C49002040450020A8
:1019A000B84E002070B4124C0130234604F170018F
:1019B00000229A719A705A7003F8072B8B42F8D163
:1019C0000C4B03EBC00090F85C5075B1066EC5EB94
:1019D000C5050023F218E1181068E050073390881D
:1019E00092798A719D428880F4D170BC704700BFA3
:1019F0002C25002044BF0208F8B5104D00242146D4
:101A000005F16400702205F1F8076C701AF009F80E
:101A10002146A7F194047B18081993F902205AB1C2
:101A20001E686A780E5107319E889B798680013244
:101A300070296A708371EED1F8BD00BF3424002094
:101A4000F0B41D4FD7F86831CBB13A781B4B03EB9C
:101A5000C2031E6E93F85C507D7086B17DB1C5EBFC
:101A6000C505002307F16400F218C1181468C450BA
:101A70000733948892798A71AB428C80F4D13B7899
:101A8000082B0CD00E2B0AD0182B0ED00C490A783C
:101A9000192B22F010020A700CD0F0BC7047084AD3
:101AA000137843F010031370F7E7054A137843F0F7
:101AB00010031370F0BC9FE73424002044BF0208D9
:101AC000C432002010B40E490E4A0C780E480F4B59
:101AD000006802EBC40203405278C1F8682113B1D8
:101AE0000123C1F868310A4B40F2DC5103F11002C6
:101AF00023F8021F9A42FBD15DF8044B704700BFE8
:101B0000342400208CD602086C49002020001000EC
:101B10002E360020F8B5BE4C438C2DED068BD4ED4F
:101B20005B8AB6EE007AC7EE287A0646FCEEE77AC4
:101B300017EE905A9D4219D2828C954200F2BB80DA
:101B4000B44BC4F87031338C13B19D4280F08F8058
:101B5000B04BC4F8C431F38B13B19D4280F0B08018
:101B6000BDEC068BAB4BC4F82C32F8BD002BE7D094
:101B7000828C002AE4D007EE903AB8EE678A07EE2E
:101B8000902AB8EE670AA44BC4F8703188EE000AB8
:101B900017F07CFE70EE009AB0EE000AF0EE690AD3
:101BA00017F0EEFFF6EE000A69EEA00AB0EE409ADA
:101BB000B0EE000A17F0E4FF984B9FED997AD3ED51
:101BC000007AF8EE677AB0EE40AA67EE877A27EEE1
:101BD000888AB0EE480A17F0AFFEF0EE409AB0EEF9
:101BE000480A17F00BFEF7EE006A39EE669AF8EE37
:101BF000007A8AEE097A8B4BC4F874312433C4F826
